:020000040800F2
:1000000000200010354103086114030865590008F9
:100010005D14030859140308551403080000000078
:100020000000000000000000000000005114030860
:100030004D14030800000000491403085556000839
:100040009D4103089D4103089D4103089D4103080C
:100050009D4103089D410308410800086D090008FF
:1000600031090008F5080008B90800082120000837
:100070001120000801200008F11F0008E11F0008FE
:10008000CD1F0008B91F00089D4103089D410308CA
:10009000091903089D4103089D4103087D080008D4
:1000A0009D410308FD4D0008AD4D00080D4E0008B0
:1000B000ED4D0008DD4D00089D4103089D410308FA
:1000C0009D4103089D4103089D4103089D4103088C
:1000D0009D410308D95700085D570008E156000804
:1000E000050800089D410308391403089D410308D1
:1000F000BD4D00089D410308CD4D00089D410308FA
:100100000000000000000000000000009D41030806
:100110009D4103089D410308A96802088D680208F3
:10012000A51F0008911F00087D1F0008691F000817
:10013000551F00089D41030800000000000000005A
:100140009D4103089D4103089D41030800000000F4
:10015000000000000000000000000000000000009F
:1001600000000000000000009D4103089D410308BD
:100170009D41030800000000000000000000000096
:08018000000000009D4103088E
:10018800152303701623C370172383712D2343701F
:100198002E2303712F23C37170470B4B984206D04F
:1001A800A3F5784398420DD04FF0FF3070470022F6
:1001B800064B03EB02135A89013292B25A815889CD
:1001C80080B270470122F3E700300140702F002011
:1001D800002870B51EDB0928044620DD012303EB47
:1001E80083035B00B0FBF3F2092AF8D87BB10E4E0B
:1001F800B4FBF3F00928CCBF57223022A6FB03E555
:10020800024403FB1044EB0801F8012BF0D1002352
:100218000B7070BD2D230B7040420131DBE730308D
:1002280001F8010BF3E700BFCDCCCCCC884230B449
:100238004FF001042ED301FB04F4B0FBF4F58D421A
:10024800F9D284B1AAB901E0B0FBF4F5092DCCBF0D
:10025800572230222A4404FB150003F8012BB4FB73
:10026800F1F4002CF0D100221A7030BC7047B0FBBA
:10027800F4F5092DCCBF372230222A4404FB15009F
:1002880003F8012BB4FBF1F4002CF0D100221A7012
:1002980030BC70470546002AEBD1D7E72DE9F04777
:1002A80014461D46064600234FF47A722046294616
:1002B80033F068FDDFF840814B4A4C4F88FB003132
:1002C8000144C31782FB002EC3EB611188FB012890
:1002D80087FB00278644464AC3EBEE2EC1EB011C80
:1002E80082FB0E29A0EB8C0C0744424A86F806C014
:1002F800C3EB27474FEAEE7C08EB010ACCEBA90CCD
:1003080082FB07824FEAE1780CEB4C0CC8EB6A18C9
:10031800AEEBCC0EC8EB0818DFF8E0C086F804E0B6
:10032800A1EB880171718CFB0010F917C1EBE21287
:1003380040F2B55101FB1272C3EBE050B2F5896F80
:100348004FEA80073CDA40F2DA239A4242DCB2F5FF
:10035800B77FB4BF4FF0000C4FF0010C4FEA4C09C7
:10036800DFF89C8009EB0C0308EBC3031FFA8CFE33
:10037800D88A09EB0C0108EBC10116310B2301E007
:1003880031F8020D824218DA013BF9D1CC4401233D
:1003980038F83C00B37007F2B2770132121ABE4443
:1003A800F270A6F800E0204629464FF47A7200233E
:1003B80033F0E8FC3281BDE8F0870133DBB2E9E7CE
:1003C8004FF0030EF44640F29650DFF834804FF0B9
:1003D8000609CEE74FF0020EDFF82480F44640F21B
:1003E80029404FF00409C4E7C5B3A29107452EC2BE
:1003F800ABAAAA2A73B06D1689888888792D03114B
:100408003057030803685A1C0260197070472DE9B9
:10041800F047089C2578002B804689460CBF4FF092
:10042800200A4FF0300A661C35B3002A29DD33460E
:1004380001E0024698B113F8011B501E0029F8D1BB
:10044800971E60B13D46013D51464046C8476B1C6A
:10045800002BF8DC257827EAE770013055B1041B3A
:1004680029464046C847301916F8015B002DF7D1D8
:10047800BDE8F087BDE8F087002A04DC2846BDE81F
:10048800F0870020EBE7571EDCE783684268D0ED71
:10049800037A00EB83010133934281ED040A836000
:1004A80004BF0023836000EB830393ED047A0368A1
:1004B80070EE277A9A42C0ED037A77EEC77AC0EDDC
:1004C800037A0CDA013307EE103AF8EEC76AB7EE92
:1004D800007A87EEA60A036030EE070A704707EE37
:1004E800102AB8EEC77A87EE870A704790ED057A2A
:1004F80090ED004AD0ED066AD0ED014AD0ED047ABD
:1005080090ED035AD0ED025AA4EE007AB0EE406A9C
:10051800B0EE470AB0EE667AA6EE247A67EEC07AA5
:10052800A0EE457AE6EE257A80ED057AC0ED067AEA
:100538007047D0ED057A90ED013AD0ED003AD0ED54
:10054800064A90ED024A90ED077A90ED035A90ED35
:10055800086AD0ED045AC0ED067AF0EE406A27EE3C
:10056800830AC0ED056AA3EEA60A80ED087AA4EE18
:10057800240AA5EE470AA5EEC60A80ED070A7047C9
:10058800D0ED007A90ED017A30EE670AE7EE007A56
:10059800B0EE670AC0ED007A704770470A4491428E
:1005A80014D030B40139551E41F2210211F8014F1F
:1005B800082380EA042004044CBF82EA400040007B
:1005C800013B80B2F7D18D42F0D130BC7047012396
:1005D80080F84530704790F8203033B1012B03D1B3
:1005E8004FF400638382704770474FF480638382BF
:1005F800704770B40468037B2268022101FA03F390
:100608001A4213D042690A495C2000FB02124FF6D5
:10061800FE7650685289C5680068296831402960AB
:10062800C168D24392B20A40C260636070BC70472E
:100638003857002030B40A4B1D7875B1094B00209B
:1006480003EBC5051A6899885062D4682143D160C4
:10065800083323F8040CAB42F4D130BC704700BF18
:10066800185A00201C5A002010B40268047B116834
:100678000223A340194209D00649406800240C709F
:1006880001684FF6FE742140016053605DF8044B29
:10069800704700BF744100200023262203600270C7
:1006A80027228270012243600271837170472DE90D
:1006B800F341056906460F467DBBD0F80080C8F3B4
:1006C8000A0323B30023D6F8008001932EF07EFDA1
:1006D800042819D1214C236943F001032361BBB2DB
:1006E800A8F800302EF072FD04282ED108F102037C
:1006F8000193019B3F0C1F802EF068FD236904289D
:1007080023F00103236125D06FF0010505E02EF0E9
:100718005DFD042805D04FF0FF35284602B0BDE83E
:10072800F0810E4C236943F002032361C4F814805E
:10073800236943F0400323612EF048FD2369042810
:1007480023F002032361BDD0E5E7236923F0010309
:100758002361D9E7336804333360DEE700200240C1
:10076800F8B504460D468E180027B54201D1206918
:10077800F8BDE368591CE160234415F8012B1A728F
:100788000429F2D1A1682046FFF791FFE7602061B4
:10079800EBE7024B186805F0C1B800BF4C230020F6
:1007A80010B490E80600047B40690223A3404B6024
:1007B80013685DF8044B4FF6FE710B40136005F0AB
:1007C80045B810B1036882881A85704710B103686C
:1007D80082889A61704738B100298388026814BFFB
:1007E800002110218B409361704730B103688288E3
:1007F8001B8A1A4214BF0120002070472DE9F041DE
:100808000B4E346873691C400FD0DFF8288001272D
:10081800B4FA84F3C3F11F0307FA03F558F8230069
:1008280003689847AC437561F2D1BDE8F08100BF19
:1008380000040140C02200202DE9F0410B4E34682D
:1008480073691C400FD0DFF828800127B4FA84F3BD
:10085800C3F11F0307FA03F558F823000368984704
:10086800AC437561F2D1BDE8F08100BF00040140DE
:10087800C02200202DE9F0410B4E346873691C40FA
:100888000FD0DFF828800127B4FA84F3C3F11F03DF
:1008980007FA03F558F8230003689847AC437561D5
:1008A800F2D1BDE8F08100BF00040140C022002061
:1008B8002DE9F0410B4E346873691C400FD0DFF806
:1008C80028800127B4FA84F3C3F11F0307FA03F55C
:1008D80058F8230003689847AC437561F2D1BDE826
:1008E800F08100BF00040140C02200202DE9F04142
:1008F8000B4E346873691C400FD0DFF8288001273D
:10090800B4FA84F3C3F11F0307FA03F558F8230078
:1009180003689847AC437561F2D1BDE8F08100BF28
:1009280000040140C02200202DE9F0410B4E34683C
:1009380073691C400FD0DFF828800127B4FA84F3CC
:10094800C3F11F0307FA03F558F823000368984713
:10095800AC437561F2D1BDE8F08100BF00040140ED
:10096800C02200202DE9F0410B4E346873691C4009
:100978000FD0DFF828800127B4FA84F3C3F11F03EE
:1009880007FA03F558F8230003689847AC437561E4
:10099800F2D1BDE8F08100BF00040140C022002070
:1009A800084A936910B5084C43F001039361204647
:1009B8004022002134F049FE4FF0FF332364C4F88D
:1009C800433010BD00100240C022002010B58B68D3
:1009D8000160044698470022FF230121A273637334
:1009E800217310BD03681B6A184770B44E1C056854
:1009F800C2728672AC69A44670BC60472DE9F041AA
:100A0800044618460D461646984632F0F1FC27680B
:100A1800E6722844A07229467D694346324620463C
:100A2800AC46BDE8F0416047036810B504461B6852
:100A38009847236820469B689847A37B0133A37394
:100A480010BD03681B69184710B5036804469B6806
:100A58009847FF2301226373227310BD427A02B9BB
:100A6800704710B504460368406804F10A019847C6
:100A78000023637210BD437A5A1C0344D2B24272F7
:100A88009972037A934200D802B9704710B50446A8
:100A98000368406804F10A0198470023637210BD97
:100AA80098B10B4B012210B402FA01F103F175045D
:100AB80002E00333A34209D01A788242F9D15A7866
:100AC8000A42F6D001205DF8044B70470020FAE78F
:100AD8009057030830B40A4D002305F1600401E083
:100AE800272B0AD003EB43020133A15C8142F7D1E3
:100AF8002A4430BC92F862007047002030BC70472E
:100B08003057030870B5448806460D46C4F30B04F5
:100B180022460021284634F098FD3369094A934259
:100B280009D3094A934206D2224628461946BDE807
:100B3800704033F0F9BB23B121462846BDE8704028
:100B4800184770BD70C3030860C40308064B074903
:100B58008B4202D30023184670471A88C2F30B024F
:100B68009042F8D01433F3E7C0BE030870C30308FB
:100B7800024A136823EA000010607047508E002074
:100B8800F8B5174D2B78A52B28D16B78BE2B25D11E
:100B9800022229464FF6FF70FFF700FD114FAC1CEB
:100BA80022884AB1A618BE4218D2052A16D921466B
:100BB800FFF7F4FC3446F3E721460222FFF7EEFC88
:100BC8000222A118FFF7EAFC0634074B641B1C80BD
:100BD80041F60F53C31A58425841F8BD0020F8BDDA
:100BE80000F0030800000408663100202DE9F04FEA
:100BF800DFF848914C4F8BB00326A7EB0907182262
:100C0800002104A834F021FD484BCDF81090059739
:100C18001A69120604D5464A5A6002F188325A60A7
:100C280001228DF824203422DA60424B424C1B8882
:100C3800ADF800300222694604A8FFF791FD0222B0
:100C480069464FF6FF70FFF7A9FCDFF8F4A080466D
:100C58004FF0000B544536D30AAC002524F8245D28
:100C68000222214604A8FFF77BFD022221464046C6
:100C7800FFF794FC40BAC043ADF80800022202A96D
:100C880004A8FFF76DFD079860B106ABC0F1040238
:100C98002946184434F0D9FC069904A8FFF707FD43
:100CA800079508909DF82430089A23B11F490B69CD
:100CB80043F080030B61013E2DD0002A9FD1FFF73E
:100CC8005FFF50B32CE065888DF80DB0C5F30B05B8
:100CD800AB1DADF808302388C3F30B02ADF80A202A
:100CE8001B0B062202A904A88DF80C30FFF738FD6B
:100CF800062202A94046FFF751FC616880462A4651
:100D080004A8FFF72DFD616840462A46FFF746FC18
:100D1800143480469EE7002AD1D0052002F0CAFE8E
:100D28000BB0BDE8F08F00BF0000040800200240AF
:100D38002301674505580308C0BE030800F00308EF
:100D480070C303080378202B024600F10100F9D094
:100D5800092BF7D02D2B2CD02B2B03BF5378B7EEB4
:100D6800000A0246B7EE000AA3F13001C8B209280A
:100D78009FED467A10D8F2EE046A07EE901AF8EE64
:100D8800E77A12F8013FE7EE267AA3F13001C8B2FC
:100D98000928B0EE677AF0D92E2B4CD003F0DF0388
:100DA800452B0BD0F7EE007A67EE276A20EE260A6D
:100DB80070475378BFEE000A0246D5E710B4517861
:100DC8002D2959D02B290ABF9178501C901C00243A
:100DD800A1F13003092B53D8002303EB830301EB64
:100DE800430310F8011FA1F13002092AA3F13003CF
:100DF800F3D9B3F59A7F28BF4FF49A73072B42D9DA
:100E0800DFED236A1A46F7EE007A083A072A67EEFA
:100E1800A67AFAD803F007032BB1F2EE046A013B75
:100E280067EEA67AFBD124B3C7EE276A5DF8044BB8
:100E380020EE260A70475378A3F13001C8B209287A
:100E480002F10102AAD8F2EE046AF0EE665A07EE41
:100E5800901AF8EEE77A12F8013F87EEA66AA3F136
:100E68003001C8B2092866EEA56A37EE067AEED9CF
:100E780094E767EE276AD9E7901C91780124A7E7E1
:100E8800F7EE007ACFE7F7EE007AC5E7000000003A
:100E980020BCBE4CB5EEC00ADFED317AF1EE10FA97
:100EA800CCBF30EE270A30EE670ADFED2E7A20EE4F
:100EB800270A30B5FDEEC07A87B017EE904A05468E
:100EC80084EAE470002303A9A0EBE4700193009383
:100ED80002932AF0DFFF002CACBF20232D2303A8A8
:100EE8008DF8003032F084FA012803A924D00228B2
:100EF8002DD0032805BF3023684668468DF8013099
:100F080034F0ABFB684632F073FA0338C4B22246B9
:100F18006946284634F0D8FB00232B55284632F082
:100F280067FA2E22431C2A540DEB0401E81834F00A
:100F3800B1FB284607B030BD302368468DF8013034
:100F48008DF802308DF8033034F087FBDAE7302370
:100F580068468DF801308DF8023034F07EFBD1E719
:100F68006F12033A00007A442DE9F041064615460F
:100F78000846B6FBF2F43CB905FB1464124B1B5D42
:100F880000F8013BBDE8F081B4FBF2F767B90E4BFE
:100F980005FB174705FB1464DA5D00F8012B1B5DA0
:100FA80000F8013BBDE8F081B7FBF2F8B8F1000F9B
:100FB80002D04046FFF7D8FF05FB1878024B13F81C
:100FC800082000F8012BE3E718850308104B2DE9EA
:100FD8003048D3E9004554EA05020BD10346012203
:100FE80000201871587198719A70DA7018801881F9
:100FF800BDE83088074B1A6814EB020B45F1000C6A
:101008005A466346FFF74AF90120BDE8308800BF19
:10101800B8240020B0850020F0B402888578154FE8
:10102800C37804794179A2F2B27202F0030606EBA2
:101038004606013D05EB8605013B37F815608579C5
:10104800008940F2B557920807FB0232931903EB67
:10105800430304EBC303C3EB031301EB8303C3EBA9
:10106800031305EB830300214FF47A72C2FB0301DB
:10107800F0BC704730570308FAB170B48E180446B4
:1010880003E0101A14D1B14214D014F8012BA2F1C4
:101098004103192B11F8013BA3F1410598BF2032F8
:1010A800192D03F12000ECD9D01A01D1002BEAD177
:1010B80070BC7047002070BC7047104670474FF0F6
:1010C800FF32FFF7D9BFA0F16103192B98BF203871
:1010D8007047A0F14103192B98BF20307047202892
:1010E80005D0093804288CBF002001207047012052
:1010F8007047613819288CBF00200120704741389B
:1011080019288CBF002001207047303809288CBF6F
:10111800002001207047A0F13003092B07D920F0E7
:101128002000413819288CBF002001207047012079
:10113800704730B402681146531C036011F8024B23
:101148000160D31C517803609378151D05601B045A
:1011580043EA0123D078234343EA006030BC704758
:101168000368591C1A46016012F8021B026058787D
:1011780041EA0020704703685A1C026018787047DB
:1011880038B504460068154633F0CEF822682A447C
:10119800226038BD036810B40A0A5C1C04601A7027
:1011A80003685A1C026019705DF8044B70470368A5
:1011B8005A1C026010B4197003680A0A5C1C0460A7
:1011C8001A7003680A0C5C1C04601A700368090E24
:1011D8005A1C026019705DF8044B704703685A1C6A
:1011E800026019700368090A5A1C02601970704776
:1011F8002DE9F047002488B080460F461E46A146D8
:1012080005AD531C0393117839B3252933D1931CA9
:10121800CDF810900393507830284ED04FF0000A44
:10122800A0F13003DBB2092B42D96C2819D064280D
:1012380000F0938024D825281CD063D9582876D06C
:1012480063281BD131784046B847039A531C03934F
:101258001178043601340029D7D1204608B0BDE8FA
:10126800F087039B5A1C03921B78642B7CD02AD8E6
:10127800252B54D1252140460134B847039AC0E7AD
:10128800732833D044D975284FD106F1040E30683D
:101298002B4600220A217646FEF7C8FF049A0095DD
:1012A800534639464046FFF7B2F8039A0444A8E784
:1012B80004AA03A92DF0F8FFB7E7D31C039390788D
:1012C8004FF0010AACE7732B10D05BD9752B3AD0DD
:1012D800782B96D1A3F15802B2FA82F230685209FB
:1012E8002B4610210436FEF7A1FFD7E73368049A8E
:1012F8000093394600234046FFF789F80436044432
:10130800039A7EE70028B9D1204608B0BDE8F087E7
:101318006E28B3D1039A336804361C6071E72AD962
:10132800582BD7D0632B8DD06BE77828A6D1A0F1A6
:101338005802B2FA82F2306852092B461021FEF7A1
:1013480075FF0436AAE706F1040E30682B46002222
:101358000A217646FEF76AFFA0E7331D3068294662
:101368001E46FEF735FF99E7331D306829461E46AD
:10137800FEF72EFF92E7002B7FF443AF204608B01C
:10138800BDE8F0876E2BC6D03BE70EB400B584B03D
:1013980005AB019053F8042B0649039301A8FFF706
:1013A80027FF019B00221A7004B05DF804EB03B01C
:1013B800704700BF0D0400082DE9F04707468CB0C0
:1013C8001E469246002A6AD1154614460A8840F2FB
:1013D800B1739A423AD98B78581E0B2836D891F8AF
:1013E80003E00EF1FF301E2830D891F804C0BCF19C
:1013F800170F2BD891F80590B9F13B0F26D88879AB
:101408003B2823D8B1F80880B8F57A7F1ED24FF070
:101418000108002E34D109890491002CB4BF2D2174
:101428002B21002CB8BF6442039005910795CDF895
:101438000890CDF804C0CDF800E0384606942F494E
:10144800FFF7A3FF40460CB0BDE8F0870023012159
:1014580018468E46ADF824308DF828308DF829309E
:101468008DF82A30ADF82C3099469C461A46984695
:101478008DF826108DF827100B4609A9002ECAD022
:101488000390CDF80890CDF804C0CDF800E03846B8
:101498001B49FFF77AFF40460CB0BDE8F087194CAE
:1014A80084FB0234A318D417C4EB6314C4EB0415EB
:1014B800A2EB85052DB2002D0846B8BF6D42FFF797
:1014C800ABFD4FF47A7200238046894632F05AFC0D
:1014D8003C230AFB030A4FF47A720023404649462C
:1014E80032F050FC4FF47A7192B20023C1FB0A2308
:1014F80009A8FEF7D3FE24B209A967E760850308A7
:1015080040850308898888880FB430B583B006AB56
:101518000B490C4853F8042B096800680193FFF73E
:1015280067FE094C0546206803685B6998470028F0
:10153800F9D0284603B0BDE8304004B0704700BF7A
:10154800402F0020442F00204C230020DFED2B7A71
:10155800B4EEE70AF1EE10FA4ADDDFED296A9FEDF5
:10156800297A01E0B0EE670AB4EEC70AF1EE10FA84
:1015780070EE667AF6DC9FED247AF4EEC77AF1EE27
:1015880010FA38D5DFED1E6A9FED207A01E0F0EE03
:10159800407AF4EEC77AF1EE10FA37EEA60AF6D4DE
:1015A800DFED1B7AB4EEE70AF1EE10FA14DDDFED99
:1015B800137A37EEC00A60EE006A9FED166A9FED57
:1015C800167ADFED167AA6EE867A20EE266AE6EE21
:1015D800877AA6EE270A7047DFED117AB4EEE70A9C
:1015E800F1EE10FA44BFDFED087A37EEC00AE2E701
:1015F800F0EE407ABFE7B0EE670AD1E7DB0F49406B
:10160800DB0FC940E4CB1641DB0F49C0E4CB16C160
:10161800DB0FC93F92E741B99730083C15A82ABEAD
:10162800DB0FC9BF09B909E0194690FBF1F301FBCB
:1016380013030846002BF7D1084670470146FBE71D
:1016480007EE901AF8EE677A9FED837A27EE800A04
:1016580020EE070AFDEEC07A17EE903A2033402BB1
:1016680000F28C80DFED7D7AB4EEE70AF1EE10FA35
:1016780040F3E880B0EE407A9FED796ADFED796A51
:1016880001E0B0EE677AB4EEE67AF1EE10FA77EEA2
:10169800467AF6DC9FED747AF4EEC77AF1EE10FA2A
:1016A80040F1CD809FED6E6ADFED706A01E0F0EEEB
:1016B800477AF4EEE67AF1EE10FA37EE867AF6D447
:1016C800DFED6B7AB4EEE77AF1EE10FA51DCDFED7C
:1016D800697AB4EEE77AF1EE10FA44BFDFED627A88
:1016E80037EEC77A27EE076ADFED635ADFED637AD4
:1016F800DFED636A9FED635AE6EE257A67EE065AD8
:10170800E6EE276AF7EE007AA5EEA67AF0EE675ABB
:10171800E7EE055AE7EE457A87EEA55ADFED547AEB
:1017280030EE277AFDEEC76A16EE903A2033402B4A
:1017380029D99FED557AF6EE006AB7EE006AF7EE02
:10174800004AC4EEA57A0023836143610362C36142
:1017580080ED045A67EEA66A27EE866A27EE877A36
:10176800C0ED006AC0ED026A80ED016A80ED037A7F
:101778007047DFED3A7A37EEC77AB3E7B7EE005A2B
:10178800F0EE455ACAE7B4EEE70AF1EE10FA5FDD6B
:101798009FED336ADFED336A01E0B0EE677AB4EEAD
:1017A800E67AF1EE10FA77EE467AF6DC9FED2E7ABD
:1017B800F4EEC77AF1EE10FA47D59FED296ADFED0E
:1017C8002B6A01E0F0EE477AF4EEE67AF1EE10FAD1
:1017D80037EE867AF6D4DFED267AB4EEE77AF1EEC4
:1017E80010FA27DCDFED237AB4EEE77AF1EE10FA8F
:1017F80044BFDFED1D7A37EEC77A27EE076ADFEDC3
:101808001E4ADFED1E6ADFED1E7AE6EE246A67EEF9
:10181800064AE6EE267AB7EE006AA4EEA77AF6EE56
:10182800006A36EE476AF8EE007A27EE277A66EE07
:10183800266A84E7DFED097A37EEC77ADDE7B0EE8E
:10184800677A3DE7F0EE407A24E7B0EE677AC2E7C0
:10185800F0EE477AAAE700BF27D4D236DB0F49401B
:10186800DB0FC940E4CB1641DB0F49C0E4CB16C1FE
:10187800DB0FC93FDB0FC9BF92E741B99730083C7E
:1018880015A82ABEF304353F0000008070B406682E
:101898008E4217D90139751E002311F8014F08220D
:1018A800634013F0800F4FEA430318BF83F0D5035A
:1018B800013ADBB2F5D18D42EFD1721C0260337070
:1018C80070BC70470023F8E710B44C09012250F8A7
:1018D800243001F01F0102FA01F10B4340F82430D3
:1018E8005DF8044B70474B0901F01F0150F82320A5
:1018F800012303FA01F1114214BF18460020704772
:101908000349044B2020082208835A75704700BFFA
:10191800888600205C86002008B540F2E93300E0A4
:101928009BB10289013B12F0020F9BB2F8D0017300
:1019380040F2E93300E043B10289013B12F0010FA4
:101948009BB2F8D0007BC0B208BDFEF726FCC0B23F
:1019580008BDF8B584894FF6FF764FF47A742BB337
:1019680011B30F78013101E0B44217D00589013C69
:10197800AD07A4B2F8D507734FF47A7402E0BCB28D
:10198800B4420BD00589ED0704F1FF37F7D5057B85
:10199800EDB20AB115700132013BE0E7FEF7FDFB3D
:1019A800003018BF0120F8BDFF27DFE70120F8BD90
:1019B800F0B55B4B5B4A97B01968914200AF00F0F5
:1019C800A3805949594A00234FF47000C1F8880090
:1019D8003B607B60136843F48033136003E03B682B
:1019E800B3F5A04F09D0136803F400337B603B685C
:1019F80001333B607B68002BF1D04C4B1B6813F420
:101A0800003318BF01237B607B68012B52D0464C02
:101A1800464B474AE260474A596A11605A6A42F09F
:101A280080725A625A6942F4FC025A610025032204
:101A380007F10801012341F6FF764FF09040FD6061
:101A4800BE603A73BB7322F047F94FF6FF7307F194
:101A580008013948BB6022F03FF907F1080137480F
:101A6800374E22F039F907F10801364822F034F9E7
:101A780007F10801344822F02FF907F1080133482B
:101A880022F02AF907F1080022F07FF9BB683049F3
:101A9800304AA1FB031330499B0CF0204FF0070E8E
:101AA8005C370B60566084F823009560C2F800E04C
:101AB800BD46F0BD294A1D4B122111605A685A6073
:101AC8005A685A605A6842F480625A605A6822F426
:101AD8007C125A605A6842F4E8125A601A6842F056
:101AE80080721A601A689201FCD559680F4A21F071
:101AF80003015960596841F002015960536803F0C5
:101B08000C03082BFAD182E700221A6062B6144B44
:101B18001B6883F30888134B1B689847FEE700BFD0
:101B2800FC9F0020EFBEADDE00ED00E0001002409B
:101B38000005FA05845A00200004004800080048FF
:101B48003F190100000C004800100048001400482C
:101B580083DE1B4310E000E0B48500200020024033
:101B680000D8FF1F04D8FF1F70B50F4C0F4DC0EBF6
:101B7800C00004EB8004686926693043686182B05C
:101B88009209667BA1600025012101A863618DF897
:101B980004608DF805208DF806508DF8071022F0A6
:101BA80065F802B070BD00BF20060020001002409A
:101BB800074BC0EBC00030B403EB8000054C05694F
:101BC80063692B4363610176427630BC704700BF7E
:101BD80020060020001002402DE9F04F5E4C54F81A
:101BE800204083B0002C71D0A66D984691465B4B7F
:101BF80072682265A160236004F15E014FF480736E
:101C080004F5AF726161A261E36023610746307E2B
:101C18002AF06EFEF068A8B1514B00215A68904234
:101C280003F11C0300F0928001310C29F6D1002049
:101C38007A1CD2B20C21FFF7BBFF236DF2686263F6
:101C48002433E364B068D8B1454B00215A68904208
:101C580003F11C0378D001310C29F7D100257A1C37
:101C6800D2B20B212846FFF7A3FF2346F27E3D4957
:101C78002846FFF779FF236DB268A2632833A3646F
:101C880094F85D0003F068F8054694F85C0003F0EA
:101C980063F818F0080F824696F819B01AD0CDB13B
:101CA80018F0110F4FF00B0307F1010714BF4E2175
:101CB8003E21EF715A46AB71284602F0ADFC18F090
:101CC800010F45D0636B5BB3A36B4BB3204603B0E6
:101CD800BDE8F08F18F0010F0CBF4FF02E084FF041
:101CE8004E0819F0020F09D045B10B227B1CAA71CE
:101CF800EB7128465A46414602F08EFC19F0010F56
:101D0800E0D0BAF1000FDDD001370C238AF8077054
:101D18005A4641468AF80630504602F07DFCD1E723
:101D2800337FB27E8DF804209B090021012201A88F
:101D38008DF805308DF806108DF8072021F096FFF4
:101D4800204603B0BDE8F08FCDB288E7C8B26FE790
:101D58002846FEF736FDB5E74C2F00200858030843
:101D680020060020A907000800B97047F0B595B013
:101D780005462BF043F86C4EC3680268326004468F
:101D8800002B00F0C380284602F0E6FF674B9864FA
:101D980018B1292200238271C371227A644D2E2141
:101DA80002F03AFC306803F09DF92AF0A1FD306892
:101DB800604A038823F001031B041B0C038014A949
:101DC8001E232B8001270F230025138021F84C7D2B
:101DD8002D230293ADF80C50ADF80650ADF80E5017
:101DE8002AF0BAFFE379ADF8145060229907ADF8EC
:101DF80016500695ADF81C50ADF81E50ADF82050A1
:101E0800ADF82250049200F1838013F0010F0CBF4B
:101E1800002202224FF48073ADF81470ADF81C2034
:101E2800ADF82030002304AA61793068069302F0E7
:101E3800F9F961793068404F2AF06EFF33685A6CBF
:101E480042F400425A641A8892B242F080021A8020
:101E5800E2796079196A92074CBF04220122824014
:101E680021EA02011962196A0A431A621A8892B2AF
:101E780042F001021A80207C00222921FFF798FEF7
:101E88002E49207C00236022FFF76EFEE068386050
:101E980020F04AF8386803684FF6FE721340036072
:101EA80020F042F809A820F011F833686279244933
:101EB80038680A913433134409938022102300258B
:101EC80009A940F22A3E0E920B934FF400724FF488
:101ED80000530D951095139511950F921293ADF827
:101EE80030E020F001F8627933680C2A98BF154970
:101EF800D86898BF31F812503A6813490543DD6035
:101F08001368012043F002031360087015B0F0BD98
:101F180013F0010F0CBF2A4608220423ADF81E2037
:101F2800ADF816307EE700BF808E0020C02200206A
:101F3800768E0020748E00207C8E002071060008AA
:101F4800905C00201C790308788E00200348D0F8A4
:101F58003C3113B100F59A701847704720060020ED
:101F68000348D0F8203113B100F58C70184770473A
:101F7800200600200348D0F804310BB1FC30184784
:101F8800704700BF200600200348D0F8E8300BB1A6
:101F9800E0301847704700BF200600200348D0F8FB
:101FA800CC300BB1C4301847704700BF2006002062
:101FB8000348D0F8B0300BB1A8301847704700BFBD
:101FC800200600200348D0F894300BB18C30184715
:101FD800704700BF200600200248836F0BB17030A5
:101FE80018477047200600200248C36D0BB15430D3
:101FF80018477047200600200248036C0BB13830A0
:1020080018477047200600200248436A0BB11C306D
:1020180018477047200600200248836803B1184714
:10202800704700BF20060020028822F040021204F8
:10203800120C0280028822F038031B041B0C59B1D1
:1020480041F48071002991FAA1F2B2FA82F108BF35
:102058004FF0FF310139C9000B439BB2038003885D
:102068009BB243F04003038070472DE9F84FDFF837
:10207800DCB0DFF8DCA03148DFF8D8800123042188
:102088008BF80030FFF7D0FFDAF80000FEF799FB75
:1020980005212A48FFF740FC00212848FFF73CFCAF
:1020A80006212648FFF738FC00212448FFF734FCB6
:1020B800234B22481C78042144F00104FFF72CFC30
:1020C80021461E48FFF728FCB8F80030B3B11D4D73
:1020D8001D4F1A4E002495F8019007213046FFF74E
:1020E8001BFC49463046FFF717FCB8F8003015F8D6
:1020F800012F07F8012F01349C42ECDB07210F4820
:10210800FFF70AFCFF210D48FFF706FC0C4B0B48B4
:102118001C780421FFF700FC21460848FFF7FCFB68
:10212800DAF80000FEF752FB02210448FFF77CFFB3
:1021380000238BF80030BDE8F88F00BF003800405E
:102148007C5100206B3F0020434D0020A44100201B
:10215800048A002054010020F8B5114D114FC1F137
:10216800030646EA800604212846FFF75DFF386823
:10217800FEF727FBF6B21024E1B22846FFF7CCFBA6
:10218800013431462846FFF7C7FB202CF4D13868C4
:10219800FEF71CFB02210248BDE8F84044E700BFF7
:1021A80000380040048A0020F8B5444C4448042113
:1021B800FFF73AFF2068FEF704FB424B1B78012B20
:1021C8006DD058D3022B4ED13F4D08232B704FF4BE
:1021D800C3733E4E3E4F338002210020FFF7BCFF01
:1021E80004213748FFF720FF2068FEF7EAFA2D7828
:1021F80033480021FFF790FB29463148FFF78CFB55
:10220800344B2F481D780221FFF786FB29462C48BE
:10221800FFF782FB304B2A481D780321FFF77CFB30
:1022280029462748FFF778FB2C4B25481D780421C1
:102238000D43FFF771FB29462148FFF76DFB206826
:10224800FEF7C4FA02211E48FFF7EEFE3288244842
:10225800002133F0FAF93B7863B1224B1B7823B3A2
:1022680000233B70F8BD184D2B785B06AFD54FF4B3
:10227800F073AEE7F8BDA0211148134DFFF74CFBF2
:1022880000210F48FFF748FB00F00603022B03D09C
:1022980000F0050001280DD008232B7097E70A4DA0
:1022A80048232B704FF4F07393E7FFF7DEFE00230B
:1022B8003B70F8BD48232B70D9E700BF048A002083
:1022C80000380040088A00207600002054010020D1
:1022D800000000200F8A0020108A00207C51002076
:1022E800444D0020A4410020F8B505015A4C5B4B31
:1022F800625961199A4204EB050704BF01230B7365
:102308000646387A2AF0F4FA3B7A03F01F015B0993
:102318000122022B02FA01F278D0032B71D0012B93
:1023280067D063190136187902F016FDF6B2074630
:1023380010B11223C67183716319587902F00CFD2C
:1023480010B11323C67183716319987902F004FDE3
:1023580010B11423C671837166190E21F2793846BB
:1023680002F05AF9707902F0F7FCF2790E2102F0C6
:1023780053F9B07902F0F0FCF2790E2102F04CF931
:102388006359364A934251D0354A934259D0354A17
:10239800934240D02C44227B002A2FD101200224D2
:1023A8009A8822F480521204120C9A80998889B271
:1023B80041F4805199801A8802F4415242F44572DE
:1023C800024322431A809A8822F470621204120C83
:1023D80042F4E0629A809A8B22F400621204120C92
:1023E80007219A8319821A8892B242F040021A8011
:1023F800F8BD1D4B996A0A439A6292E70020044689
:10240800CEE7194B19690A431A618AE7164BD9684E
:102418000A43DA6085E702F5EA32116941F40041BE
:102428001161116921F400411161B3E702F56042BD
:10243800D16841F48051D160D16821F48051D160D4
:10244800A8E702F5EC32116941F480411161116984
:1024580021F4804111619DE7702F00200030014078
:1024680000380040003C004000100240F0B53E4CEF
:10247800059D00EB800004EB80046468002C71D09B
:102488003A4E49004FF42040CFB2F064A1690904E4
:1024980054D46068DFF8E0E047F4903100EA0E00B9
:1024A80001434FF420406160F06403E0411E0028BE
:1024B80048D00846A1698907F8D54FF42040A262A0
:1024C800F06403E0421E00283CD01046A269520680
:1024D800F8D5274A6168DFF8A0E0F06442EA0342D1
:1024E800174301EA0E0217436760C3B1013BDBB231
:1024F80001332B44A0694FF4204210F0040002F18C
:10250800FF3207D1511C26D0A06910F0040002F157
:10251800FF32F7D0626A05F8012B9D42EAD14FF4E9
:102528002040F06402E0431E60B11846A3699B0690
:10253800F9D52023F064E3610120F0BD411E08B104
:102548000846A3E70B4A138801339BB24FF0FF31CB
:102558001380F164F0BD0749F2640B8801339BB224
:102568000B80F0BD2046F0BD50850020C022002021
:102578000024000264310020009800FCF0B50D46EC
:102588000178012983B00446164618D0022902D0E2
:10259800002003B0F0BD80681F46FEF712F945F031
:1025A80080016068FFF7B8F93B4632460021606851
:1025B800FFF7CFF9A068FEF709F90120E9E790F9DC
:1025C8000400421CE4D00228E2DC617900962A4625
:1025D800FFF74CFFDDE7F0B5037C012B85B004461F
:1025E80063D0022B67D1836913B11A689B8813855E
:1025F800606940F2E93301E0002B6CD00289013BAD
:1026080012F0020F9BB2F7D0C323037340F2E933F1
:1026180001E0002B5FD00289013B12F0010F9BB251
:10262800F7D0037B60694FF0060E838902AE4FF442
:102638007A734FF6FF71FF2703E0013B9BB28B4291
:102648003CD002899507F8D507734FF47A7302E0F6
:10265800ABB28B4232D00289D20703F1FF35F7D5EE
:10266800027BD2B20EB132700136BEF1010EE8D152
:10267800A36913B11A689B8893619DF80C009DF8B3
:1026880008609DF809109DF80A509DF80B209DF8E8
:102698000D3041EA062143EA002342EA05220120DF
:1026A80021876287A38705B0F0BD90F91400431C09
:1026B80001D0022805DD002005B0F0BDFDF76DFD55
:1026C800D6E702AB617D009343220623FFF7CEFED7
:1026D8000028D2D1EFE7FDF760FDA3E7F0B5037A54
:1026E800012B85B0044663D0022B67D1036913B16F
:1026F8001A689B881385E06840F2E93301E0002BF3
:102708006CD00289013B12F0020F9BB2F7D0BB23B9
:10271800037340F2E93301E0002B5FD00289013BEB
:1027280012F0010F9BB2F7D0037BE0684FF0060E62
:10273800838902AE4FF47A734FF6FF71FF2703E0E7
:10274800013B9BB28B423CD002899507F8D50773B1
:102758004FF47A7302E0ABB28B4232D00289D207CF
:1027680003F1FF35F7D5027BD2B20EB132700136D4
:10277800BEF1010EE8D1236913B11A689B889361F1
:102788009DF80C009DF808609DF809109DF80A5006
:102798009DF80B209DF80D3041EA062143EA0023FD
:1027A80042EA05220120E1822283638305B0F0BD5D
:1027B80090F90C00431C01D0022805DD002005B06B
:1027C800F0BDFDF7EAFCD6E702AB617B00933B2244
:1027D8000623FFF74BFE0028D2D1EFE7FDF7DDFC1B
:1027E800A3E7B0F1FF3F56D0022854DCF0B4334CD5
:1027F80000EB800004EB80004468002C5BD0304E76
:1028080049004FF42040CDB2F064A169090444D4D2
:1028180060682C4F45F08071384041F49031014395
:102828004FF420406160F06403E0411E002838D076
:102838000846A1698F07F8D54FF42040A262F064DA
:1028480002E0421E68B31046A2691106F9D5626813
:102858001C4945F0007545F480350A4015434FF48E
:1028680020406560F06402E0421ED0B11046A269C3
:102878009207F9D54FF42040A362F06402E0431EAA
:1028880078B11846A3699B06F9D52023F064E36163
:102898000120F0BC704700207047411E08B108466F
:1028A800B3E7094A138801339BB24FF0FF31138015
:1028B800F164F0BC70472046FBE700BF508500205C
:1028C800C0220020009800FC643100202DE9F04F60
:1028D80087B090F855300190002B40F0E483019ABE
:1028E800137C012B00F07B84022B44D1936913B134
:1028F8001A689B881385019B586940F2E93302E006
:10290800002B00F0E1840289013B12F0020F9BB218
:10291800F6D06B23037340F2E93302E0002B00F09A
:10292800D3840289013B12F0010F9BB2F6D0037BDE
:10293800019B586940F2E93302E0002B00F0C084A3
:102948000289013B12F0020F9BB2F6D08023037379
:1029580040F2E93302E0002B00F0B2840289013B27
:1029680012F0010F9BB2F6D0037B019B9B6913B158
:102978001A689B8893616423A94CAA4DDFF8ACA21E
:10298800A948DFF8ACC24FF010084FF47A779E469A
:10299800DAF80430C3F30803002B40F04E82EFF35B
:1029A8001183002B40F049822168826800BF2368A8
:1029B8009942F9D12E6807FB06F39B1AB3FBF6F38D
:1029C80007FB013101260091DAF80430C3F308034C
:1029D800002B40F01582EFF31183002B40F010829A
:1029E8002368816800BF22689342F9D1D5F800B006
:1029F80007FB0BF2521AB2FBFBF207FB0323009A08
:102A08009B1AB3F57A7FDFD3BEF1010EC0D1019ACC
:102A1800137C012B51D0022B58D1936913B11A683A
:102A28009B881385019B586940F2E93302E0002B2B
:102A380000F05F840289013B12F0020F9BB2F6D0CE
:102A48006B23037340F2E93302E0002B00F051845A
:102A58000289013B12F0010F9BB2F6D0037B019B68
:102A6800586940F2E93302E0002B00F03184028912
:102A7800013B12F0020F9BB2F6D00323037340F21E
:102A8800E93302E0002B00F023840289013B12F0B5
:102A9800010F9BB2F6D0019E037BB269002A00F0B9
:102AA8001E84136892889A61307C96F85010012829
:102AB80000F0DF81022855D114E0164603236B226B
:102AC800717D96F91400FFF78CFE337C0198012B79
:102AD80090F8501000F0CD81022B43D1826912B1D9
:102AE800136892881A85019B40F2E932586902E01E
:102AF800002A00F018840389013A13F0020F92B2F9
:102B0800F6D01923037340F2E93202E0002A00F0FC
:102B18000A840389013A13F0010F92B2F6D0037BBD
:102B2800019B40F2E932586902E0002A00F0F8837C
:102B38000389013A13F0020F92B2F6D0017340F202
:102B4800E93302E0002B00F0EB830289013B12F02D
:102B5800010F9BB2F6D0037B019B9B6913B11A68E6
:102B68009B8893610F23DFF8C4A02F48DFF8C0C00B
:102B78004FF010084FF47A779E46DAF80430C3F322
:102B88000803002B40F07382EFF31183002B40F011
:102B98006E822168826800BF23689942F9D12E6845
:102BA80007FB06F39B1AB3FBF6F307FB013101267B
:102BB8000091DAF80430C3F30803002B40F03A829E
:102BC800EFF31183002B40F035822368816800BF42
:102BD80022689342F9D1D5F800B007FB0BF2521ADC
:102BE800B2FBFBF207FB0323009A9B1AB3F57A7F2B
:102BF800DFD3BEF1010EC0D10198027C90F84E10CF
:102C0800012A00F09F81022A40F0A581836913B14F
:102C18001A689B881385019B40F2E93258690CE0D9
:102C2800B0850020B485002010E000E000ED00E051
:102C3800AC850020002A00F070830389013A13F064
:102C4800020F92B2F6D01A23037340F2E93202E07F
:102C5800002A00F062830389013A13F0010F92B24F
:102C6800F6D0037B019B40F2E932586902E0002A62
:102C780000F043830389013A13F0020F92B2F6D0B1
:102C8800017340F2E93302E0002B00F03683028939
:102C9800013B12F0010F9BB2F6D0037B01988269C9
:102CA800002A00F03183136891889961027C012A17
:102CB80000F09F82022A00F05981012A00F0E28088
:102CC800022A40F0E880019B9A691AB1136891883A
:102CD8001985019B586940F2E93302E0002B00F0A6
:102CE800EC820289013B12F0020F9BB2F6D01C2342
:102CF800037340F2E93302E0002B00F0DE82028920
:102D0800013B12F0010F9BB2F6D0037B019B58697F
:102D180040F2E93302E0002B00F0BF820289013B58
:102D280012F0020F9BB2F6D01823037340F2E93376
:102D380002E0002B00F0B1820289013B12F0010F82
:102D48009BB2F6D0037B01988269002A00F0AC821E
:102D5800136891889961027C012A00F05481022A43
:102D680000F0A480012A00F05A81022A45D1019B73
:102D78009A6912B1136892881A85019B586940F2C2
:102D8800E93302E0002B00F085820289013B12F052
:102D9800020F9BB2F6D03823037340F2E93302E006
:102DA800002B00F077820289013B12F0010F9BB2E1
:102DB800F6D0037B019B586940F2E93302E0002B0F
:102DC80000F065820289013B12F0020F9BB2F6D037
:102DD8000123037340F2E93302E0002B00F057822D
:102DE8000289013B12F0010F9BB2F6D0037B019BD5
:102DF8009B6913B11A689B88936107B0BDE8F08F8F
:102E0800EFF3118988F3128881680368DB0344BFF4
:102E1800CCF8006081682368DCF800205FFA89F943
:102E280089F31188D5F800901A4407FB09F35B1A57
:102E3800B3FBF9F307FB0233E1E5EFF3118288F303
:102E4800128886680368D90303D50123CCF80030BB
:102E580086682368DCF80010D2B282F311882A68E9
:102E6800194407FB02F39B1BB3FBF2F307FB013189
:102E7800A8E501980B461922417D90F91400FFF747
:102E8800B0FC6FE6019C1C221823617D94F91400A4
:102E9800FFF7A7FC227C012A00F0B580022A7FF404
:102EA80061AF019B9A691AB1136891881985019BD2
:102EB800586940F2E93302E0002B00F0E58102890D
:102EC800013B12F0020F9BB2F6D03723037340F296
:102ED800E93302E0002B00F0D7810289013B12F0B0
:102EE800010F9BB2F6D0037B019B586940F2E9338E
:102EF80002E0002B00F0B7810289013B12F0020FBB
:102F08009BB2F6D00223037340F2E93302E0002BB0
:102F180000F0A9810289013B12F0010F9BB2F6D0A3
:102F28000199037B8A69002A00F0A48113689288BA
:102F38009A61097C012972D002293FF41DAF07B0BC
:102F4800BDE8F08F04460B461A22417D90F9140023
:102F5800FFF747FC227C012A00F04B81022A7FF40C
:102F6800ACAE019B9A691AB1136891881985019BC7
:102F7800586940F2E93302E0002B00F071810289C0
:102F8800013B12F0020F9BB2F6D01B23037340F2F1
:102F9800E93302E0002B00F063810289013B12F063
:102FA800010F9BB2F6D0037B019B586940F2E933CD
:102FB80002E0002B00F044810289013B12F0020F6D
:102FC8009BB2F6D01823037340F2E93302E0002BDA
:102FD80000F036810289013B12F0010F9BB2F6D056
:102FE800037B01988269002A00F031811368918877
:102FF8009961027C012A3FF445AF022A3FF468AE8A
:10300800012A7FF44BAF019C37220223617D94F99A
:103018001400FFF7E6FB227C012A7FF4A6AE019894
:103028000123417D90F914003822FFF7DAFB07B03D
:10303800BDE8F08FEFF3118988F31288816803687F
:10304800DB0344BFCCF8006081682368DCF800200B
:103058005FFA89F989F31188D5F800901A4407FBBB
:1030680009F35B1AB3FBF9F307FB0233BCE5EFF393
:10307800118288F3128886680368D90303D501236F
:10308800CCF8003086682368DCF80010D2B282F3EE
:1030980011882A68194407FB02F39B1BB3FBF2F360
:1030A80007FB013183E51D09013D052D03F00F03E1
:1030B80000F2C180A34A32F8150040FA03F2D4079F
:1030C80040F1B980012404FA03F3013B184030F0C1
:1030D800A9FE9D4BDFF88C825F5D074418EBC7059E
:1030E80000F0A98020220023AA71EB7158F837005C
:1030F800964A00F138439B0AD25C02F01F0352093A
:10310800022A04FA03F300F01781032A00F00F8162
:10311800A24200F08B80AB88049304A90024059494
:1031280020F0DAFDAB88019E894AF260B3FA83F297
:10313800C2F11F02511C3FD0D1B201F0FC0303F1D0
:10314800804303F5803301F00301D3F808E08800D9
:103158004FF00F0C58F837107E4FDFF80C820CFA3E
:1031680000FC2EEA0C0E06F10C0C47F822C0C1F345
:103178008721C3F808E0D3F808E0814008EB020093
:1031880041EA0E0190F800A199604FF00109724BD5
:1031980009FA02F15744196004A808238DF815307C
:1031A8008DF8169004928DF814402BF0FBF997F8DF
:1031B8004030F02B27DCAB88B3FA83F3C3F11F034D
:1031C800581C3FF48CAB012202FA03F363490A68E6
:1031D8001343019A0B60137C012B7FF485AB1046D7
:1031E8008023417D90F914006B22FFF7FAFAFFF76C
:1031F800C2BB019C1B221823617D94F91400FFF7C0
:10320800F0FA227C59E5D044F02298F810318DF874
:103218000C3003A803238DF80E408DF80F9087F823
:1032280040208DF80D3020F021FDC4E74C4A51694B
:103238000B4353616FE7019A454BD3600123C5E700
:10324800FCF7ABFF01988269002A7FF4CFAE027CBD
:10325800012A03463FF416AE022A3FF43BAD1AE6B4
:10326800FCF79BFFA0E6FCF798FF01998A69002A02
:103278007FF45CAE0B7C012B3FF4D1AE022B3FF404
:103288007CAD07B0BDE8F08FFCF787FF2CE6FCF7B4
:1032980084FFACE5FCF781FF8CE5FCF77EFF019825
:1032A8008269002A7FF454AD027C012A03463FF468
:1032B800AAAE022A3FF4FCAD54E5FCF76EFF25E503
:1032C800FCF76BFFFFF751BBFCF767FFFFF730BB5D
:1032D800FCF763FF019EB269002A7FF4E2AB337CFE
:1032E80096F85010012B3FF4C4AD022B3FF4FBAB12
:1032F80038E4FCF752FFFFF7B2BBFCF74EFF01982A
:103308008269002A7FF4CFAC027C012A03463FF48D
:1033180070AF022A3FF42CAECFE4FCF73EFFA1E4E5
:10332800FCF73BFF18E4FCF738FFFFF7F9BB0C4A42
:10333800D1690B43D361EEE6094A91690B43936166
:10334800E9E600BF987F0308A47F0308AC7F030861
:10335800D7050008C02200201404014000040140E1
:1033680000100240E88A0020305703081749184B1C
:10337800184A194810B4D1F8884044F47004C1F8C8
:1033880088401C6844F001041C605C6822405A6054
:103398001A6822F0847222F480321A601A6822F4C1
:1033A80080221A605A6822F4FE025A60DA6A22F011
:1033B8000F02DA621A6B002410404FF000621863A3
:1033C8009C608A605DF8044B704700BF00ED00E028
:1033D800001002400CC07FF8CCFC00FF38B50B4C45
:1033E80023688BB15A68821A002A054604DA0CE071
:1033F8005A68AA1A002A07DB9A68226018461A68CF
:1034080090472368002BF3D138BD38BD2C350020F8
:103418000B4B002210B4027203F1A004042102E055
:10342800072A09DC9979890702D51979815401326B
:103438009C4203F11403F3D15DF8044B704700BFBD
:10344800047E030810B40D4C04232146002200E03A
:103458008B7913F0010301F1140106D10132092A15
:10346800F6D103705DF8044B704702EB820204EB5F
:1034780082025DF8044B137903707047047E0308D9
:1034880010B40123022414212222047241704271D3
:10349800037003715DF8044B704700BF2DE9F041DC
:1034A8000B78057BDB43DFB200F1130200F11D034B
:1034B80002F8015F9342FBD1DFF890E000F12701A9
:1034C800002203F8012F9942FBD11421052400267C
:1034D80047FA04F303F00103002B1E4414BF4FF016
:1034E80019084FF00A0814F0010FF6B214BFAC46E1
:1034F8004FF0000C0023CA1810FA82F2013343453A
:1035080082F814C0F7D15A1E92B20132013C8B18CE
:10351800621C9BB201D01946DAE716F0010F14BFFE
:1035280019240A240022991810FA81F10132A242C2
:103538000D75F8D113449BB25A1C0344002192B272
:103548001975AEF800200261BDE8F0814023002023
:103558002DE9F04FDFF890A0BAF802300B3383B0B2
:103568001FFA83F901F1060B4FF001084FF0000C28
:10357800002711F801EB3E464C460122A4F10B034B
:103588009BB2019105E001339BB2017B29759C42F6
:1035980008D0C518002AF6D1C51801339BB29C4241
:1035A8002A75F6D103190136092F019983F814C039
:1035B800F6B20CD0092E15D008FA07F313EA0E0F4D
:1035C80014BF012200220C34A4B20137D6E709F156
:1035D800780959451FFA89F9CAD1AAF802C003B077
:1035E800BDE8F08F0022EEE7402300202DE9F047E8
:1035F800DFF85C80B8F8043004331FFA83FC01F16B
:1036080009094FF0010E11F8017B64460026231FBB
:103618000EFA06F29BB23A40C2B1B0F80CA0C51837
:1036280001339BB29C4285F814A0F5D101360434CD
:10363800082EA4B2EBD10CF1200C49451FFA8CFCE2
:10364800E1D10023A8F80430BDE8F0879246E6E708
:103658004023002010B50168047B0A680223A340B8
:103668001A420AD0054A406800241470026822F001
:1036780001021204120C02604B6010BDAB2700203F
:10368800436A8269D154436A0169826B01338B4270
:1036980028BF00234362002A2FD0EFF31181502363
:1036A80083F31288836B1A68D2072CD470B45E68CF
:1036B8006EB9456A826A954217D084691444DC6001
:1036C8000ED9AA1A5A608562002280F854201A6816
:1036D80042F00102C9B21A6081F3118870BC7047C8
:1036E8000469A21A5A608662EEE7012380F8543012
:1036F800C9B281F3118870BC7047026D136843F03A
:10370800800313607047C9B281F31188704700BF06
:10371800426B10B462B1436CC2684469D11A013B70
:10372800615C5DF8044B08BF13464364C8B2704738
:10373800016A4369C4685B5C0131A14228BF114634
:1037480001625DF8044BD8B2704700BF836B13B1B8
:1037580090F854007047836A406A181AB0FA80F0EB
:1037680040097047416A836A99420AD3CB1A816B30
:10377800026961B14968501E0B4483420AD2C01ADB
:10378800704702691144CB1A816B0029F2D1501E8F
:10379800C01A704700207047436B43B1426C5B68A6
:1037A80093422FBF981AC0689B1AC0187047C26905
:1037B800036A9A422FBFD01AC0688018C01A70478F
:1037C8000A4B30B503F10C0493F900205D78072A01
:1037D800C8BF143A811804338D7213F8025C8554FB
:1037E80013F8012C0A75A342EED130BD48580308DE
:1037F80003682DE9F041DF691FB13B46BDE8F041A0
:103808001847002A164611DD04460D460E4400E00E
:1038180023689B68204698470028F9D0236815F844
:10382800011B1B6820469847AE42F1D1BDE8F081E4
:1038380000232322027043708370C370704700BF57
:103848002DE9F0470569C3681D4028D00F46064694
:103858004FF000484FF00009B5FA85F328FA03F253
:10386800D2431B3B32611540042B16D8DFE803F026
:103878003129211903007B6A002B32D003F1FF3A6A
:103888001FFA8AFAC7F824903C6A34B123682046A4
:10389800514698476468002CF8D1002DDCD1BDE86A
:1038A800F0873868716B036889B29847002DD3D1C7
:1038B800F5E77868B16B036889B29847002DCBD1DA
:1038C800EDE7B868F16B036889B29847002DC3D15A
:1038D800E5E7F868316C036889B29847002DBBD1D9
:1038E800DDE7F36A1FFA83FACEE700BF30B5044676
:1038F800006D61710368A26823F00103036087B05B
:10390800A379009213F004023DD04FF4805213F0D3
:103918000203019244D102934FF48063002203937F
:1039280011F00103059237D1049308238D076946E6
:1039380048BF04931EF05AFA6079236DA17900F00C
:103948000202002A15BF4FF440324FF480324FF480
:103958000034002410F0010F586808BF2246CC0735
:103968004CBF024320EA02025A609A6809074CBF1A
:1039780042F0080222F008029A601A6842F0010236
:103988001A6007B030BD13F0020301920BD04FF458
:10399800005513460295C1E7042304930C23C5E799
:1039A8004FF40053B7E70293B8E700BF10B50446D9
:1039B800006DA160036823F001030360A37986B05A
:1039C80013F00402009141D04FF4805213F0020327
:1039D800019244D102934FF4806362790393D10733
:1039E8004FF000030493059345BF04230493082371
:1039F8000C236946920748BF04931EF0F7F96079D3
:103A0800236DA17900F00202002A15BF4FF440325D
:103A18004FF480324FF40034002410F0010F58683E
:103A280008BF2246CC074CBF024320EA02025A6074
:103A38009A6809074CBF42F0080222F008029A600F
:103A48001A6842F001021A6006B010BD13F00203B2
:103A5800019207D04FF4005113460291BDE74FF48D
:103A68000053B7E70293B8E7022828BF022010B432
:103A7800084C094B207000EB8002C0EBC2020749DA
:103A88005DF8044B013003EB4203C0B20B602DF02C
:103A980087BB00BF948C0020208D0020E4640020A8
:103AA80008B513F0B9FAFDF7A1F8BDE8084013F01E
:103AB8009BBA00BF2DE9F04F013085B0C3B2039324
:103AC8008E4D8F4F8F4C904E0A2302933220DFF891
:103AD800409229F079FB4FF4FA7A4FF0100C4FF42A
:103AE8007A70D9F80430C3F30803002B40F0C8807B
:103AF800EFF31183002B40F0C3802968A26800BF50
:103B08002B689942F9D1D7F800E000FB0EF39B1A15
:103B1800B3FBFEF300FB01314FF0010E0191D9F820
:103B28000430C3F30803002B40F08E80EFF31183B9
:103B3800002B40F089802B68A16800BF2A68934257
:103B4800F9D1D7F800B000FB0BF2521AB2FBFBF226
:103B580000FB0323019A9B1AB3F57A7FDFD3BAF1EE
:103B6800010ABED1039B002B40F0C4804FF47A7A3F
:103B7800DFF89C9150464FF0100CD9F80430C3F38D
:103B88000803002B40F09980EFF31183002B40F0DD
:103B980094802968A26800BF2B689942F9D1D7F8A8
:103BA80000E000FB0EF39B1AB3FBFEF300FB0131B0
:103BB8004FF0010E0191D9F80430C3F308033BBB61
:103BC800EFF3118323BB2B68A16800BF2A689342D7
:103BD800F9D1D7F800B000FB0BF2521AB2FBFBF296
:103BE80000FB0323019A9B1AB3F57A7FE3D3BAF15A
:103BF800010AC2D1029B013B02937FF467AF43499C
:103C0800434B4448444A0860DA6005B0BDE8F08F89
:103C1800EFF311888CF31288A1682368DB0344BF93
:103C2800C6F800E0A1682B6832685FFA88F888F364
:103C38001188D7F800801A4400FB08F35B1AB3FB1D
:103C4800F8F300FB0233CDE7EFF311888CF3128809
:103C5800A1682368DB0344BFC6F800E0A1682B68AD
:103C680032685FFA88F888F31188D7F800801A4418
:103C780000FB08F35B1AB3FBF8F300FB023369E7B8
:103C8800EFF311828CF31288D4F808E02368D90383
:103C980003D501233360D4F808E02B683168D2B229
:103CA80082F311883A68194400FB02F3A3EB0E0370
:103CB800B3FBF2F300FB01312EE7EFF311828CF333
:103CC8001288D4F808E02368D90303D501233360A8
:103CD800D4F808E02B683168D2B282F311883A68C8
:103CE800194400FB02F3A3EB0E03B3FBF2F300FB52
:103CF80001315DE7184629F0D7F837E7B08500208D
:103D0800B485002010E000E0AC850020FC9F002076
:103D180000ED00E0EFBEADDE0400FA0538B5434B18
:103D28005A899989914224BF00225A81198ADA89CD
:103D3800914224BF0022DA81DA788AB3072A2FD089
:103D48003B493C4D91F85300012400210A282C706E
:103D58009C70D9713DD00C2865D0DFED377A8ABBCD
:103D6800364C9FED370AA278002918BFF0EE407A4A
:103D7800062A04D8334901EB820191ED030A21791F
:103D880059B3013A032A4DD8F7EE007A87EE800A34
:103D980030F09EFC2388984228BF1846208038BD02
:103DA800D97921B198780428B8BF042098702048A0
:103DB80090F853000A280CD00C28CED1DFED227AD7
:103DC800002ACDD0072ACBD00A282CD1DFED1F7AC4
:103DD800C6E70A20DFED1E7AC1E79B78154A07EE91
:103DE800103A1178B8EEC77A27EE277A07EE901ABC
:103DF800F8EEE77A67EE877AB4EEE70AF1EE10FAA2
:103E080010DDC0EE077AFDEEE77A17EE903A102B38
:103E1800A8BF1023012BB8BF0123DBB28B4238BFE8
:103E28000B46137038BDDFED0B7A99E7745200200A
:103E380088520020B83E00206F1203391057002026
:103E48006F120338485803080AD7A3390F506E3A3F
:103E58005304E9386F12833A2DE9F047A64FA74E6D
:103E680013F0DAF8BE421ED2DFF80C83DFF80C93A9
:103E78004446258862197DB14A450DD2052D0BD9D6
:103E880033886188C3F30B03994200F0D980144644
:103E980025886219002DEFD1716830461436FCF779
:103EA80031FEBE42E4D3964A1378A3F117010229E2
:103EB8000FD9944911F83300002840F0ED80D8005C
:103EC8000144497829B1904911F83330002B00F0AA
:103ED8000B818E4B5A78022A40F2D88000228C49F6
:103EE8005A701A788B48022A016000F2CB8002EBE4
:103EF8008201894BC2EBC10203EB4203998C5A8CB5
:103F0800864C9142236001D300225A84844B9A78CC
:103F1800042A00F0E08032B91A88B2F5F07F84BF35
:103F28004FF4F0721A807F4DFFF7F8FE2B687E4A37
:103F38001A40002A00F0DB80D80700F1C780590436
:103F480000F1BF801A0700F1B7809B0400F1AD8033
:103F58002AF08CFF10B975482CF000FD4020FCF7C2
:103F680007FE8020FCF704FE4FF40070FCF700FE0B
:103F78004FF00070FCF7FCFD4FF08060FCF7F8FD97
:103F88001CF0B8FC00213022694831F05EFB206843
:103F98001BF0C2FB674B276803F1500102E00433B2
:103FA80099426DD01A78002AF9D19C78D878844241
:103FB800F5D26149614B0D79614962480A70624ED8
:103FC800624C0460C822642111FB0521002259605B
:103FD8009A60DA601A615A619A61DA6183F820207E
:103FE80083F82120376015F0B5FF594B9FED595ADA
:103FF8001B88594A9FED596A5079594906EE903AFB
:10400800F8EEE66A1388C5EE265A07EE103A53888A
:104018001279C1ED005A07EE903AB8EEC77A514BC3
:10402800F8EEE77A18725A7227EE067A67EE867A01
:10403800BDE8F04783ED017AC3ED007A12F0D4BFF2
:1040480063799B077FF423AF716894F804A0304626
:10405800FCF758FD3388BAEB133F04D01436BE4240
:10406800FFF406AF1FE773887068AA1FC3F30B033A
:104078009A4204F10601A8BF1A4630F055F9EDE757
:10408800012296E700221A70234B37E7204902EBFA
:10409800420201EB820124E7D8000C186468002C66
:1040A8007FF40EAF172414700AE72F48FCF760FD61
:1040B8004020FCF75DFD4BE72C48FCF759FD2B68C9
:1040C80043E72B48FCF754FD2B683BE72948FCF7EE
:1040D8004FFD2B6833E79A8AB2F57A7FBFF423AF96
:1040E8004FF47A729A821EE718231370F1E643F0B0
:1040F80008032B6020E700BF70C30308C0BE030895
:104108005C390020207A0308A06B0308948C0020F7
:1041180098510020E8640020208D0020E4640020ED
:1041280010570020508E0020096000028886002069
:10413800382400209035002094470020403F00207C
:10414800E42000207C2400206C240020CA3E0020AB
:1041580078260020C0C9FB48AC24002017B7D13806
:104168007C260020944500200940000201600002DE
:10417800092000020860000202F003080000040899
:1041880008B512F049FFFCF731FD12F02DFFFFF7DB
:1041980063FE0120BDE808402DF002B838B50D4C8B
:1041A8000D4DAC4206D2616820461434FCF7AAFCD7
:1041B800AC42F8D3FDF7A4FB084A094B094C14603C
:1041C800002209491A705A7008480860BDE838404A
:1041D80018F0E0BCC0BE030870C30308E464002004
:1041E800948C0020208D0020E86400209851002045
:1041F80008B5FFF7D3FF12F00FFFFCF7F7FCBDE897
:10420800084012F0F1BE054B10B59A68044C2178AD
:10421800501C09B99A6010BD0246F8E740230020F7
:10422800AB270020F0B50C292BD8DFE801F06F2A66
:104238002A2A4C2A2A2A2B2A2A2A0700046AB2F890
:104248000CE097881668674D24F480540462036A6A
:104258004468C16923F4005343EA0E3321F4E6416C
:10426800A84243EA073341EA062100F0B58005F584
:104278000065A84200F0B08092684460C1610264A1
:104288000362F0BD046A96899588D2F800E0554F1C
:1042980024F480740462036A4468C16923F40073D7
:1042A80043EA062321F07301B84243EA052341EAB1
:1042B8000E017ED04C4DA8427BD092684460C1610B
:1042C800C2630362F0BD046A96899588D2F800E05B
:1042D800444F24F010040462036A4468816923F09F
:1042E800200321F0807143EA061321F4E641B84225
:1042F80043EA051341EA0E2148D03B4DA84245D078
:1043080092684460816182630362F0BD046A9389A4
:10431800B2F804E01768334E24F001040462056A19
:104328004468816943EA0E0321F4803125F00205CF
:104338009BB221F07301B04243EA050341EA070149
:1043480014D0294DA84211D005F54065A8420DD0DA
:1043580005F58065A84209D005F58065A84205D015
:1043680092684460816142630362F0BDD689158A10
:10437800578A23F0080333433D43D68824F4407416
:1043880023F00403ADB233432C43E9E7D589178AF8
:10439800D68823F0800343EA051324F44064558A41
:1043A80023F0400344EA870443EA061344EA8504F9
:1043B800A6E7D589178AD68823F4006343EA05233C
:1043C80024F44054558A23F4806344EA071443EAEA
:1043D800062344EA051470E7158A24F4804444EA65
:1043E800851449E7002C0140003401402DE9F04FC5
:1043F800C822002183B07848784CDFF80492784DC1
:10440800784E794FDFF8FC8131F01FF97748784909
:10441800DFF8F4E1DFF8F4C100221359834200F019
:10442800C180B3F1804F00F0C980AB4200F0C88072
:10443800B34200F0C780BB4200F0C680734500F06D
:10444800C580634500F0C480434500F0C380DFF8B1
:10445800C0A153457ED00AF5806A534508BF092399
:1044680079D01432B42AD8D15C4C624D624E604F78
:1044780004F1B40802E01434A04568D0A379002BF5
:10448800F9D023794FEA131909F1FF39B9F1050F6A
:1044980003F00F03EFD835F8190040FA03F2D207FA
:1044A800E9D54FF0010A0AFA03F3013B18402FF04F
:1044B800B9FC16F809305149184411EBC002DAD09A
:1044C80051F83000DFF84CE1217A00F138439B0ABB
:1044D8001EF8033003F01F0E5B09022B0AFA0EFACE
:1044E80062D0032B65D0012B03D17B694AEA030311
:1044F8007B6193880093B3FA83F3C3F11F039BB2E4
:10450800DA0800EB820203F00703D2F820E09B00F0
:104518004FF00F0C0CFA03FC2EEA0C0EC2F820E048
:10452800D2F820E001FA03F343EA0E031362694666
:104538000023022214348DF804208DF805308DF8FC
:1045480006308DF807301FF0C7FBA04596D103B0A1
:10455800BDE8F08F082309EBC3034FF0010B93F874
:104568002CA00AF01F034FEA5A1ABAF1020F0BFAED
:1045780003F30BD0BAF1030F0ED0DA457FF471AF15
:10458800D1F814A043EA0A034B616AE7D1F818A0EE
:1045980043EA0A038B6164E7D1F81CA043EA0A03E3
:1045A800CB615EE70023D6E7BB694AEA0303BB6138
:1045B8009FE7FB694AEA0303FB619AE70123CAE71D
:1045C8000223C8E70323C6E70423C4E70523C2E799
:1045D8000623C0E70723BEE7344C0020047E030807
:1045E800000400400008004000100040002C01407A
:1045F80000100240987F0308A47F0308E88A00207F
:1046080048580308004001400014004000340140AD
:1046180000440140AC7F0308002867D003682DE9F7
:10462800F04F03F138445C4EA40A0125345D04F0D0
:104638001F066409022C05FA06F558D0032C00F071
:10464800A580012C58D08088B0FA80F4C4F11F04EA
:10465800A4B2E50803EB850504F007042E6AA4005C
:104668000F27A74026EA07062E622E6A01F00307E5
:10467800A2407C1E3243012CC1F3810CC1F3001807
:104688002A62C1F341113CD9C60700F18980850728
:1046980000F19580440700F1A380020700F1B18082
:1046A800C60600F1BF80850600F1CD80440600F102
:1046B800DB80020600F1E980C60500F1F780850578
:1046C80000F10581440500F11381020500F1218103
:1046D800C60400F12F81850400F13D81440400F1F6
:1046E8004B81020400F15981BDE8F08F70472B4CD3
:1046F800A6693543A561A6E7284C66693543656117
:10470800A1E7002422464FF0010E4FF0030904E010
:104718000132102A04F10204E6D00EFA02F636EA53
:104728000005F5D1D3F808A009FA04F5ED430AEA23
:10473800050AC3F808A0D3F808B00CFA04FA4AEA44
:104748000B0AC3F808A0B3F804A01FFA8AFA2AEAE9
:1047580006069E80B3F804A008FA02F646EA0A069E
:10476800B6B29E801E682E401E60D3F800A007FADD
:1047780004F646EA0A061E60D3F80CA001FA04F60D
:1047880005EA0A0A46EA0A05DD60C1E7034CE6695C
:104798003543E56157E700BFAC7F030800100240CE
:1047A8001A6822F003021A601A683A431A60DA6833
:1047B80022F003020A438507DA607FF56BAF1A68B7
:1047C80022F00C021A601A6842EA87021A60DA6854
:1047D80022F00C0242EA81024407DA607FF55DAFFD
:1047E8001A6822F030021A601A6842EA07121A6040
:1047F800DA6822F0300242EA0112DA6002077FF535
:104808004FAF1A6822F0C0021A601A6842EA87128B
:104818001A60DA6822F0C00242EA8112C606DA603B
:104828007FF541AF1A6822F440721A601A6842EAAA
:1048380007221A60DA6822F4407242EA01228506E9
:10484800DA607FF533AF1A6822F440621A601A689A
:1048580042EA87221A60DA6822F4406242EA812238
:104868004406DA607FF525AF1A6822F440521A60D0
:104878001A6842EA07321A60DA6822F4405242EAB9
:104888000132DA6002067FF517AF1A6822F4404257
:104898001A601A6842EA87321A60DA6822F44042DB
:1048A80042EA8132C605DA607FF509AF1A6822F458
:1048B80040321A601A6842EA07421A60DA6822F43B
:1048C800403242EA01428505DA607FF5FBAE1A689C
:1048D80022F440221A601A6842EA87421A60DA68AB
:1048E80022F4402242EA81424405DA607FF5EDAEC7
:1048F8001A6822F440121A601A6842EA07521A60CB
:10490800DA6822F4401242EA0152DA6002057FF5C1
:10491800DFAE1A6822F440021A601A6842EA875227
:104928001A60DA6822F4400242EA8152C604DA6068
:104938007FF5D1AE1A6822F040721A601A6842EA0E
:1049480007621A60DA6822F0407242EA016285045E
:10495800DA607FF5C3AE1A6822F040621A601A68FE
:1049680042EA87621A60DA6822F0406242EA8162AB
:104978004404DA607FF5B5AE1A6822F040521A6036
:104988001A6842EA07721A60DA6822F0405242EA6C
:104998000172DA6002047FF5A7AE1A6822F040427D
:1049A8001A601A6842EA87771F60DA6822F0404284
:1049B80042EA8171D960BDE8F08F00BF03682DE934
:1049C800F04F03F13845644EAD0A0124755D05F0DA
:1049D8001F066D09022D04FA06F400F0A280032DCB
:1049E80000F0A480012D52D08088B0FA80F4C4F180
:1049F8001F04A4B2E50803EB850504F007042E6A3A
:104A0800A4000F27A74026EA07062E622E6A01F0A7
:104A1800030702FA04F47A1E3443012AC1F3810C15
:104A2800C1F300182C62C1F3411135D9C60700F152
:104A38009780850700F1A380440700F1B180020741
:104A480000F1BF80C60600F1CD80850600F1DB804D
:104A5800440600F1E980020600F1F780C60500F17E
:104A68000581850500F11381440500F121810205C6
:104A780000F12F81C60400F13D81850400F14B81CE
:104A8800440400F15981020455D4BDE8F08F334D38
:104A98006E6934436C61A7E7002422464FF0010E8B
:104AA8004FF0030904E00132102A04F10204ECD0AB
:104AB8000EFA02F636EA0005F5D1D3F808A009FA8D
:104AC80004F5ED430AEA050AC3F808A0D3F808B0CC
:104AD8000CFA04FA4AEA0B0AC3F808A0B3F804A0CF
:104AE8001FFA8AFA2AEA06069E80B3F804A008FA92
:104AF80002F646EA0A06B6B29E801E682E401E607E
:104B0800D3F800A007FA04F646EA0A061E60D3F8AE
:104B18000CA001FA04F605EA0A0A46EA0A05DD606D
:104B2800C1E70E4DAE693443AC615DE70B4DEE69EC
:104B38003443EC6158E71A6822F040421A601A6858
:104B480042EA87771F60DA6822F0404242EA8171C0
:104B5800D960BDE8F08F00BFAC7F030800100240A9
:104B68001A6822F003021A601A683A431A60DA686F
:104B780022F003020A438507DA607FF55DAF1A6801
:104B880022F00C021A601A6842EA87021A60DA6890
:104B980022F00C0242EA81024407DA607FF54FAF47
:104BA8001A6822F030021A601A6842EA07121A607C
:104BB800DA6822F0300242EA0112DA6002077FF571
:104BC80041AF1A6822F0C0021A601A6842EA8712D6
:104BD8001A60DA6822F0C00242EA8112C606DA6078
:104BE8007FF533AF1A6822F440721A601A6842EAF5
:104BF80007221A60DA6822F4407242EA0122850626
:104C0800DA607FF525AF1A6822F440621A601A68E4
:104C180042EA87221A60DA6822F4406242EA812274
:104C28004406DA607FF517AF1A6822F440521A601A
:104C38001A6842EA07321A60DA6822F4405242EAF5
:104C48000132DA6002067FF509AF1A6822F44042A1
:104C58001A601A6842EA87321A60DA6822F4404217
:104C680042EA8132C605DA607FF5FBAE1A6822F4A3
:104C780040321A601A6842EA07421A60DA6822F477
:104C8800403242EA01428505DA607FF5EDAE1A68E6
:104C980022F440221A601A6842EA87421A60DA68E7
:104CA80022F4402242EA81424405DA607FF5DFAE11
:104CB8001A6822F440121A601A6842EA07521A6007
:104CC800DA6822F4401242EA0152DA6002057FF5FE
:104CD800D1AE1A6822F440021A601A6842EA875272
:104CE8001A60DA6822F4400242EA8152C604DA60A5
:104CF8007FF5C3AE1A6822F040721A601A6842EA59
:104D080007621A60DA6822F0407242EA016285049A
:104D1800DA607FF5B5AE1A6822F040621A601A6848
:104D280042EA87621A60DA6822F0406242EA8162E7
:104D38004404DA607FF5A7AE1A6822F040521A6080
:104D48001A6842EA07721A60DA6822F0405242EAA8
:104D58000172DA6097E600BF10B50409013C052C22
:104D680017D80D4B33F8142000F00F0042FA00F367
:104D780013F001030DD0012303FA00F001381040AD
:104D88002FF050F8054A064B125D104403EBC000A3
:104D980010BD002010BD00BF987F0308A47F030842
:104DA800E88A002001490248FEF74ABDD44C002099
:104DB8000048014001490248FEF742BDAC4C0020C2
:104DC8000034014001490248FEF73ABDAC4C0020CE
:104DD8000034014001490248FEF732BD844C0020EE
:104DE8000004004002494FF08040FEF729BD00BF93
:104DF8005C4C002001490248FEF722BD344C0020DB
:104E0800002C014001490248FEF71ABD344C00202D
:104E1800002C01402DE9F04104684A4DA30AAB4239
:104E280072D009D8B3F5801F6AD04A3DAB425AD137
:104E38004FF0700E022608E0434DAB4268D00535AE
:104E4800AB4252D14FF0C00E042647794FEA970C77
:104E5800002961D0B000634685190227D4F80C8078
:104E68009F400CEB4503BFB2384D03F1040C47EAF1
:104E7800080745F8231045F82C20E760EFF3118167
:104E8800502282F31288821905EBC202136973B3A8
:104E980013620433821905EBC202576917B11F6008
:104EA80053690433821905EBC202976917B11F6071
:104EB80093690433821905EBC202D76917B11F60E1
:104EC800D36904330027CAB21F6082F311883044C3
:104ED80005EBC000036A6BB9E3684FF6FE72134036
:104EE800E360BDE8F081BDE8F081BDE8F08105EB45
:104EF8000E03CFE7E36843F00103E360BDE8F08108
:104F08004FF0480E0126A0E74FF0200E00269CE740
:104F18004FF0980E032698E7BF08022306FA03F01D
:104F2800BB40DB43E768094D9BB23B4087190CEB5C
:104F3800470CE3600CF1040345F82C1045F82320D6
:104F48009CE700BF4B0010004D001000344C0020BF
:104F580030B503685C4D18885C4CB4FBF2F201393B
:104F6800013AAB4294B283B089B282B266D0584853
:104F7800834263D0B3F1804F60D0A0F5983083426C
:104F88005CD000F58060834258D0524883425BD0A1
:104F980000F5806083427DD022F4407200F58C30A9
:104FA80092B283421A80D9621C850ED0484A934235
:104FB8000BD002F54062934207D002F5806293421B
:104FC80003D002F58062934201D100221A860122A1
:104FD8005A611A883C4992B242F001028B421A8007
:104FE80062D0B3F1804F61D03B4A934260D002F562
:104FF800806293425ED002F5006293425CD002F573
:10500800806293425AD002F59032934258D002F50A
:105018004062934256D002F5806293421ED002F558
:105028008062934208BF092219D002A84FF00123D9
:1050380040F8043D1EF01AFE03B030BD254822F0AA
:105048007002834292B2A3D101201A80D9621C85D2
:1050580058611A8892B202431A80C5E708221F4B8A
:1050680003EBC20301A893F82D408DF804400123F7
:1050780000228DF805308DF807308DF806201EF0D7
:10508800F5FD1B2CD8D1164B019301A81EF0EEFD9F
:1050980003B030BD01201A80D9621C8558611A8876
:1050A80092B202431A809CE70022D8E70122D6E791
:1050B8000222D4E70322D2E70422D0E70522CEE772
:1050C8000622CCE70722CAE7002C014000A24A04C6
:1050D8000034014000100040000400404858030814
:1050E80019010001204B98422DD0B0F1804F2CD0EF
:1050F800A3F5943398422AD003F58063984228D0C8
:1051080003F50063984226D003F58063984224D0C3
:1051180003F59033984222D003F54063984220D09B
:1051280003F58063984207D003F58063984208BF6F
:10513800092202D00020704708220C4B03EBC2035F
:1051480093F82C0070470022F7E70122F5E70222C6
:10515800F3E70322F1E70422EFE70522EDE7062251
:10516800EBE70722E9E700BF002C01404858030895
:105178002DE9F04F013085B0C3B203930B4602917D
:105188008B4C8C4E002B00F09A8032208A4D8B4F2E
:10519800DFF82C9228F018F84FF4FA7A4FF0100C38
:1051A8004FF47A70D9F80430C3F30803002B40F0A9
:1051B800DE80EFF31183002B40F0D9802968A268C4
:1051C80000BF2B689942F9D1D7F800E000FB0EF335
:1051D8009B1AB3FBFEF300FB01314FF0010E019166
:1051E800D9F80430C3F30803002B40F08780EFF3AD
:1051F8001183002B40F082802B68A16800BF2A68C9
:105208009342F9D1D7F800B000FB0BF2521AB2FB67
:10521800FBF200FB0323019A9B1AB3F57A7FDFD3D5
:10522800BAF1010ABED1039B002B40F0BD804FF4B8
:105238007A7ADFF88C9150464FF0100CD9F8043088
:10524800C3F30803002B75D1EFF31183002B71D141
:105258002968A26800BF2B689942F9D1D7F800E005
:1052680000FB0EF39B1AB3FBFEF300FB01314FF07A
:10527800010E0191D9F80430C3F3080313BBEFF30F
:105288001183FBB92B68A16800BF2A689342F9D142
:10529800D7F800B000FB0BF2521AB2FBFBF200FB8E
:1052A8000323019A9B1AB3F57A7FE3D3BAF1010A73
:1052B800C4D1029B013B0293002B7FF466AF05B07B
:1052C800BDE8F08FEFF311888CF31288A16823688A
:1052D800DB0344BFC6F800E0A1682B6832685FFAB8
:1052E80088F888F31188D7F800801A4400FB08F37F
:1052F8005B1AB3FBF8F300FB0233D2E7EFF3118834
:105308008CF31288A1682368DB0344BFC6F800E069
:10531800A1682B6832685FFA88F888F31188D7F893
:1053280000801A4400FB08F35B1AB3FBF8F300FB98
:10533800023370E7EFF311828CF31288D4F808E097
:105348002368D90303D501233360D4F808E02B6818
:105358003168D2B282F311883A68194400FB02F32B
:10536800A3EB0E03B3FBF2F300FB01317FE7EFF38E
:1053780011828CF31288D4F808E02368D90303D586
:1053880001233360D4F808E02B683168D2B282F385
:1053980011883A68194400FB02F3A3EB0E03B3FB30
:1053A800F2F300FB013118E7184627F07DFD3EE7D0
:1053B80010E000E0AC850020B0850020B485002016
:1053C80000ED00E0204B5B68C3F3080330B4BBB9C1
:1053D800EFF31183A3B91D4B1D4C1868A16800BFDA
:1053E8001A689042F9D11B4B1C684FF47A7202FB81
:1053F80004F3591AB1FBF4F130BC02FB00107047FA
:10540800EFF31182102383F3128811498C680B681B
:1054180013F4803F104B02D0012018608C680B49B0
:10542800D2B20D68186882F311880A4B19684FF4D4
:105438007A72284402FB01F31B1B30BCB3FBF1F367
:1054480002FB0030704700BF00ED00E0B08500208F
:1054580010E000E0B4850020AC8500202DE9F84F6D
:105468008046FFF7AFFF254E2549DFF8A0E0254A23
:10547800254D844610274FF47A740120DEF8043055
:10548800C3F30803D3B9EFF31183BBB90B68D2F8A0
:1054980008A000BFD1F800904B45F7D1D6F800B06E
:1054A80004FB0BF9A9EB0A09B9FBFBF904FB03930D
:1054B800A3EB0C034345E1D3BDE8F88FEFF3118A62
:1054C80087F31288D2F808B01368DB0344BF28605A
:1054D800D2F808B00B68D5F800905FFA8AFA8AF318
:1054E8001188D6F800A0994404FB0AF3A3EB0B0338
:1054F800B3FBFAF304FB0933DAE700BFB4850020F5
:10550800B085002010E000E0AC85002000ED00E050
:105518002DE9F04FDFF830C1474A4849484E494D18
:105528008046102718F1FF38C0F08480DCF804307A
:10553800C3F30803002B5CD1EFF31183002B58D180
:105548000B68946800BF08688342F9D1D6F80090C8
:105558004FF47A7000FB09FEAEEB040EBEFBF9FEB9
:1055680000FB03EEDCF80430C3F308034FF47A744D
:105578000120FBB9EFF31183E3B90B68D2F808A057
:1055880000BFD1F800904B45F7D1D6F800B004FB26
:105598000BF9A9EB0A09B9FBFBF904FB0393A3EB8D
:1055A8000E03B3F57A7FBDD2DCF80430C3F30803E9
:1055B800002BDFD0EFF3118A87F31288D2F808B0F6
:1055C8001368DB0344BF2860D2F808B00B68D5F82D
:1055D80000905FFA8AFA8AF31188D6F800A09944F5
:1055E80004FB0AF3A3EB0B03B3FBFAF304FB093345
:1055F800D5E7EFF3118487F31288D2F8089013687F
:10560800D80303D501232B60D2F808900B682868CB
:10561800E4B284F31188D6F800A04FF47A7400EB52
:10562800030E04FB0AF3A3EB0903B3FBFAF304FB31
:105638000E3E97E7BDE8F08F10E000E0B08500204F
:10564800B4850020AC85002000ED00E030B4EFF315
:105658001183102282F312880649074C0A6807480A
:10566800013200250A602560DBB2026883F31188E5
:1056780030BC7047B0850020AC85002010E000E009
:105688000F4B1B88014643B90E4B0F4A1B78106815
:105698000BB981F00101FBF79EB80C4B5A691AB19E
:1056A80018B91A68106058747047094A1868118840
:1056B800084A92FBF1F2012102605974704700BF59
:1056C800888500208A8500208C8500209085002010
:1056D800A885002020A107001D4B70B59C68236D8C
:1056E800626BDD69C2B1A36B2BB12B0702D5236DA9
:1056F80008221A6270BD2A06F7D5A26A616A8A4230
:1057080020D0511CA069A162825C2069266D81426B
:105718003285EAD3A362E8E7A906E4D5E26A22B1B2
:10572800988C216B80B29047DDE7E1699B8C6069BA
:10573800DBB24E1CE6614354E169E368994228BF35
:10574800E261D0E7226D136823F080031360CCE791
:105758004C2F00201D4B70B55C68236D626BDD69B2
:10576800C2B1A36B2BB12B0702D5236D08221A6295
:1057780070BD2A06F7D5A26A616A8A4220D0511CF8
:10578800A069A162825C2069266D81423285EAD3D4
:10579800A362E8E7A906E4D5E26A22B1988C216BF6
:1057A80080B29047DDE7E1699B8C6069DBB24E1CF3
:1057B800E6614354E169E368994228BFE261D0E7B2
:1057C800226D136823F080031360CCE74C2F002070
:1057D8001D4B70B51C68236D626BDD69C2B1A36B8C
:1057E8002BB12B0702D5236D08221A6270BD2A0639
:1057F800F7D5A26A616A8A4220D0511CA069A162C9
:10580800825C2069266D81423285EAD3A362E8E78B
:10581800A906E4D5E26A22B1988C216B80B2904740
:10582800DDE7E1699B8C6069DBB24E1CE66143549D
:10583800E169E368994228BFE261D0E7226D136805
:1058480023F080031360CCE74C2F002070B4EFF3F3
:105858001186502383F31288836B1A68D20720D4E9
:105868005D686DB9446A826A944217D081691144AF
:10587800D9600ED9A21A5A608462002280F8542096
:105888001A6842F00102F1B21A6081F3118870BC03
:10589800704701698A1A5A608562EEE7012380F829
:1058A8005430F1B281F3118870BC704703685B6AA9
:1058B80003B11847704700BF03681B6A03B1184754
:1058C800704700BF03682DE9F041DF691FB13B460F
:1058D800BDE8F0411847002A164611DD04460D467A
:1058E8000E4400E023689B68204698470028F9D0BA
:1058F800236815F8011B1B6820469847AE42F1D172
:10590800BDE8F0810368DB68184700BF03689B683F
:10591800184700BF03685B68184700BF03681B6827
:10592800184700BF10B40B4B0B4A1C780123834067
:10593800234052F8200031B9B3FA83F149095DF8E0
:10594800044BFAF748BF191C18BF01215DF8044B36
:10595800FAF741BF788500207C8500201C4C08B5EB
:1059680001210220FFF7DEFF237803F00502052A54
:105978002AD003F00903092B08D000210120FFF7E2
:10598800D1FF00210846FFF7CDFFFEE7114A124B71
:1059980011681A680B68114C4FF6FE7003400B60D3
:1059A8001388206823F001031B041B0C138018B113
:1059B8002A2200238271C3710A224E21FEF72CFE8F
:1059C8002068FAF7FEFED8E71AF040FA2378D0E705
:1059D800482F0020B4270020B8270020E42F0020FB
:1059E800054B53F8203033B11A689B88918A0B42D3
:1059F80018BF1B04936170477C850020036803F17E
:105A080038422DE9F04F920A584DAA5C02F01F0562
:105A180052090124022A04FA05F400F08C80032AB2
:105A280000F08E80012A3CD001F003077A1E012A7B
:105A3800C1F3810CC1F300188088C1F3411135D935
:105A4800C60700F19780850700F1A380440700F19D
:105A5800B180020700F1BF80C60600F1CD8085063F
:105A680000F1DB80440600F1E980020600F1F780CE
:105A7800C60500F10581850500F11381440500F193
:105A88002181020500F12F81C60400F13D818504C2
:105A980000F14B81440400F15981020455D4BDE85A
:105AA800F08F334A55692C435461BDE700242246E0
:105AB8004FF0010E4FF0030904E00132102A04F1FF
:105AC8000204ECD00EFA02F636EA0005F5D1D3F856
:105AD80008A009FA04F5ED430AEA050AC3F808A084
:105AE800D3F808B00CFA04FA4AEA0B0AC3F808A07B
:105AF800B3F804A01FFA8AFA2AEA06069E80B3F8C9
:105B080004A008FA02F646EA0A06B6B29E801E68A3
:105B18002E401E60D3F800A007FA04F646EA0A06EB
:105B28001E60D3F80CA001FA04F605EA0A0A46EA50
:105B38000A05DD60C1E70E4A95692C43946173E755
:105B48000B4AD5692C43D4616EE71A6822F04042AB
:105B58001A601A6842EA87771F60DA6822F04042C2
:105B680042EA8171D960BDE8F08F00BFAC7F0308BD
:105B7800001002401A6822F003021A601A683A43B9
:105B88001A60DA6822F003020A438507DA607FF5B3
:105B98005DAF1A6822F00C021A601A6842EA87029E
:105BA8001A60DA6822F00C0242EA81024407DA60DD
:105BB8007FF54FAF1A6822F030021A601A6842EA7D
:105BC80007121A60DA6822F0300242EA0112DA603B
:105BD80002077FF541AF1A6822F0C0021A601A68FE
:105BE80042EA87121A60DA6822F0C00242EA811299
:105BF800C606DA607FF533AF1A6822F440721A607D
:105C08001A6842EA07221A60DA6822F4407242EA05
:105C180001228506DA607FF525AF1A6822F4406212
:105C28001A601A6842EA87221A60DA6822F4406227
:105C380042EA81224406DA607FF517AF1A6822F437
:105C480040521A601A6842EA07321A60DA6822F487
:105C5800405242EA0132DA6002067FF509AF1A685B
:105C680022F440421A601A6842EA87321A60DA68F7
:105C780022F4404242EA8132C605DA607FF5FBAE83
:105C88001A6822F440321A601A6842EA07421A6017
:105C9800DA6822F4403242EA01428505DA607FF58B
:105CA800EDAE1A6822F440221A601A6842EA874266
:105CB8001A60DA6822F4402242EA81424405DA6036
:105CC8007FF5DFAE1A6822F440121A601A6842EAB9
:105CD80007521A60DA6822F4401242EA0152DA6086
:105CE80002057FF5D1AE1A6822F440021A601A68DC
:105CF80042EA87521A60DA6822F4400242EA815284
:105D0800C604DA607FF5C3AE1A6822F040721A60E2
:105D18001A6842EA07621A60DA6822F0407242EAB8
:105D280001628504DA607FF5B5AE1A6822F0406238
:105D38001A601A6842EA87621A60DA6822F04062DA
:105D480042EA81624404DA607FF5A7AE1A6822F05D
:105D580040521A601A6842EA07721A60DA6822F03A
:105D6800405242EA0172DA6097E600BF2DE9F04F2F
:105D78004A484B4B4B4C4FF090414FF0010A4FF0C3
:105D880002094FF004084FF0080C4FF0100E2027BE
:105D98004026802530F8022B12F0010F03D019603D
:105DA800A3F804A0083312F0020F03D01960A3F877
:105DB8000490083312F0040F03D01960A3F804808C
:105DC800083312F0080F03D01960A3F804C0083391
:105DD80012F0100F03D01960A3F804E0083312F092
:105DE800200F02D019609F80083312F0400F02D0B4
:105DF80019609E80083312F0800F02D019609D80D0
:105E0800083312F4807F05D04FF4807B1960A3F823
:105E180004B0083312F4007F05D04FF4007B1960FA
:105E2800A3F804B0083312F4806F05D04FF4806BE8
:105E38001960A3F804B0083312F4006F05D04FF4CA
:105E4800006B1960A3F804B0083312F4805F05D022
:105E58004FF4805B1960A3F804B0083312F4005FB4
:105E680005D04FF4005B1960A3F804B0083312F4AE
:105E7800804F05D04FF4804B1960A3F804B0083365
:105E8800D20B04D04FF4004219609A80083301F510
:105E98008061A1427FF47EAFBDE8F08F987F030850
:105EA800E88A002000180048002852D0036803F14F
:105EB80038422DE9F04F920A504DAA5C02F01F05B6
:105EC80052090124022A04FA05F443D0032A00F0F7
:105ED8009080012A43D001F003077A1E012AC1F3FA
:105EE800810CC1F300188088C1F341113CD9C60761
:105EF80000F18880850700F19480440700F1A280B2
:105F0800020700F1B080C60600F1BE80850600F1E8
:105F1800CC80440600F1DA80020600F1E880C6056C
:105F280000F1F680850500F10481440500F1128135
:105F3800020500F12081C60400F12E81850400F1DC
:105F48003C81440400F14A81020400F15881BDE813
:105F5800F08F70472A4A95692C439461BBE7284A19
:105F680055692C435461B6E7002422464FF0010ED0
:105F78004FF0030904E00132102A04F10204E6D0CC
:105F88000EFA02F636EA0005F5D1D3F808A009FAA8
:105F980004F5ED430AEA050AC3F808A0D3F808B0E7
:105FA8000CFA04FA4AEA0B0AC3F808A0B3F804A0EA
:105FB8001FFA8AFA2AEA06069E80B3F804A008FAAD
:105FC80002F646EA0A06B6B29E801E682E401E6099
:105FD800D3F800A007FA04F646EA0A061E60D3F8CA
:105FE8000CA001FA04F605EA0A0A46EA0A05DD6089
:105FF800C1E7034AD5692C43D4616CE7AC7F030839
:10600800001002401A6822F003021A601A683A4324
:106018001A60DA6822F003020A438507DA607FF51E
:106028006CAF1A6822F00C021A601A6842EA8702FA
:106038001A60DA6822F00C0242EA81024407DA6048
:106048007FF55EAF1A6822F030021A601A6842EAD9
:1060580007121A60DA6822F0300242EA0112DA60A6
:1060680002077FF550AF1A6822F0C0021A601A685A
:1060780042EA87121A60DA6822F0C00242EA811204
:10608800C606DA607FF542AF1A6822F440721A60D9
:106098001A6842EA07221A60DA6822F4407242EA71
:1060A80001228506DA607FF534AF1A6822F440626F
:1060B8001A601A6842EA87221A60DA6822F4406293
:1060C80042EA81224406DA607FF526AF1A6822F494
:1060D80040521A601A6842EA07321A60DA6822F4F3
:1060E800405242EA0132DA6002067FF518AF1A68B8
:1060F80022F440421A601A6842EA87321A60DA6863
:1061080022F4404242EA8132C605DA607FF50AAFDE
:106118001A6822F440321A601A6842EA07421A6082
:10612800DA6822F4403242EA01428505DA607FF5F6
:10613800FCAE1A6822F440221A601A6842EA8742C2
:106148001A60DA6822F4402242EA81424405DA60A1
:106158007FF5EEAE1A6822F440121A601A6842EA15
:1061680007521A60DA6822F4401242EA0152DA60F1
:1061780002057FF5E0AE1A6822F440021A601A6838
:1061880042EA87521A60DA6822F4400242EA8152EF
:10619800C604DA607FF5D2AE1A6822F040721A603F
:1061A8001A6842EA07621A60DA6822F0407242EA24
:1061B80001628504DA607FF5C4AE1A6822F0406295
:1061C8001A601A6842EA87621A60DA6822F0406246
:1061D80042EA81624404DA607FF5B6AE1A6822F0BA
:1061E80040521A601A6842EA07721A60DA6822F0A6
:1061F800405242EA0172DA6002047FF5A8AE1A68DA
:1062080022F040421A601A6842EA87771F60DA680B
:1062180022F0404242EA8171D960BDE8F08F00BFA8
:106228002DE9F04FBF4B1E788BB0002E40F0BC809C
:10623800BD4BBE4C1D78DFF814A3DFF81493DFF8CC
:10624800148305F00105A4F10A0B54F80A3CBBB10C
:10625800CC2707FB06B71846FFF75CFB80B154F85C
:106268000A0CFFF74FFB14F8023C8BB9242831D0F5
:10627800F5B154F80A3C1846FFF74CFB0028EED15C
:106288000136032E04F1CC04DFD10BB0BDE8F08F4A
:10629800012B23D0022B2BD0032B37D0042B67D014
:1062A800052B40D0062B4FD054F80A2C1346D2E7C2
:1062B80054F80A3C23281A4600F087819C4991F833
:1062C80022108142C7D19B4BCAF80090C3F80C80BA
:1062D8001346C0E7012304F8023CCAE74D2854F8E6
:1062E8000A2C0CBF0223002304F8023C1346B2E731
:1062F80000233C2804F8023C45D03E28D4D1012292
:10630800032304F8012C04F8023CB2E7C02814D88F
:106318000022042304F8050C04F8040C04F8062CE5
:1063280004F8023CA5E714F8063C14F8052C9A4238
:106338002FD814F8043C834203D0002304F8023C0D
:1063480097E7062304F8023C14F801ECBEF1000FAD
:1063580000F07E81BEF1010F00F0C28101360023FA
:10636800032E04F8023C04F1CC047FF46EAF8CE7F2
:1063780014F8043C04F8030C5840052304F8040CF2
:1063880004F8023C75E7032204F8013C04F8022CE7
:106398006FE714F8042CF9184240013304F8042C70
:1063A80004F8063C887264E7634B186800283FF4D9
:1063B8006CAFFAF753FBDFF8A0A1604DDFF89C91B2
:1063C800DAF80000FFF7A6FA00283FF45EAFDAF823
:1063D8000000FFF797FA09281BD03F2819D02B682F
:1063E800002B66D1042800F0A6810C2800F0E68076
:1063F8007F28E5D0A0F12002D2B25E2AE0D80BB9FE
:106408002028DDD05A1C09F803002A600EF002FA91
:10641800D6E72C68002C5AD1494B264603F59478C8
:10642800002E08BF1E4608334345F9D1002E00F060
:106438007681A3F1080B3068DBF80020075D135D57
:106448009F42204402EB040140F06781671E4F44DD
:1064580022460BB9FD2A5CD907F8013F01322A60B0
:1064680010F8013F11F801EF9E45F2D00AB1B3458B
:1064780012D034480EF0D6F9B34508D356F8080BB5
:106488000EF0D0F909200EF0C5F95E45F6D92E4870
:106498000EF0C8F92A680024944291D2661E4E4430
:1064A80016F8010F0EF0B6F92B6801349C42F7D3A9
:1064B80086E70C2800F082800A2851D00D284FD09A
:1064C8007F2800F0FA80FF2B3FF67AAF92E71C4F47
:1064D8004FF0000B07F594785E4602E00837474511
:1064E8000DD0224639684846FAF7C6FD0028F5D18E
:1064F800BB46002EF2D13E4608374745F1D1002E63
:1065080099D1BBF1000F3FF45BAF0E480EF08AF94A
:10651800B4E7511C202009F80200296009F801306D
:106528000A46A4E7A3410020484B00205E810020D2
:106538008886002000ED00E05830002060310020FF
:10654800B47103089085030898850308FC9F002010
:10655800EFBEADDE0400FA055C300020603000209C
:106568000EF0E1F923217C482FF086F8002800F08E
:10657800E080A0EB0900286088B1431E19F80310D9
:10658800202940F0E68009EB030204E012F8011D1F
:10659800202946D10346581E002BF7D12B604FF413
:1065A8008072002148462FF050F86C4B1B78002B66
:1065B8003FF46BAE6A480EF035F901E769480EF012
:1065C80031F967480EF02EF9FAE667496748C97845
:1065D800674ADFF8CCE1D360003118BF01210170B0
:1065E80064491161402153611176557662496348C7
:1065F8000B601032CEF80020584A012313700EF0B9
:1066080063FD57480EF00EF94FF400600AF0C4FE1F
:106618005B4B93F82230232B00F0938014F8023C54
:1066280040E62B60574C002204F5947809F80320C3
:1066380002E00834444578D0216848460DF0EAFF66
:106648000028F6D0444570D2636898470023A5E730
:106658004D4BADF822E00FCB0DF1280C02AF87E8C7
:106668000F004CF824ED14F8051C14F8033C0694AC
:1066780004EB010E624639464FF0010C06A8CDF82E
:106688001CE0ADF820308DF824C002F055FFE8B9C1
:10669800019F002304F8023C002F3FF4F1AD54F8A9
:1066A8000A0C2AF0A9F9013654F80A0CB847032E47
:1066B80004F1CC047FF4C9ADE7E5013B002233487F
:1066C8002B6009F803200EF0ADF879E6029A304BFA
:1066D80003923946A4F10A0002930BF01DFCD7E798
:1066E80014F8053C14F8032C0694234407936E2AE7
:1066F8004FF0000308930993ADF820207FF42EAEE5
:1067080006A8FAF738FD06A8FAF72AFD06A8FAF748
:1067180027FD06A8FAF724FD20E62246A6E61D482E
:10672800A3F1080B0EF07EF8A8E61B480EF07AF8E5
:106738008CE7286820E708480CF07FFE0BB0BDE81E
:10674800F08F164A14F8023CC2F80C80CAF8009080
:10675800A8E5034666E700BF60300020A34100209B
:1067680098850308A0850308948C00201828002029
:1067780040230020F93700085C300020CC8503084E
:1067880088860020B4710308C0580308C885030828
:106798000890002090850308AC85030800ED00E010
:1067A800583000202DE9F04F2DED068BA04BA14A63
:1067B8001C7897B000F59C41203181460B911160FF
:1067C800002C00F0EA869C4A1268904240F28380CE
:1067D8009A4A069216689A499A4A0591013C1C7091
:1067E800994B049206F480560893002E40F081805D
:1067F800964B1B78022B01F09481042B01F08381C6
:10680800012B01F03781924B9945089B9B7800F248
:106818009685002B40F097858E4B0793069B1E6844
:1068280016F4805740F08786DFF860A2049BB3F91E
:106838000610059B5D8BA942B4BF00250125864B38
:106848001B6813F080535ED0079A127812F0010289
:106858005FD00598408C884241F3B882002D5ED104
:106868007E4C94F88C10002959D17D487D490068E8
:1068780090F82D0000240C604C608C607A49002848
:106888004ED10870002A4FD0F0064DD5774A1278BD
:10689800D10649D4002F47D1002B45D1720243D4E9
:1068A800734B1B78002B02F01982724B9B78002DDA
:1068B80042F081823BB1704A704B12681B689B1A88
:1068C800002BC2F26D821020644C2AF083FB012356
:1068D80084F88D3028E0594B06931E68594B584A66
:1068E800049306F48056584B05920893002E3FF403
:1068F8007FAF00215848FAF7F6FF00287FF478AFF9
:106908001EF08CFE74E774029ED4079A127802F087
:106918000102524C002184F88C10002DA5D0524958
:1069280001200870002AAFD1554B1A78002A40F090
:10693800BD800599049C488BB4F90070898BB4F923
:106948000240B842B4BF8026002646F04003B94250
:10695800D8BF33469B0843F08006A042B8BF3346F1
:10696800049F43F04006A142C8BF33469B08B7F9CD
:106978000440B7F9066043F08007A042B8BF3B4621
:1069880043F04007A142C8BF3B469B0843F080073D
:10699800324C8642C8BF3B4643F0400794F88EE02D
:1069A8008E42B8BF3B469E4501F04A84A4F8902029
:1069B80084F892202E4984F88E300E78002E01F04B
:1069C8004B835F2B01F0BE836F2B01F0FD83079B88
:1069D8001B78DE076AD494F89210002966D1B4F9BE
:1069E8009030322B62DD94F88E200120572A84F8EB
:1069F80092004DD0069B1B685D0741F199825A2A87
:106A080041F0968294F89430002B42F05E8194F81D
:106A1800963083F0010384F89630002B42F0D6813B
:106A28000C202AF0D7FA174B174D099341E000BF05
:106A380028350020D43300202435002010550020AC
:106A48005C8600204A840020403F002082380020D5
:106A5800404B4C00484B0020A43E00209C230020C3
:106A6800E4640020FC380020482600206C600020E8
:106A7800E4200020E43E0020B0850020FC4C0020EB
:106A8800FB410020E8640020E0640020E03500209D
:106A9800884B894A19684FF47A73B3FBF1F3C3EB57
:106AA800431103EB8103DB00A2F8A830834B844D2C
:106AB8000993069B1B685F0700F1B4860DF1500926
:106AC800804E0A950022C9F804203446149240F6F4
:106AD800330B4FF0190840F28337049D02E0043469
:106AE800544522D0A178E378994218FB0170F6D278
:106AF80094F801E00EF1040E18FB037135F91E300D
:106B08005B45A8BF5B46B3F5617FB8BF4FF46173BF
:106B18009842E4DA9942E2DB21782729DFD848460F
:106B28000434FAF7D1FE5445DCD1674A0A9D13783C
:106B3800664A99E8030082E80300002B40F0F085DC
:106B4800634B1A78002A00F06A8501215F48FAF73A
:106B5800CAFE002840F0E782089BDB78002B40F053
:106B6800E2825C4B0A932B881FB227F001071FFAB9
:106B780087F84345A5F8008001F00280564F4FF092
:106B880002090E204FF0140A4FF0FF0B87F800900F
:106B980087F801A087F802B02AF01CFA49464B484A
:106BA800B5F80080FAF79FFE002841F09A8228F095
:106BB80002039BB243452B800BD0474B0220142184
:106BC800FF2218700E2059709A702AF003FAB5F84F
:106BD8000080424B424A197850680C9318F0030F12
:106BE80008BF81F00201C1F340010B92F9F7F3FDF0
:106BF80024213648FAF777FE30B9079A13785F07E9
:106C080044BF23F0040313700A9B1B6813F00A0F98
:106C180011D006212D48FAF766FE002801F0AD8054
:106C28002B88580641F1258207212848FAF75BFE90
:106C3800002840F0C8870C212448FAF754FE2A8817
:106C4800002800F0508342F480739A422B8009D0C8
:106C5800214B022214211A700E20FF2259709A70BB
:106C68002AF0B8F91F4B1B78082B00F048830E2B2D
:106C780000F04583069BD3F8008018F4806F6BD032
:106C8800194B1B79002B00F0308214210F48FAF7BA
:106C98002AFE002840F02E8224F076FC01202AF0FB
:106CA800E7F8002855D0DFF844A000274FF0CC0BB8
:106CB800A14620E00055002088520020E86400200A
:106CC800E06400209035002034570020A43E0020C6
:106CD800A34100208C64002008450020788500200E
:106CE8007C8500205C390020F04B00205481002076
:106CF800DFB2022F2CD80BFB07F87B1C5AF8084090
:106D0800002CF5D1032290F9023002940192C27846
:106D1800E24951F8222000921846224623460121D2
:106D280029F02AFF034607EB470000EB00100A93FF
:106D380053B121460AEB8000CC222EF086FC0A9B38
:106D48004AF808300137FFB228F038FB0028D0D1C4
:106D58004C46069BD3F80080079B93F800A0D04BC5
:106D68001AF0010A00F0418201221A70099B049965
:106D78001B68B1F906105A89CA4801279142077061
:106D880080F21982C84B4FF07E521A60059BC74F9C
:106D9800B3F81890049B97F90420B3F900303878B9
:106DA80097F801C0002AA3EB090714BF01224FF08E
:106DB800FF32002FB8BF7F42B7F5FA7FA8BF4FF464
:106DC800FA77B84280F2F4813F1A07EE907AF8EE2B
:106DD800E77AB74F4B45C7ED007A03DAF1EE677AE9
:106DE800C7ED007A049BB3F902E0AEEB0903002B70
:106DF800B8BF5B42B3F5FA7FA8BF4FF4FA73984265
:106E080080F2D3811B1A07EE903AF8EEE77AF14543
:106E1800C7ED017A03DDF1EE677AC7ED017A049BCD
:106E2800B3F90400A0EB0903002BB8BF5B42B3F52C
:106E3800FA7FA8BF4FF4FA736345CCBFA3EB0C03EA
:106E4800002302FB03F207EE902AF8EEE77A4845A2
:106E5800C7ED027ABCBFF1EE677AC7ED027A18F483
:106E6800805800F07F81B1F5FA6F924BA8BF4FF4BC
:106E7800FA61B1F57A7F1A78B8BF4FF47A71A1F543
:106E88007A71002A41F01D818B4ADFF844E282FBC7
:106E98000130CB17C3EB6013581C6FF0630C3EF93D
:106EA80010003EF913E00CFB0313A0EB0E0003FBEC
:106EB80000F382FB0312DB17C3EB62139E440FFA45
:106EC8008EFE07EE90EAB8EEE78A87ED038AB8F1FE
:106ED800000F40F066842B885A0640F1FB80774902
:106EE800774A91ED018AD2ED019A92ED026A91ED0D
:106EF800034A92ED030A91ED029A92ED007AD1EDE0
:106F0800005AD7ED011A97ED002A6E4A6E4938EEFD
:106F1800445A79EEC63A77EE007A65EE233A75EE72
:106F2800C96A75EE890A37EE401A66EEA76AB0EEAE
:106F3800633AA0EE813A13F00303B0EE665A78EE96
:106F4800044A79EE867AA0EE815AF0EE638AA4EEBE
:106F5800A73AD4EEA78AA4EEE75A33EE263AF0EE23
:106F6800687AF0EE674AF6EE008A35EE88AAE0EE17
:106F7800C14A28EEC33A35EE635A77EE293A77EEDE
:106F8800E67AAAEE233A25EE285A76EE403A34EE0F
:106F980049AAE0EE817A74EEA64AAAEE235A34EEA4
:106FA800094A37EE697A64EEA84A63EE036AE4EEAA
:106FB800074A75EEC85A36EE006A67EEA87AB0EE50
:106FC800667A95EE057AE5EE056AE5EE867AB1EE23
:106FD800648AF0EE665AF0EE476AB1EE674AE8EE68
:106FE800246A63EE270A67EEA43AE4EE275AB1EE64
:106FF800450AB0EE609AB0EE631AA4EE277A23EE43
:10700800244AE7EEA76AA5EE249AA0EE031AE8EE52
:10701800245AB0EE448A31EEA16AE0EE240AA5EEC5
:10702800278A66EEA16A72EE028AE5EE033A61EEFD
:10703800211A26EE096AA4EEA47AA0EE274A0CBF0C
:10704800D7ED022ADFED212A82ED005AA2EE256A49
:10705800E8EEA06AE2EE081A73EEA33A27EE227A67
:1070680034EE044AF0EE005AE3EEA26AA4EE226A75
:10707800A1EEA57AC7ED016AC1ED366A81ED356AE0
:1070880087ED006A81ED377A82ED013AC2ED027A26
:10709800C2ED034AF3B987ED027A1BE0DC790308F5
:1070A800494B002080260020FC250020BC3E002003
:1070B800004C0020A02700201F85EB514401002030
:1070C80078000020B00000209C2300200000000071
:1070D8009C470020BAF1000F40F024812BF0B4FF48
:1070E80017B0BDEC068BBDE8F08F079B1B78D9075E
:1070F8007FF5D2AD4FF40F7025F018F900283FF452
:1071080028AE0AF06EFF4FF40F7025F077F80028CC
:107118003FF41FAE0AF065FF4FF40F7025F06EF8CC
:107128000028EED115E69A4B0A931B689B077FF55A
:107138001AADB5F8008018F0010F7FF438AD48F0AB
:10714800010398452B803FF432AD924B0222142163
:107158001A700E20FF2259709A7029F03BFFB5F87B
:10716800008024E5059B5A8B9142C0F20685B1F553
:10717800FA6FD4BFC2EB0101C2F5FA614FF47A731A
:1071880003FB01F184480378C2F5FA62B1FBF2F11E
:10719800002B3FF479AE4378804A01FB03F182FB70
:1071A8000123C917C1EB63116EE6DFED7D7A2EE688
:1071B800DFED7B7A0DE6B1F5FA6F80F2D784187AA5
:1071C8008B1A03FB00F3C2F5FA6293FBF2F3C3F1E7
:1071D800640307EE903AF8EEE77A9FED727A724B05
:1071E80067EE877AC3ED007AD0E51B780693002B0B
:1071F8007FF4BCAD6D4A1268002A3FF4B7AD6C4A03
:10720800079212F8030CDFF8E0B11146D71E19F007
:10721800D5FA9BF80090079A002800F03086069B64
:10722800B9F1000F53D107F10801787919F0C6FABE
:10723800002841F02D855F49B87A19F0BFFA002877
:1072480000F03086B9F1020F41F01E855A49F87BEB
:1072580019F0B4FA002841F013855849387D19F01F
:10726800ADFA002800F03086B9F1040F41F004852A
:107278005349787E19F0A2FA002841F0F98451495F
:10728800B87F19F09BFA002800F03086B9F1060F94
:1072980041F0EA844C4997F8230019F08FFA002846
:1072A80041F0DE84494997F8280019F087FA002848
:1072B80000F03086B9F1080F41F0CE84444997F8C0
:1072C8002D0019F07BFA00283FF450AD09231A4627
:1072D80002EB820217443F4A7878B9788BF800307D
:1072E8001070517042E522F480739BB29A422B8051
:1072F8007FF4AEAC384B1B78082B7FF4B8AC2A88E7
:1073080022F040039BB29A422B803FF4B3AC214B4E
:10731800022214211A700E20FF2259709A7029F047
:1073280059FEA7E40C9B19780B9B01F00101186822
:10733800F9F751FA17B0BDEC068BBDE8F08F13B919
:10734800089A01239370254B089A1D7892F82140DA
:1073580007931B2019F06AFA012C05F001088146F1
:1073680000F0088705F00205089A1D4E92F82030B3
:10737800DFF878A01B4F09959346052B00F29E87EE
:10738800DFE813F0BE00B4003600FC00FE00F10098
:107398008C64002008450020A02700201F85EB51A1
:1073A800000000000AD7233CFC2500204C4B00209D
:1073B800C6440020D0440020D5440020DA440020F0
:1073C800DF440020E4440020E9440020EE4400208B
:1073D800F3440020504B00205C390020484B00202B
:1073E80094470020DC64002015000020E4200020E1
:1073F800012C04BF05238BF82030B8F1000F12D000
:10740800059B3088B3F918100022134661F30F0268
:1074180060F31F4261F30F03049861F31F43036095
:10742800032342600993BF4DDBF814102A68914288
:1074380080F0028647F230510322CBF81C108BF8FB
:107448002020022009F0A8FF1EF0E8F82968DBF8E0
:107458001C200A440421CBF818208BF82010012C9A
:1074680040F07D872A68DBF81810914280F0268763
:107478009AF8000020B919F0D9F9002840F01E87C1
:107488003A6822F002023A602A687388642101FB94
:1074980003234FF480600022CBF810308BF82020B3
:1074A8008BF8032009F048FF9BF8203065E719F0B6
:1074B800C3F9012807D19B4D72882B68642101FB11
:1074C8000233CBF81030B9F1000F02D0B379002B9A
:1074D8004BD1012C00F0F286924DDBF810102A688F
:1074E8009142C0F0318701238BF82030012C3AD02B
:1074F800F379012B46D019F01FF99BF820303CE7AF
:10750800B8F1000FD3D1099D4FF48060B9F1000F95
:1075180000F0568309F028FF089A00231361002D14
:107528003FF47CA9284629F055FD069B1E6816F4F1
:1075380080573FF479A91D217B48FAF7D4F9002830
:107548007FF472A9794B03F1500A03E004339A459A
:1075580000F0BA861A78262AF8D19978DA78914212
:10756800F4D2FFF763B96F4D8EE719F0E5F80322FF
:107578004FF47A738BF82020CBF81C30694D60E704
:10758800684D6CE719F0D8F8032240F6B8338BF849
:107598002020CBF81C30634D53E7654F3B78002B18
:1075A80001F05782634BDFF89881DFF898B1DFF874
:1075B80098A1059345465E46049099460EE019F851
:1075C80004109847032C28DC88B93B782AF8020F66
:1075D80001349C4205F1040580F24981072CE1B28F
:1075E8003046DBF80430EADD984700B2EDE738F8BA
:1075F80024206B88801A4FF47A719B1A01FB00F0E3
:1076080040F6CA0290FBF3F00844904240F2EE23A1
:10761800A8BF10469842B8BF184600B2D5E7DFF8B1
:107628002C91DFF82CA1444F0A9209F15A084FF027
:10763800010B494619F8010C19F0C0F800B399F884
:10764800040099F8023099F803E000EB400107EBD9
:107658008101013BD1F8A02003EB4303534493423B
:107668000ED097F8CC20C1F8A0300BFA00F022EA2F
:1076780000000A9B81F89CE0C1F8A43087F8CC0090
:1076880009F10609C145D4D12C4B264A1B780A9327
:10769800099BDFF8C0A012681B680B93AAF19C092C
:1076A8004FF0000B9046DAF8043083B31F7877B3B5
:1076B800DAF80820A8EB0202002A0CDB99F8CC20A3
:1076C800012101FA0BF122EA010208F5FA7189F8A1
:1076D800CC20CAF808100A9ACAB19AF8002059783A
:1076E8000432D2B2002940F0B58305990498098B79
:1076F80030F9122001F1C800824240F3F78599F869
:10770800CC109A7841FA0BF3D80740F181860BF137
:10771800010BBBF1040F0AF10C0AC4D1FFF715BA2B
:10772800024B1DE0B0850020A43E002090350020CB
:10773800543600205C8600209C230020353F002022
:1077480068360020E05100209A230020DD43002005
:10775800D05803083824002004339C423FF4F0A991
:1077680019782329F8D19878DA789042F4D2AD487C
:10777800FAF7B9F800283FF4E3A9AB4B1B6813F4F8
:10778800003341F013820022A84B1046995C14295B
:1077980002F10C0201F0BC8001301828F6D1FFF785
:1077A800CFB91D219F48FAF79EF828B100F060BDB7
:1077B8000436B4423FF48FAB31782629F8D1B27839
:1077C800F3789A42F4D2089BDB78002B7FF483ABE2
:1077D8009448FAF788F8DFED967A002801F050818E
:1077E80038EE678A934A9449FDEEC87ACDED047A5B
:1077F800BDF910301B0382FB0302DB17C3EBA21297
:10780800C9F57A731BB203FB02F343F30F334B44FE
:1078180007EE903AF8EEE77A0123C7ED037A0B708A
:10782800FFF759BB854C94F896305BB1079B1B78E2
:10783800DE0707D5049BB3F90620059B5B8B9A42AC
:1078480000F3D88511217748FAF74DF8002800F0A1
:10785800AB8294F89A302BB994F8943013B9322348
:10786800A4F89830012384F89A30FFF727B9DDF897
:107878001090734A06926F49126842F2010AA1FBFE
:10788800091B12EA0A0A4FEA9B1B00F08A826D4D17
:107898006D486E4C6E492E780078267008701EB1BF
:1078A8006B490E7886F00106644C0F2184F8241089
:1078B800002B00F0E683059D664BB5F826C0B5F8A9
:1078C80024E0059D109318462D8B0078624B129585
:1078D80094F825500995614D0495A3FB00535B0866
:1078E80003EB4303C31ADBB20F90CDF834C002F4A4
:1078F80080520C9304F128000BF59673CDF8449050
:1079080097F80080DDF82490DFF860C10994534CA3
:107918000E91139200210A930896CDF81CE0089B5B
:10792800002B00F02B83099B079D33F911201FFAC8
:1079380082FEAE454FEA410303D30D9DAE4540F2AA
:1079480062835CF82120934580F02283E25EBAF1DD
:10795800000F40F0378301314145E25200F1060043
:10796800DDDB0E9A099C3E4B84F824200F2A4946F9
:107978000CBF01220022DDF8449084F825101A700B
:1079880000F08683374B3049314ADFF8E4B008937A
:107998001C46042001230B70137009F0FDFCDBF872
:1079A8000030A1686268E3605B1A934284BF0023D9
:1079B80084F82130069B3C781E68002C01F04D802D
:1079C800059A294DB2F824E0178B244916F48056FD
:1079D800284640F0998332460EE0437803EB830350
:1079E80003EB830303F2EE239BB20132A24221F898
:1079F800023B00F102000ED015F81230002B00F007
:107A08000683022BE9D001320B8821F8023BA242FF
:107A180000F10200F0D1109A137801331370FEF7C9
:107A2800E4BE00BFA43E0020D043002044750308F4
:107A380000007A44D34D6210742600209C23002055
:107A480010550020B033002058000020353F00209A
:107A58005900002045350020ABAAAAAA4A84002074
:107A6800DE510020403F00209C3600204835002091
:107A7800B0850020D84CD4F88830A9EB0303002B3C
:107A8800FEF6C1AED54AD64B527C059933F8123072
:107A98008A7DDFEDD46A9FEDD46AC97D9BB207EE7B
:107AA800102A07EE903AB8EEC77AF8EEE77A27EE92
:107AB800267A67EE867A0B9AC4F88820C7EE876A1A
:107AC80040F2FF32FCEEE67ACDED077ABDF81C30C5
:107AD800934228BF134609B1D31A9BB2C348C44D79
:107AE8000178C44C35F81160226825F81130921BD2
:107AF80013440131C04D236001F00F021B090270CD
:107B08002B80FEF780BEFDF75DFCBC4BBC4A1B68B2
:107B1800C31A93427EF777AEB74B00221A80FEF75E
:107B280072BE059A0499537DD27D013B31F9133019
:107B38001AB1C3F53B6308331BB2A3F57A7307EE9A
:107B4800903A9FEDB07AAC4AF8EEE77A40F2FF310E
:107B580067EE877AFCEEE77ACDED077ABDF81C3040
:107B68008B4228BF0B461380FEF74DBE1B7AC3F12C
:107B7800640307EE903AFFF72EBB4146FFF702BBBE
:107B88000221A148F9F7AFFE00283FF410A82F8082
:107B980018F0020F7FF41DA848F0020343452B801C
:107BA8003FF417A8994B022214211A700E20FF22C5
:107BB80059709A7029F00EFAB5F80080FFF709B8E5
:107BC80009F0BAFBA8E4924AB2F90030002BB8BF1A
:107BD8005B42B3F5E17FBFF62EA8B2F90230002B65
:107BE800B8BF5B42B3F5E17FBFF625A8894B93ED9B
:107BF800096AD3ED076A93ED057AD3ED037A76EE39
:107C0800866A77EE877A76EEA66AB7EE007A37EE5E
:107C1800666A77EEA77AB0EEC66AF0EEE75AB4EE77
:107C2800E56AF1EE10FAB4BFB0EE655AB0EE465A06
:107C3800B5EE405AF1EE10FA40F0AD839FED767A3A
:107C4800B4EEE56AF1EE10FA44BF9FED746A36EEC1
:107C5800477AB7EE006AF4EEC66AF1EE10FAC8BFCA
:107C6800DFED6F6AF5EEC07AC8BF36EEC77AF1EE7F
:107C780010FA48BFB1EE477AF6EE007A27EE677A37
:107C8800DFED667A77EE276ABDEEE66A16EE103A01
:107C98002033402B40F25786DFED626A624ADFEDFF
:107CA800617AC2ED006AFDEEC76AC2ED017A16EE8E
:107CB800903A2033402BC2ED027A49D8DFED587A4A
:107CC800B4EEE77AF1EE10FA40F3E8879FED576AD1
:107CD800DFED576A01E0B0EE677AB4EEE67AF1EECE
:107CE80010FA77EE467AF6DC9FED527AF4EEC77A10
:107CF800F1EE10FA40F1E0879FED4C6ADFED4E6A35
:107D080001E0F0EE477AF4EEE67AF1EE10FA37EE9B
:107D1800867AF6D4DFED417AB4EEE77AF1EE10FA1E
:107D280040F38186DFED3E7A37EEC77A27EE076AA1
:107D3800DFED425ADFED426ADFED427AE6EE256A70
:107D480067EE065AE6EE267AA5EEA77AF0EE477AAF
:107D58003D4BC2ED037A1A6812F4003240F05486A3
:107D68003A4B1046995C0A2902F10C0200F0518541
:107D780001301828F6D1FEF75EBF2A8822F04003AA
:107D88009BB29A422B803EF44FAF204B0222142123
:107D98001A700E20FF2259709A7029F01BF9FEF70D
:107DA80043BF2B490E787AE594F89430002B3EF4C3
:107DB80085AE079B1B7813F001037EF47FAE01228A
:107DC80084F8943084F89520FEF778BE024C01219F
:107DD80084F88C10FEF7A3BD9C2300202885002082
:107DE800488500200000C8420000804483380020F5
:107DF800883800208438002044600020C0240020F7
:107E080060E316006F12833FA43E0020084500205F
:107E18009064002088000020A7DFA834DB0FC93F4A
:107E2800DB0F49400000000044010020DB0FC9407F
:107E3800E4CB1641DB0F49C0E4CB16C192E741B948
:107E48009730083C15A82ABED04300204475030883
:107E5800353F0020012900F0038599F8CC20012343
:107E680003FA0BF30BF1010B1343BBF1040F89F871
:107E7800CC300AF10C0A7FF416ACFEF766BE511D31
:107E8800787918F09BFC00283FF4D5A9B9F1010FC7
:107E980040F0FE8607F10D01B87A18F08FFC002833
:107EA80040F0F286B549F87B18F088FC00283FF4CA
:107EB800D4A9B9F1030F40F0E386B149387D18F031
:107EC8007DFC002840F0D886AE49787E18F076FC14
:107ED80000283FF4D4A9B9F1050F40F0C986AA4992
:107EE800B87F18F06BFC002840F0BE86A74997F8C9
:107EF800230018F063FC00283FF4D4A9B9F1070F58
:107F080040F0AE86A24997F8280018F057FC0028E0
:107F180040F0A2869F4997F82D0018F04FFC0028E2
:107F28003EF424AFB9F1090F3EF420AFFFF7CEB904
:107F38005D2A00F065855B2A00F06F825E2A00F0FA
:107F4800F885562A00F00586972A00F07586A72A34
:107F580000F0E585904D2B889B0740F0B285A2F193
:107F6800B703072B00F28B82DFE813F07D0289024A
:107F7800890289027102890265026502079B002B4A
:107F88003FD05CF8212093454FEA4103FFF4DEAC73
:107F9800824A824DD25C05EB030E002A00F09480E1
:107FA800022A47D19EF8012002EB820202EB8202EC
:107FB80002F2EE2292B2032933DD12B2BAF1000FB7
:107FC8003FF4C9AC0C9D20F81520B9F1000F03D17E
:107FD8000F9D022D7FF6BFACB0F802900288B0F872
:107FE80004E04A4496446E4A0FFA8EFE82FB0E5213
:107FF8006C4DA2EBEE7225F803E012B24FF00109C6
:10800800A9E41A464B000A9D4CF821509FE4D3B2CC
:10801800022B04D9032B7FF4F6AC7346E5E43B4608
:10802800E3E4012505FA01FE0E9D25EA0E0512B2CC
:108038000E958CE4E25ABEE75B4A1278002A7FF478
:10804800F9A9B8F1000F3FF4F5A9012C40F03681E9
:108058009BF82030FFF791B931465448F9F743FCB3
:10806800002800F0C98084F893601DF0C5FDFEF774
:10807800AEBC43F0400293422A807FF486AEFEF7FE
:10808800D3BD4B4B4B4A109201221A704A4B0493B2
:108098001B214648F9F727FC00287FF473AC474BAF
:1080A800DFF820B108931946DBF80030CA688B6006
:1080B8009B1AC82B00F2D584069B1E6806F48056CE
:1080C800A9E45B78FFF768B8CAB2022A40F2BC8319
:1080D800032AAFD1129A139D079E002D08BF32467E
:1080E80069E728F0010292B242452A803FF450AD78
:1080F8000E2087F8009087F801A087F802B028F0D2
:1081080069FFB5F8008043E500220FE0437803EBF0
:10811800830303EB830303F2EE239BB20132A242F3
:1081280021F8023B00F102003FF475AC15F812305B
:108138001BB1022BEAD00B88F0E7D3B2032BFAD895
:108148003B46EBE7B2F5FA7FFEF6B0AC94F8923016
:10815800002B7EF4ABAC079B1B7801210B4084F805
:10816800921000F0BA831DF059FA154B0A4D099385
:10817800FEF79FBC0025FFF7F7B800BFD5440020E5
:10818800DA440020DF440020E4440020E9440020D1
:10819800EE440020F3440020E06400209C360020D8
:1081A800565555550C24002038260020A43E0020A2
:1081B800DE510020453500204A840020403F002041
:1081C800E8640020B0850020B2F5FA7FFEF66EACB8
:1081D80094F89230002B7EF469AC079A127801214A
:1081E800D70784F8921000F117841DF005FDC24BE3
:1081F800C24D0993FEF75DBC079BC14A1B7810600E
:10820800DB077EF5E8ABBF4B1B78002B3EF44EAC8A
:10821800089BDB78002B7EF449AC94F8933001334B
:10822800DBB2032B84F893307EF640ACB64B5B7818
:1082380013B9002D7EF43AAC1DF0F0F9FEF7C7BB78
:10824800B24AB3491068B4F99020C66981FB0601A7
:108258008911F617701A00F5FF407F3082423EF709
:10826800A9AB891B0A4412B2A4F89020FEF7A2BB5E
:10827800089BDB78002B7FF49FAADFEDA67AA44940
:1082880038EE678AC9F5FA63FDEEC87A1BB2CDED00
:10829800047ABDF91020120381FB0201D217C2EB48
:1082A800A11203FB02F343F30F334B4407EE903A5A
:1082B800B8EEE78A87ED038AFFF77EBA099D002D9D
:1082C8003EF4ACAAFFF72EB9934A059BD588049AC9
:1082D8001B8BB2F906105A1B914240F388802B443D
:1082E8009942B4BF00250125FEF7A9BAC8398A42C8
:1082F80042DA99F8CC109A7841FA0BF3D9073FF58E
:1083080006AA524201200C9228F04AFF7B1E0C9AC2
:10831800162B00F28281DFE813F004021802EC0148
:108328003D022C025102D701C201AD01980183011F
:1083380080013D0272015102D701C2015D0149016C
:10834800350166021F01DA0018F0F6F9032140F63C
:10835800B8328BF82010CBF81C20FFF772B8AB4668
:108368000899DBF80020CB69099D13448B61002D27
:108378003EF454AAFFF7D6B899F8CC30012202FA95
:108388000BF223EA020308F5FA7289F8CC30CAF82E
:108398000820FFF7BCB9B4EEE56AF1EE10FA8CBF1D
:1083A800B0EE654AB0EE464AC4EE054A9FED5B2A38
:1083B8009FED5B5ADFED5B1ADFED5B2A9FED5B3AC1
:1083C800DFED5B3A9FED5B4AA4EE825AE4EEE12AC8
:1083D800A4EE857AA4EEA23AB0EE475AB0EE637ADC
:1083E800A4EE837AA4EE874A84EE057A28E4012570
:1083F800FEF725BA00215048F9F775FA00287FF4EE
:1084080021AA322384F89600A4F89830FFF71ABA04
:10841800002A0CBF0120022075E7484B01220220E8
:108428004749484C0B60344B2270344D099328F06F
:10843800B7FEFEF73EBB304A424B09921146424A0C
:108448000A6002225A7018F055FAFEF732BB2A4A1F
:108458003C4B099211463D4A0A6000225A7018F0B6
:1084680049FAFEF726BB244A364B09921146384A88
:108478000A6001225A7018F03DFAFEF71ABB792AF1
:1084880000F082847A2A00F076849E2A00F06B84B9
:108498009D2A00F06084AE2A00F05584AD2A00F0D1
:1084A8004A84EF2A00F04484FD2A00F03E84FB2A27
:1084B80000F02B84FE2A00F07084F72A00F07884FC
:1084C8007B2A00F01B840C4B0993FEF7F2BAD9F80B
:1084D800D000204B90F836109B7811446429A8BF2F
:1084E800642121EAE17180F83610002B40F099846C
:1084F80017F068FAB1E400BFE8640020E0640020E7
:10850800004D0020353F0020E43E00204C6600204E
:10851800D34D621000007A447C47002099FB243F29
:1085280069A2163E39094E3DE3B59E3E88FA163ECD
:1085380045FE7F3FA7DFA834A43E00206E8D0020B3
:10854800E4640020948C0020B05100209851002051
:10855800A45100206E600020D9F8D000BC4B90F8E0
:1085680037109B781144FE29A8BFFE2121EAE1714A
:1085780080F83710002BBBD0162018F0A1F9D9F8D5
:10858800D000B5E7D9F8D000B14B81781144C8299B
:10859800A8BFC82121EAE17181709B78002BA7D080
:1085A800142018F08DF9D9F8D000A1E7D9F8D00037
:1085B800A74B41781144C829A8BFC82121EAE17115
:1085C80041709B78002B93D0132018F079F9D9F8D3
:1085D800D0008DE7D9F8D0009D4B01781144C82907
:1085E800A8BFC82121EAE17101709B78002B3FF4F4
:1085F8007FAF122018F064F9D9F8D00078E7944BCF
:108608000B989B78417911446429A8BF642121EA19
:10861800E1714171002B40F0F383D9F8D00067E78E
:10862800D9F8D0008A4B017A9B781144C829A8BF91
:10863800C82121EAE1710172002B3FF459AF0B20E8
:1086480018F03EF9D9F8D00052E7D9F8D000804B9D
:10865800C1799B781144C829A8BFC82121EAE171D2
:10866800C171002B3FF444AF0A2018F029F9D9F85A
:10867800D0003DE7D9F8D000754B81799B7811443B
:10868800C829A8BFC82121EAE1718171002B3FF4F4
:108698002FAF092018F014F9D9F8D00028E7D9F835
:1086A800D0006B4B417993F802E01144C829A8BF68
:1086B800C82121EAE1714171BEF1000F40F08E83BB
:1086C800112F7FF462AF13E7D9F8D000604B01791E
:1086D80093F802E01144C829A8BFC82121EAE17132
:1086E8000171BEF1000F40F09283102F7FF461AF4B
:1086F800FEE60B99564B0F790C931744642FA8BFCD
:10870800642727EAE7770F7118F0F4F80C9B9B7839
:10871800002B82D00320394618F0D2F8D9F8D000BF
:10872800E6E60B984A4B01781144FA29A8BFFA21CA
:1087380021EAE17101709B78002B3FF46EAF0120B4
:1087480018F0BEF8D9F8D000D2E60B98404B8178E3
:1087580011446429A8BF642121EAE17181709B78E2
:10876800002B3FF45AAF022018F0AAF8D9F8D0002D
:10877800BEE60B98364BC1799B78114481F308010A
:10878800C171002B3FF449AF052018F099F8D9F8CA
:10879800D000ADE60B982E4B817993F802E0114496
:1087A8006429A8BF642121EAE1718171BEF1000F3B
:1087B80040F01E830D2F7FF423AF2EE7D9F8D000A9
:1087C800234BC17893F802E01144C829A8BFC821F7
:1087D80021EAE171C170BEF1000F40F027830F2F2D
:1087E8007FF4FBAE84E60B98194B41781144B1F540
:1087F800967FA8BF4FF4967121EAE17141709B788A
:10880800002B3FF40AAF152018F05AF8D9F8D00019
:108818006EE61049D1F800E04200BEF1000F08D022
:10882800171803EB87079EF801E07F787745BEF4B9
:1088380002AA1044084F094A03EB800300200B608A
:1088480038801060FEF7F7B9129AFFF7B4BB00BF83
:108858006E600020F4250020DC260020E0260020A1
:1088680004999B7831F91220B2F5617F4FF4966133
:1088780091FBF3F3C0F2E48040F633019142A8BFC4
:1088880011460C2FA1F5617191FBF3F100F077818E
:10889800182F7FF4E2AAC9B2C8290B46A8BFC8237B
:1088A800D9F8D020D77DD8B2B8423FF4D6AADF1B7A
:1088B800C44BD07548BF0737FF109B780137FFB20C
:1088C8003BB9002F3FF4C9AA384628F069FCFFF7E6
:1088D800C4BA182017F0F4FFF3E7BB49096811F48C
:1088E800003140F04581B94B08465D5C0F2D01F120
:1088F8000C0170D001301828F7D10023FA3A84F817
:108908009230B34BA4F89020B24D0993FEF7D1B83A
:10891800B149D1F800E04200BEF1000F08D01718A5
:1089280003EB87079EF801E07F787745BEF408A936
:108938000244AA4FAA4803EB820300220B603A8044
:108948000260FEF7FDB8B4EEE77AF1EE10FA40F3F4
:10895800AC81DFEDA45A9FEDA46A01E0F0EE676AEE
:10896800F4EEC66AF1EE10FA76EEE57AF6DCDFEDA3
:108978009F6AF4EEE67AF1EE10FA40F19381DFEDAA
:10898800995A9FED9B6A01E0F0EE667AF4EEC67A9A
:10899800F1EE10FA77EEA56AF6D4DFED967AF4EEEA
:1089A800E76AF1EE10FA40F3C880DFED937A77EECC
:1089B800E66A66EEA65A9FED915A9FED916ADFED41
:1089C800917AA5EE856A26EEA55AE5EE867AE5EE59
:1089D800276AFFF763B980490F68450037B12E1839
:1089E80003EB86067F787678BE4286D205447B4EB6
:1089F8007B4803EB850300250B60358005607CE729
:108A0800814B002201200BE5804B1B78032B00F0E3
:108A18001F810022FFF7A4B97D4A6E4D13606C4B8D
:108A28000993FEF746B8DFED7B7AB4EEE77AF1EE0C
:108A380010FA44BFDFED6D7A37EEC77AFFF776B9E3
:108A48000C2F00F0BC80182F7FF407AA00210B46DA
:108A580026E7714A0592FEF70CBF06F48056FEF72A
:108A6800DABF6E4A069B1E68136823F0040313607E
:108A7800089A012306F4805682F82130FEF7CBBF0E
:108A880038EE678A664B67491870FDEEC87AC9F5F3
:108A9800FA63CDED047ABDF91020120381FB0201BF
:108AA800D217C2EBA1121BB203FB02F343F30F333D
:108AB8004B4407EE903AF8EEE77AC7ED037AFEF7F3
:108AC8000ABA0023BB2A149300F0BF80B72A00F02B
:108AD800EF80BE2A00F0E080BD2A7FF4D0AC4FF6CC
:108AE800FE71514A3A48D689099090893344014425
:108AF800D38191810EF090FAF8F778F80EF074FAB5
:108B0800FBF7AAF9012028F04BFBB4F890300022BB
:108B1800FA3BA4F8903084F89220FDF7CABF434A84
:108B28002C4D137843F004031370294B0993FDF778
:108B3800C0BF3F4B0222032072E4DFED367AF4EE29
:108B4800E76AF1EE10FA44BFDFED287A77EEE66ABD
:108B58002FE70EF061FAF8F749F80EF045FAFBF73F
:108B68007BF9012028F01CFB94F88E20FFF7ECB964
:108B780026490978032900F0A3801946B3E6CFB245
:108B88002C4B0D915B78BB423FF467A90D4B0C93BE
:108B980038461DF0AFFE0C9B0D999B781BB1C9B2EE
:108BA8000C2017F08DFE0137FFB28AE6174B1B78B1
:108BB800032B7EF4E8AD28F0F1F9FDF7C1BF0027DB
:108BC8003946DDE76E600020D04300204475030875
:108BD800E8640020E0640020F4250020DC26002062
:108BE800E0260020DB0FC940E4CB1641DB0F49C06B
:108BF800E4CB16C1DB0FC93FDB0F494092E741B90F
:108C08009730083C15A82ABE208D0020785B0020EC
:108C1800004D0020DB0FC9BF5C860020DC6400200B
:108C280074260020D34D6210C43E00206C600020E2
:108C3800BC8D0020948C0020814B824D4FF4C8726B
:108C48001A80814B0993FDF734BF1946022348E780
:108C580028F0A4F9FDF7EFBF08231A46FEF738BB42
:108C680007231A46FEF734BB06231A46FEF730BB25
:108C780005231A46FEF72CBB04231A46FEF728BB29
:108C880003231A46FEF724BB02231A46FEF720BB2D
:108C980001231A46FEF71CBB022122E7F0EE477AB1
:108CA800FFF722B8F0EE676A77E6F0EE667A5EE6DE
:108CB80019464FF6FE7314E7B0EE677AFFF72AB845
:108CC80028F06CF9B4F9902017E65F4B84F89410FB
:108CD80084F895005B4D0993FEF7A5BD002D3DF482
:108CE800F2AD5A4C94F88D30002B3DF41DAE28F0AF
:108CF80055F9002384F88D30FDF716BE4FF4FA615C
:108D080002201DF015FDFFF7DEBB002102201DF03B
:108D18000FFDB4F890304C4A0992963B0022A4F813
:108D2800903084F89220FDF7C4BE00210120EEE7C0
:108D380000210846EBE7FF2100201BF017FA94F802
:108D48008E20FFF7AEBB012100201BF00FFA94F82C
:108D58008E20FFF7A3BB0021FF201BF007FA94F831
:108D68008E20FFF798BB002101201BF0FFF994F833
:108D78008E20FFF78DBB364A334B0993137A43F0A5
:108D880001031372FDF795BE314A2F4B0993137AED
:108D980023F001031372FDF78CBE00210320B6E710
:108DA8002A4C1CF03BFC002384F88D30FDF7BCBD39
:108DB80000210420ABE7002B93D02649264A0968F6
:108DC8004FF47A7000FB031313608AE70B2028F036
:108DD80001F91D4B1B4D0993FDF76BBE11200D9337
:108DE8000C9217F06DFDD9F8D0000D9B0C9A67E432
:108DF8000D200D930C9217F063FD0D9B0C9AD9E48E
:108E08000E2017F05DFDD9F8D000FFF771BB1020D8
:108E18000D930C9217F054FDD9F8D0000D9B0C9AC5
:108E280063E4172017F04CFDFFF7F7BB0F200D93F5
:108E38000C9217F045FDD9F8D0000D9B0C9ACEE4A2
:108E4800FE8F0020E0640020E86400209C230020BE
:108E5800C4510020B0850020FC4C00202DE9F047CB
:108E6800C74C636820469847002800F0C380C54B6C
:108E78001B780122042B84F83C2000F0BD80B4F953
:108E88001610B4F91820B4F91A3021636263A36389
:108E9800BD4B1B88002B69D0BC4DD4ED0C7AD5EDA9
:108EA800004A95ED050A95ED015A95ED067AD5ED3E
:108EB800035A95ED026AF8EEE76AD5ED047AA4EE56
:108EC800A60AA5EE267A67EEC07AA5EEC07AE6EE87
:108ED800267A85ED057AC5ED067A2BF0F9FBD4EDF7
:108EE8000D6AD5ED094A95ED0E0A95ED0A5A95EDEC
:108EF8000F7AD5ED0D7AD5ED0C5A95ED0B6A2063F6
:108F0800F8EEE66AA4EEA60AA5EE267A67EEC07A1F
:108F1800A5EEC07AE6EE267A85ED0E7AC5ED0F7AD3
:108F28002BF0D6FBD4ED0E6AD5ED124A95ED170A53
:108F380095ED135A95ED187AD5ED167AD5ED155AA3
:108F480095ED146A6063F8EEE66AA6EEA40AA6EE4A
:108F5800857A67EEC07AA0EE657AE6EE867A85EDC8
:108F6800177AC5ED187A2BF0B3FBA063884FA17F61
:108F7800884810F071FF3B88002B40F08480864EB3
:108F8800D6F8E050854B1B685B0743D4B5F90070F1
:108F9800216B636BA06B824A824E92ED026AD2ED1E
:108FA800006AD2ED015AC91B2163B5F90270DB1BB7
:108FB8006363B5F904703568C01B07EE900AB8EE14
:108FC800E75A07EE901AB8EEE77A07EE903AF8EE0D
:108FD800E77A36EE056A36EE877A77EEA57A0135B6
:108FE800A06382ED026A82ED007AC2ED017A3560F3
:108FF800BDE8F087BDE8F0876B4BB4F91600B4F90B
:109008001810B4F91A2018802063598061639A8077
:10901800A2633DE7B6F89820322A00F08880002A3B
:1090280066D196F89530002BB0D06048D6F8FC2071
:109038005F4980FB0273D217C2EB23122A80D6F84D
:10904800002180FB0273D217C2EB23126A80D6F884
:109058000431A78A80FB0302DB17C3EB2213DB1B57
:10906800AB800023CB6086F895300DF0D5FFF7F77D
:10907800BDFD0DF0B9FFFAF7EFFE012028F090F8DA
:10908800D6F8E05082E7444E226BD6F8E050B3F5AC
:10909800C87F4FF0000323632B80398818BFD6F8A8
:1090A800E400B7F8008008BF0020B1F5C87F18BFFA
:1090B800D6F8E830616B02440B440020B8F5C87F4D
:1090C8006063C6F8E420C6F8E830688052D0D4F867
:1090D80038E0D6F8EC10A0637144B8F1010FA8800D
:1090E800C6F8EC1068D008F1FF38A7F8008049E707
:1090F800D6F8FC00236B00210344C6F8FC3021633A
:109108002980D6F80001636B61630344C6F8003117
:109118006980A36BD6F80401A1630344012AC6F849
:109128000431A98075D0013AA6F8982079E72B88F0
:1091380020491F48276BA6F8F0300023B5F802E055
:10914800B5F804C0C0684B608B602363C6F8FC7038
:109158002B80616BC6F8001163636B80A16BC6F846
:109168000411A363A6F8F2E0A6F8F4C0C6F8F80064
:10917800AB80D8E7A36BC6F8EC30A063A880B2E751
:1091880098640020DC4A0020A43C0020A83C002071
:10919800FE8F0020C86400209C230020105500206A
:1091A8008845002084450020E04A00201F85EB51B7
:1091B800C43E002098240020DFF804C1DFF8F0E066
:1091C800C8328CFB02A9C833D217C2EBE9128CFB58
:1091D80003A9DB17C3EBE913C8316B802A808CFB2A
:1091E800013CA28ACB17C3EBEC139B1AAB80CEF8D9
:1091F8000C000DF011FFF7F7F9FC0DF0F5FEFAF78A
:109208002BFE404627F0CCFFB7F80080D6F8E05098
:1092180069E7254B86F89A101B6886F8942013F4A2
:10922800003334D119462148475C0B2F01F10C015A
:1092380010D00133182BF7D1B6F8F0101C4B298049
:10924800B6F8F270B6F8F400D6F8F8106F80A88077
:10925800D96068E7174FD7F800C05900BCF1000F74
:1092680009D001EB030E00EB8E0E9CF801C09EF8AE
:1092780001E0E645E0D20B44DFF848E00E4900EB98
:10928800830000233860AEF800300B60D4E70B4B46
:109298001B78032B01D00B46C5E727F07FFED6F8D5
:1092A800E050B6F89820C7E7D0430020447503087B
:1092B800C43E0020F4250020E0260020785B002032
:1092C8001F85EB51DC2600202DE9F0478C4B1B78DD
:1092D800DB07074644D58B4B8B4D1C788B4E012CF6
:1092E80059D01CD3022C07D189498A4A0988128887
:1092F800914201D901241C70EB7AE3B12B89D3B1D7
:10930800854B1B78BBB108F0F9FB002800F09B8067
:109318002B7B83422CBF0121002131700CE07C495A
:109328007E4A098810886A7B801A8842E2DAEB7ADA
:109338000024002BE2D131782A79632A06D8022C3E
:10934800774E00F0BA803378002B5DD1754AAB7A3E
:109358008C4238BF0C461470002B4CD1BDE8F08706
:109368006B4B694D19885B88E878CB1A83EAE372FE
:109378008142A2EBE3721DD32B788B421AD3614B47
:109388001C78E01E012861D96749097802294FD065
:10939800012C5E4EA5D15F4A5D491288687B098819
:1093A800121A914239DD5D4A12888A42A4D20024F9
:1093B8001C70A1E7B1EB400FE1DC524B1C78E11EB9
:1093C800012940F29480022ADEDC57494F4E087882
:1093D800DFF84481DFF844C1DFF838E100210324D5
:1093E800022834701C7088F80010ACF80010AEF831
:1093F800001081D11FE0012C71D0022C0BD1072065
:10940800BDE8F04727F0E6BD7068381A474B984228
:1094180058DD72709AE7BDE8F08702241C706BE78C
:10942800022AD2DD4049097802294FF0040464D1A8
:109438003949364E09783E48022ACCBF002201221B
:10944800C28081804BE70221317075E7022A9BDCDC
:1094580095F800C091FBFCFC0CF1010CBCF1080F65
:10946800DFF8B4A0304EA87895F801E096F80080AF
:109478002A4CDFF8A090254EA8BF4FF0080C8AF8B8
:1094880000C01FFA8CFA10FB0AF01EFB0AFE80B21D
:10949800DFF88CA02080A9F800E000244FF0640ECB
:1094A800B8F1020F34701C70CAF804408AF801E061
:1094B8007FF439AF0FFA8CF1BDE73078A0B90123FA
:1094C80077603370C2F164021A4B00FB02F083FB31
:1094D8000023C017A0EBA3506430707036E7082053
:1094E800BDE8F04727F076BD7368F81A8EE7032CBD
:1094F80096D10D49097802299AD0044EFCE600BF9E
:10950800484B0020982700207C640020A8270020D2
:10951800E84B00209C270020FE4B00209A270020C3
:10952800A0270020785B0020DC4A00207F96980066
:10953800E04A00206BCA5F6B2DE9F04FB0F9085084
:109548000D81EDB2442D93B00C46174600F06D82A4
:10955800064642D9812D00F0AB8200F29580542D49
:1095680000F0C98040F2FC816E2D00F02C82802D25
:1095780040F01D81994B93F8009009F1020919F008
:10958800FF0900F09580964B964F974EDFF88CA216
:10959800994403F101080A2516E0322D01F03884B8
:1095A800A5F13C00C0B2132841F23C840023226894
:1095B800511C216015702268C14502F1010121602A
:1095C800137075D018F8015B0A2DE6D1BAF800308F
:1095D800FF2BA8BFFF23DBB2E9E7052D00F01382BC
:1095E8001ED8022D7FD040F2A881032D00F0E08123
:1095F800042D40F0DC802A467C492046F7F7C0FD60
:1096080000212046F7F7EAFD22680221531C0125B4
:10961800236028462B461170638113B0BDE8F08F94
:10962800242D5ED040F24081282D00F00682382D8E
:1096380040F0BD800A686E4B0125511C21601570F1
:109648002268052150192060117022680A215019DA
:109658002060117022680021501920601170226862
:1096680019785019206011702268597850192060B3
:10967800117022689978531923602B461170284677
:10968800638113B0BDE8F08FA02D18D040F22A8175
:10969800B82D00F00B82FE2D40F08980554D05F164
:1096A800080635F8021B2046F7F798FDAE42F8D1B8
:1096B80001252B462846638113B0BDE8F08F4E4B39
:1096C80008461968F7F773FD4C4B20461968F7F7F9
:1096D8006EFD4B4B196820460125F7F768FD2B46B0
:1096E800E8E7484BF6E70422474920460125F7F703
:1096F80047FD2B46C3E70B68444A454F581C1121C8
:109708002060197023681278591C21601A70236828
:1097180097F85520591C21601A70236897F854202F
:10972800591C21601A70B7F850102046F7F756FDFB
:1097380023680022591C21601A7023682822591CAA
:1097480021601A70B7F852102046F7F747FDBD1E82
:1097580007F14E0635F8021F2046F7F73FFDB542E0
:10976800F8D122682B4B0D21501C20605D18117018
:10977800226813F8011F501C9D4220601170F7D118
:1097880023680222591C21601A70B7F85610204627
:10979800F7F724FDB7F858102046F7F71FFD012505
:1097A800B7F85A102046F7F719FD2B4667E7214608
:1097B800284606F0C3FD014600287FF479AF742DD2
:1097C80000F0EC80772D2BD1336872689A4240F014
:1097D800DA81114A204627F091FD69E7BD4A002049
:1097E8001859030867666666482700209A8C002087
:1097F8000B8D0020E04A0020ACF7FF1FB0F7FF1FD9
:10980800B4F7FF1F508E0020D48503080C8A00206F
:109818000C5B0020695B00205909030870270020B1
:10982800F52D00F0DD8170683768A5F12103C21BB2
:10983800362B00F26583DFE813F03D026303630310
:10984800630363036303630363035C0263036303E8
:1098580063036303630363036303630363036303D0
:10986800630363036303630363032D0263036303F7
:1098780063036303630363036303630363036303B0
:1098880063036303630363036303630363036303A0
:1098980063036303630363036303630363030E03E5
:1098A8006303E80263037102202D80D10B68B84D71
:1098B800591C6A7821601A7023682A78591C21601B
:1098C8001A702368AA78591C21601A7029892046C1
:1098D800F7F784FC23686A79591C21601A7022689A
:1098E800A97993E6822D7FF462AF0B68A94AAA4D45
:1098F8001178A74A581C2060197011892046F7F77B
:109908006DFCA64B22681B88FF2B02F10101A8BF42
:10991800FF2321601370A96881F3100189B22046E2
:10992800F7F75CFC296801F30F0189B22046F7F7C5
:1099380055FC9B4B2268197868E6012D7FF437AFF8
:109948000B680022591C21601A7023685A1C226077
:109958001D7022682521531C23602B4611708EE64A
:10996800522D7FF424AF0A688E4E531C03212360C6
:1099780006F10C0733461170062501202268511C98
:10998800216010702268BB4202F10101216015704C
:1099980000F0D6809879DD790633EFE7336872688E
:1099A8009A4240F0EC80804A204627F0A7FC7FE6E8
:1099B8000B685A1C0A601D700B685A1C0A601D70DF
:1099C8000A68002122E6754B0A681B88724DFF2B36
:1099D800A8BFFF23511C21601370A96881F31001EF
:1099E80089B22046F7F7FAFB704B20461988F7F73B
:1099F800F5FB296801F30F0189B220460125F7F725
:109A0800EDFB2B463BE60B2269492046F7F7B8FBEE
:109A1800082268492046F7F7B3FB01250722664963
:109A28002046F7F7ADFB2B4629E6002A3FF440AE67
:109A3800624B136001252B4621E60B68DFF89C81F9
:109A48005F4E591C022221601A70236806275A1C8F
:109A580022601F7023680A22591C21601A7023682B
:109A680001255A1922601D70B8F800102046F7F732
:109A7800B5FBB8F802102046F7F7B0FB23685A196F
:109A880022601F7023685022591921601A702368B8
:109A98000022591921601A7031882046F7F79EFB79
:109AA80071882046F7F79AFB2B46E8E5454B11E607
:109AB800454B1E78033616F0FF063FF4F9AD434BCD
:109AC800434F1E4403F101094FF00A0820E0B8F1A2
:109AD800500F01F0A481B8F1320F01F0B981A8F15B
:109AE8003C00C0B2132841F2B781002529462368FB
:109AF8005A1C2260204683F80080F7F76FFB29463E
:109B08002046F7F76BFB4E453FF4D2AD19F8018BB1
:109B1800B8F10A0FDBD12F4B9D68196805EB850555
:109B28004FF6FF736D009D42A8BF1D469942A8BF1E
:109B3800194625EAE57521EAE171ADB289B2D6E7A1
:109B4800254B21681A78481C20600A70002A3FF4C7
:109B5800AFAD013AD2B202EB420206EB42025278B2
:109B6800002A3FF4A5AD0132D5180133226813F855
:109B7800011F501CAB4220601170F7D198E55A1CA8
:109B8800326019780FE75A1C3260197821E600BF55
:109B98007C640020FE4B0020BC620020E84B0020C3
:109BA800785B002090590308D90903084460002015
:109BB800DC850308E8850308F48503087D000108AF
:109BC80030270020D0430020BD4A00202859030830
:109BD80040270020FC26002000870020B43E0020FB
:109BE800336872689A4241F05081B64BFF221A706E
:109BF8004FF00009B44D1BF0D5FC49462022B3486C
:109C080085F800902BF021FD8DF808909DF808301C
:109C1800072B01F2E981DFF8DC82AC4E4A469DF859
:109C2800083003EB430308EBC3035B7CE3B19DF807
:109C3800083003EB430308EBC30320215B699BB1A6
:109C48009DF8083003EB430308EBC303586946F853
:109C58002200FCF729F92B7856F82300F6F7B6FD11
:109C68002A780132D2B22A709DF808300133DBB26B
:109C78008DF808309DF80830072BD0D92368591C77
:109C880021601A70002F3FF413AD914B3B60012502
:109C98002B46F4E47B1C33603B780A2B01F02381CC
:109CA8003046F7F768FA3046F7F765FA3046F7F7BF
:109CB80062FAFDE43B467A1C3260864D13F8022BAB
:109CC8006A7033607B782B70FB1C3360BB78AB7099
:109CD8003046F7F745FA33682881591C1A4631602F
:109CE80012F8021B697132605B78AB7101252B4653
:109CF800C5E47B1C33603B780A2B01F0EE80502BC7
:109D080040F08F853046F7F72BFA734F388030468E
:109D1800F7F726FA012578802B46B0E47B1C3846F5
:109D2800336010F8375B0DF107020133336013F825
:109D3800011C02F8011F9842F7D1DFF8BCA19AF87C
:109D48000070002FFDD1DFF8B4B16448634E4FF0C6
:109D5800010804218AF80080F8F766F9DBF80000AA
:109D6800F6F72FFD5E4B3946304683F80080F7F74B
:109D7800D3FD39463046F7F7CFFD09213046F7F7CE
:109D8800CBFD29463046F7F7C7FD0DF108084546D3
:109D98000DF13E09A5EB0807FFB20A213046F7F797
:109DA800BBFD39463046F7F7B7FD15F8017B0B21A7
:109DB8003046F7F7B1FD39463046F7F7ADFD0020DC
:109DC800FBF70EFEA945E5D1444808210546F7F7FB
:109DD800A3FDA0212846F7F79FFDA0212846F7F705
:109DE8009BFD00212846F7F797FD10F02006F4D1D7
:109DF800DBF80000F6F7EAFC012502213748F8F7FE
:109E080013F98AF800602B4639E47B1C336097F815
:109E18000080B8F1FF0F01F0AF80B8F1FE0F01F03C
:109E280073803046F7F79CF996E80C009B1A002BD4
:109E380007DD531C336013781BB9B8F10C0F41F2DE
:109E4800C880B8F1270F00F2DC82264B012523F8E1
:109E580018002B4613E47B1C33603878032800F283
:109E6800D082431E204D2149DBB203EB430305EBAF
:109E7800430308705D7800283FF41AAC531EDBB228
:109E8800AB4240F0BE820022C1F80620C1F8022091
:109E98008A725BB1581C336808444A1C013333602A
:109EA80013F8011C02F8011F9042F7D1104B1B78E0
:109EB800002B3FF4FDAB012525F0E6F92B46FFF713
:109EC800DEBB00BFA824002005450020F434002094
:109ED800B5DD01087C6400203027002000380040F0
:109EE800344D00200C5B00209059030800870020A7
:109EF800A927002050560020A4410020048A0020F1
:109F08000B3DEF2D00F27D8201A353F825F000BF31
:109F18000BAB00080BA400080BA400080BA4000856
:109F28000BA400080BA400080BA400080BA400084D
:109F38000BA400080BA400080BA400080BA400083D
:109F48000BA400080BA400080BA400080BA400082D
:109F58000BA400080BA400080BA400080BA400081D
:109F68000BA400080BA400080BA400080BA400080D
:109F78009BAA00080BA4000881AA00080BA40008EB
:109F88005FAA00080BA400080BA400080BA4000893
:109F980037AA00080BA40008DDA900080BA40008D4
:109FA80059A900080BA4000833A900080BA400084D
:109FB80007A900080BA40008B3A800080BA4000810
:109FC80067A800080BA400080BA400080BA400084D
:109FD8000BA40008B99600080BA400083BA80008C9
:109FE8000BA400080BA4000819A900080BA400087A
:109FF800E1A700080BA400080BA400080BA40008A4
:10A008000BA400080BA400080BA400080BA400086C
:10A018000BA40008A1A700080BA4000853A7000878
:10A028000BA400080BA40008ADAD00080BA40008A1
:10A038000BA400080BA400080BA400080BA400083C
:10A048000BA400080BA40008D5AC00080BA400085A
:10A0580039AD00080BA4000833AC00080BA40008B5
:10A06800A3AB00080BA400087BAB00085DAB00089D
:10A0780041AB00080BA400080BA400080BA40008BF
:10A088000BA400080BA400080BA400080BA40008EC
:10A098000BA400080BA400080BA400080BA40008DC
:10A0A8000BA400080BA400080BA400080BA40008CC
:10A0B8000BA400080BA400080BA400080BA40008BC
:10A0C8000BA400080BA400080BA400080BA40008AC
:10A0D8000BA400080BA400080BA400080BA400089C
:10A0E8000BA400080BA400080BA400080BA400088C
:10A0F8000BA400080BA400080BA400080BA400087C
:10A108000BA400080BA400080BA400080BA400086B
:10A118000BA400080BA400080BA400080BA400085B
:10A128000BA400080BA400080BA400080BA400084B
:10A138000BA400080BA400080BA400080BA400083B
:10A148000BA400080BA400080BA400080BA400082B
:10A158000BA400080BA400080BA400080BA400081B
:10A168000BA400080BA400080BA400080BA400080B
:10A178000BA400080BA400080BA400080BA40008FB
:10A188000BA400080BA400080BA400080BA40008EB
:10A198000BA400080BA400080BA400080BA40008DB
:10A1A8000BA400080BA400080BA400080BA40008CB
:10A1B8000BA400080BA400080BA400080BA40008BB
:10A1C800EFAD00080BA400083DA7000813A700087E
:10A1D8000BA400080BA400080BA400080BA400089B
:10A1E8000BA400080BA400080BA400080BA400088B
:10A1F8000BA400080BA400080BA400080BA400087B
:10A208000BA40008B9A600080BA4000881A6000842
:10A218000BA40008E5A5000887A500086BA50008A1
:10A228000BA4000851A500080BA4000829A50008E4
:10A238000BA40008CFA400080BA40008A1A40008E0
:10A248000BA400080BA400087FA4000851A4000870
:10A258003DA4000815A40008EDA30008CBA300083E
:10A268000BA400080BA400080BA400080BA400080A
:10A278000BA400080BA400080BA400080BA40008FA
:10A288000BA400080BA400080BA400080BA40008EA
:10A298000BA400080BA400080BA400080BA40008DA
:10A2A800B1A300080BA400080BA4000859A30008D8
:10A2B8000BA400080BA400080BA40008F3A20008D4
:10A2C8000BA400080BA400080BA40008D9A20008DE
:10A2D800B14B1B78DB0700F194800125F9F7E0FB0F
:10A2E800F9F7BAFD2B46FFF7CAB93046F6F738FF3B
:10A2F8003368ADF808001A46591C316012F8021B81
:10A3080032608DF80A105A788DF80B20DA1C32600A
:10A318009A788DF80C201A1D3260DA788DF80D20A5
:10A328005A1D32601B798DF80E3002A80023ADF853
:10A338001030F6F771FE994A994B1268801A4FF05F
:10A34800010561F10001C3E904012B46FFF797B944
:10A358007B1C33603B780F2B53D8BA1C3260C3EB9D
:10A36800C303904A7978D154F91C31601344BA7800
:10A378005A703A1D3260FA789A707A1D32603A79CA
:10A38800DA70BA1D32607A791A71FA1D3260BA79B8
:10A398005A7107F108023260FA799A71012514F0AE
:10A3A800EDFE2B46FFF76BB93046F6F7D9FE7E4F28
:10A3B800F8813046F6F7D4FE0125B8812B46FFF721
:10A3C8005EB93046F6F7CCFE784F38823046F6F75D
:10A3D800C7FE78823046F6F7C3FE0125B8822B46C1
:10A3E800FFF74DB93B467A1C326013F8020B336015
:10A3F800FB1C79783360BA781FF0C8FA00287FF41C
:10A4080057A94FF0FF352B46FFF739B93B467A1C61
:10A418003260674A13F8021B11703360624A7B7816
:10A428009370FB1C3360634BBA789A7001252B46F6
:10A43800FFF725B9604B614918684E22012529F0BC
:10A4480073FF2B46FFF71BB93A467B1C33605C4B06
:10A4580012F8021B197032607A785A70FA1C32604E
:10A46800BA789A703046F6F77BFE564B0125D880AD
:10A478002B46FFF704B93046F6F772FE514F388085
:10A488003046F6F76DFE78803046F6F769FE01250E
:10A49800B8802B46FFF7F3B8DFF8388198F800301A
:10A4A800002B3FF405A9484F00253046F6F758FE23
:10A4B80015F0B8FB98F80030A7EC010A01359D4269
:10A4C800F3DBFFF7F5B80D2A9BD17B1C33603D7891
:10A4D800072D96D8DFF8008130460C27F6F740FEA6
:10A4E80007FB05F708EB0705A8803046F6F738FEA6
:10A4F800E8803046F6F734FE336828811A46591C3E
:10A50800316012F8021BA97232605B78EB72304638
:10A51800F6F70FFE012548F807002B46FFF7AFB8FE
:10A528007B1C33603878060600F1A4851A4B1B782B
:10A53800DD073FF5BDA8032828BF00200125F9F74E
:10A5480093FA2B46FFF79BB8134B1B78D8073FF5B8
:10A55800AFA80125F9F74CFEF9F77EFC2B46FFF76B
:10A568008EB80D4B1B78DA073FF5A2A8174A137867
:10A57800012543F0040313702B46FFF780B8064B00
:10A588001B78D9073FF594A8114B4FF4C8720125E1
:10A598001A802B46FFF773B8484B0020B08500207F
:10A5A800A8240020E4420020C43E002010570020C8
:10A5B80074520020D43E0020E46400201077030881
:10A5C800BC3E00207C470020383000206C60002012
:10A5D800FE8F0020BD4A002024420020092A7FF770
:10A5E80010AFDFF8E8833B467A1CD8F80050326099
:10A5F80013F8022B2A7033607B78AB70FB1C336036
:10A60800BB78642BA8BF64233A1D6B713260FB785A
:10A61800642BA8BF64237A1DAB7132603B79EB7160
:10A62800BB1D33607B79642BA8BF6423FA1D2B7292
:10A638003260BB79EB7007F108033360FB792B714B
:10A648003046F6F78DFD726833686881D11A0029A3
:10A658000CDD591CD8F800003160521A002A19780C
:10A66800417203DD9A1C32605B784370012516F055
:10A6780041F92B46FFF703B8C24B1868FB1C02468A
:10A688002137991E316013F8031C1170591E31606F
:10A6980013F8021C5170336013F8011C91700333D6
:10A6A8009F4202F10302ECD115F08CF9FFF700B8D4
:10A6B800C2F34705122D3FF6A4AEB5B112AB0DF1AA
:10A6C800060803EB4507C146423F3046F6F748FD0A
:10A6D80029F8020F4F45F8D1AB4B38F8022F23F871
:10A6E800022FC845F9D1112D09D8A84A6B00023BA1
:10A6F80013440021223223F8021F9A42FBD1A44AB4
:10A7080001231D461370FEF7BABF7B1CA1493360B5
:10A718000A783B78002A40F0898404220A709E4A0D
:10A728009B001380FAF74EFE9C4B012598612B463F
:10A73800FEF7A5BF9A4F002330463B60F6F7F9FCB9
:10A74800012538602B46FEF79ABF7B1C336097F8CB
:10A758000080B8F1110F3FF654AEBB1C3360914D29
:10A768007B7805F818303046F6F7FAFC40F6CA034D
:10A778009842A8BF184640F2EE23984205EB4801DC
:10A78800B8BF18460125A0F2EE222B46192092FBED
:10A79800F0F24A70FEF773BF3B467A1C824D326076
:10A7A80013F8022B2A7133607B786B713046F6F709
:10A7B800D7FC336828805A1C32601B78AB7130464E
:10A7C800F6F7CEFC336868805A1C32601B78EB7150
:10A7D80001252B46FEF753BF7B1C3360734B3A7839
:10A7E800DFF8EC811A700023C8F800303046F6F71D
:10A7F800A0FC3268D8F800306D496E4D0343501CF8
:10A80800C8F80030306013780B723046F6F7A8FCB1
:10A8180028603046F6F7A4FC68603046F6F7A0FCDE
:10A82800A8603046F6F79CFC3046F6F799FCFEF730
:10A838003FBF3B467A1C32605F4A13F8021B917097
:10A8480033607978517083423EF432AFFB1C336039
:10A85800524BBA781A7201252B46FEF710BF072310
:10A86800B2FBF3F3C3EBC301521A7FF4CAADDBB2F8
:10A8780003F1FF395FFA89F9002B3EF419AFDFF8CD
:10A888003CA109F1010915467B1C33604B4B97F934
:10A898000020002793F90210914203F1080300F009
:10A8A80046830137042FF5D1ABE57B1C33603B7839
:10A8B8000E2B3FF6A6ADBA1C3260787803283FF617
:10A8C800A0AD3F49062202FB03F28B18FD1C58710C
:10A8D8003560B87888543A1D3260FA785A707A1D13
:10A8E80032603A799A70BA1D32607A79DA70FA1D54
:10A8F8003260BA791A7101252B46FEF7C0BE7B1C5F
:10A9080033602B4B3A785A7501252B46FEF7B7BEB4
:10A918002C4B07F108020137376017F8011C03F8C0
:10A92800011FBA42F7D1FEF7C3BE7B1C33603D78E6
:10A938001F2D3FF666AD052A7FF463AD3046F6F766
:10A94800F8FB214B43F8250012F024F9FEF7B0BEBE
:10A958001D4D05F140073046F6F702FC3368A5F8AF
:10A968008000591C1A46316012F8021B85F88210C3
:10A9780032605B7885F883300435AF42EBD1FEF75F
:10A9880097BE00BFE4640020D6330020D8330020EF
:10A99800FC3300208238002044600020A8240020D6
:10A9A800D04300209C360020944700205C390020CA
:10A9B8005C860020A82F0020E43E00208886002026
:10A9C800DC4300205B860020985B0020E8640020C0
:10A9D800508E00207B1CAF4D33603B782B72304685
:10A9E800F6F7BEFBA8833046F6F7BAFB2883304655
:10A9F800F6F7B6FB32686883531C33601278EA7442
:10AA08007268D31A032B00F370833368D11A0529AF
:10AA180000F35B83D21A002A7EF74AAE5A1C3260D2
:10AA28001B7885F8213001252B46FEF728BE7B1CB4
:10AA38003360994A39781170C01A00287EF738AE09
:10AA4800BB1C33607B78003318BF0123012553708A
:10AA58002B46FEF714BE3046F6F782FB8F4F386060
:10AA68003046F6F77DFB78603046F6F779FB01252E
:10AA7800B8602B46FEF703BE894F00233B60304683
:10AA8800F6F757FB3B68012503433B602B46FEF76F
:10AA9800F6BD7B1C33603D780191132D3FF6B1ACB8
:10AAA800BB1C3360787826F063FC00283FF4A9AC1F
:10AAB8007C4B027803F82520FA1C326003EB8505ED
:10AAC800BA786A703A1D3260FA78AA707A1D3260D4
:10AAD8003A79EA70019903F1500202E00433934293
:10AAE80007D018780028F9D19D78D8788542F5D212
:10AAF80001216D4B81F00101012519702B46FEF7EC
:10AB0800BEBD6A4B102A4FF0000128BF1022196001
:10AB180059609960D9601974002A3EF4C9AD31684A
:10AB2800013B0A440131316011F8010C03F8010FAF
:10AB38008A42F7D1FEF7BCBD7B1C33603B78002B03
:10AB480000F0BA824FF40040012506F025FC2B46A0
:10AB5800FEF795BD564B1B7813F001017FF451ACFD
:10AB68007B1C3360387801251BF0E2FD2B46FEF78D
:10AB780086BD3B467A1C32604E4A13F8021BD170E0
:10AB880033604D4A7B785371FB1C33604B4BBA786A
:10AB9800DA7001252B46FEF772BD3046F6F7E0FA6B
:10ABA8003046F6F7DDFA3046F6F7DAFA3046F6F7C9
:10ABB800E2FA3368424D1946581C2A68306011F889
:10ABC800020B82F82C003160597882F83610D91CB3
:10ABD80031609B7882F837303046F6F7CCFA304649
:10ABE800F6F7C9FA3046F6F7C6FA30462F68F6F790
:10ABF800B7FA788730462F68F6F7B2FA3368726882
:10AC08003887D11A01290ADD591C2A6831601B7856
:10AC180082F82E303046F6F7AEFA33687268D31AE7
:10AC2800032B00F3818228683EE57B1C3360244DAA
:10AC3800DFF894803B7888F8053030462F68F6F7BF
:10AC48008FFA388430462F68F6F78AFA72683368C4
:10AC5800F883D11A072900F31882D11A032900F3BF
:10AC6800EA81D21A002A05DD591C2A6831601B784E
:10AC780082F82630F9F752F81DF078F8114B1B6866
:10AC8800002B00F069822868012514F00BFB2B4685
:10AC9800FEF7F5BC5C8600205C390020A82F002058
:10ACA800508E002090350020E420002046600020CF
:10ACB800484B0020C43E00202C660020D43E0020D3
:10ACC800E46400204439002074520020C84B1B68FB
:10ACD800002B3EF4EDAC1CF0C7FDFF283EF4E8ACB9
:10ACE8003046F6F73DFA3F2840F22982C14F002549
:10ACF8003D7033687268B880D21A012A7EF7D8ACE2
:10AD08001A46591C316012F8021BB97012A8326039
:10AD180000225D7800F8402D1CF078FD9DF8083081
:10AD2800AB423EF4C5AC28461CF094FDFEF7C0BC0F
:10AD38003B467A1C3260DFF8EC8213F8022B88F865
:10AD480002203360AC4A7B781370FB1C3360AB4D38
:10AD5800BB782B713B1D3360FB78092BA8BF0923F7
:10AD68003046AB70F6F7FCF9336872682880D11A60
:10AD7800012905DD3046F6F7F3F933687268E88192
:10AD88009A4240F0F481F8F7C9FF336872689A4232
:10AD98003EF48EAC5A1C32601B78EB7001252B46B2
:10ADA800FEF76DBC964B1B78012B3EF681AC7B1CE5
:10ADB8003A463360DFF8708212F8023B88F80230B6
:10ADC8003260FB1C97F801E03360C31A012BB97895
:10ADD80040F33E813046F6F7C3F90125A8F8000094
:10ADE8002B46FEF74CBC3B467A1C326013F8025BDC
:10ADF8003360FB1C78783360B978002D00F034811B
:10AE0800012D7EF455AC1BF059FD2B46FEF737BCDF
:10AE18003388FF2BA8BFFF23DBB2FEF7C8BB794BF3
:10AE2800FEF77ABE19F0DCFE00283EF4BFAB0378CB
:10AE38000A2B28D8B0F9023087FB0312DB17C3EBC3
:10AE4800A2039BB2FF2BA8BFFF23DBB2FEF7AFBB69
:10AE580097E82200FEF762BE19F0C2FE00283EF411
:10AE680044AE03780A2B3EF640AEB0F90430B0F990
:10AE7800061003EB830383F3500521EAE171ADB2B9
:10AE880089B2FEF734BE0023DFE75A1C1946326048
:10AE98005D4811F8022B027031605B784370042A18
:10AEA80006D9FF2A3EF4A4AE22680021FEF7AEBB05
:10AEB80056490978994203D8022AF5D1FF2BF3D1D4
:10AEC800236801255A1922601D70002F3EF4F0AB4B
:10AED8004F4B3B602B46FEF7D2BB3046F6F740F9A6
:10AEE8004C4FFEF713BFBB1C33604B4B7A781A707C
:10AEF800FA1C3260BA785A703A1D3260FA789A7041
:10AF080001252B46FEF7BBBBBB1C33607D78022DA9
:10AF18003FF677AA3046F6F723F9404B03EB450393
:10AF28004FF0FF35A3F856002B46FEF7A8BB0AEBF7
:10AF3800C708304688F80220F6F712F933682AF86D
:10AF480037001A46591C316012F8021B88F80310A2
:10AF580032605A7888F80420DA1C32609A7888F8C7
:10AF680006201F1D37600135DB7888F80530A945B4
:10AF78007FF48AACFEF79CBBBB1C3360284B7A7805
:10AF88001A70FB1C3360DFF89480BB7888F8553062
:10AF98003B1D3360FB7888F854303046F6F7E0F80C
:10AFA800A8F850003046F6F7DBF83046F6F7D8F840
:10AFB80096E80C009B1A012BA8F852007EF778AB94
:10AFC8003046F6F7CDF80125A8F85A002B46FEF7CB
:10AFD80056BB124B0030984418BF0120012588F851
:10AFE8005E002B46FEF74BBB4A46FEF747BE00BF46
:10AFF8004C4B0020504B0020B83E0020105700203A
:10B008003E8E002034270020A8240020BD4A0020BE
:10B0180095000108B43E00200B8D00200C5B002039
:10B028000C8A0020745200206E600020042A7EF4EE
:10B038003FABFFF774BB3046F6F792F8A8F80E005E
:10B048003046F6F78DF833687268A8F8100008E6FD
:10B058004B4B1A88012512FB0EF22B4692FBF1F29C
:10B06800A8F80020FEF70BBB012514F039FB2B468E
:10B07800FEF705BB00F07F00032828BF002001254C
:10B088001BF038FC2B46FEF7FABA3046F6F768F89C
:10B09800A8F80A003046F6F763F8A8F80C0030461E
:10B0A8002F68F6F75DF8788430462F68F6F758F879
:10B0B80033687268B884D0E5324A1368012523F4EE
:10B0C800004313602B46FEF7DABA5A1C32601B782D
:10B0D800EB723046F6F72DF83368E8605A1C326098
:10B0E8001B782B743368726894E43046F6F738F8A6
:10B0F800A8843046F6F734F833687268E884D11AC1
:10B1080003297FF783AC1A46591C316012F8021BD9
:10B11800A97732605B7885F820303046F6F720F85A
:10B1280033687268688471E430462F68F6F718F857
:10B13800788630462E68F6F713F8B08673E5C508AA
:10B1480000F0070301350133EDB20F4F28461946C9
:10B158007B7019F0A7FCCBE50C480D490D4A0E4B46
:10B16800036001250B6013602B46FEF788BA5A1C52
:10B1780032601B78003318BF012388F8073002E6D5
:10B18800223D0020DC640020504B0020B845002000
:10B198000C46002074460020A30500082DE9F04F56
:10B1A8002DED0E8BDFF8F4B093B0DBF8042004909B
:10B1B80058469047002800F08E82BBF8A8700021FE
:10B1C8008BF85110002F6DD1BBF93A00DBF82450F1
:10B1D800DBF82810BBF93860DBF82040BBF93C20CD
:10B1E800DFF8BCA0401B521ACBF830009BF8521075
:10B1F800CBF83420341B0BF12C00CBF82C400EF08C
:10B208002BFEDAF80020910041F1B787DBED0C5AEC
:10B218001F4CDBED0B7A1F4994ED406AD4ED416A6F
:10B2280094ED427AD4F80C2109681B4B0293B8EECE
:10B23800E58ADBED0D5AF8EEE77AF8EEE58A013299
:10B2480077EE867A38EE268A78EE878A8A42C4EDC7
:10B25800407A84ED418AC4ED428AC4F80C2101F099
:10B26800508393F800E0BEF1140F02F09287002398
:10B27800D4F814510393062D01F29D84DFE815F0EC
:10B28800FA15BC161D15CF16080C39177F1500BF07
:10B29800D02400206C390020DC4A0020885200208D
:10B2A80010550020DE4BDF481A6805934FF47A7575
:10B2B800B5FBF2F2C2EB421502EB8502D500DA4B80
:10B2C800DFF8C88344780293ADB2AF421E78B8F96C
:10B2D800060003F07880DBF87C30BBF93810DBF827
:10B2E800602003F1010E07EE901A0A44BEF1010F27
:10B2F800CBF87CE0CBF86020F8EEE77A03F07080BA
:10B30800DBED1B5ADBED1D6A07EE10EA37EEE56A46
:10B31800B8EEC75A012F86EE057A37EE257A77EE12
:10B32800C77A8BED1C7AE7EE866A8BED1B7AF0EE16
:10B33800667ACBED1E6ACBED1D6A03F00D84DBF84F
:10B348009030BBF93A10DBF8642003F1010E07EEE8
:10B35800901A0A44BEF1010FCBF890E0CBF86420B4
:10B36800F8EEE77A03F05780DBED205ADBED226A2E
:10B3780007EE10EA37EEE56AB8EEC75A012F86EEF7
:10B38800057A37EE257A77EEC77A8BED217AE7EEE4
:10B39800866A8BED207AF0EE667ACBED236ACBEDE8
:10B3A800226A03F0B183DBF8A430BBF93C10DBF868
:10B3B800682003F1010E07EE901A0A44BEF1010F4E
:10B3C800CBF8A4E0CBF86820F8EEE77A03F03E80EB
:10B3D800DBED255ADBED276A07EE10EA37EEE56A62
:10B3E800B8EEC75A012F86EE057A37EE257A77EE42
:10B3F800C77A8BED267AE6EE276A8BED257AF0EE92
:10B40800667ACBED286ACBED276A03F07083874C08
:10B41800A8F80600BBF8A820029B013A1E78ABF8F2
:10B42800A82005990022072E4A608A60CA6040F069
:10B438005981F9F7C7FF029BDFF850821E78049BF9
:10B44800C01A94F82831A8F800000693002B40F0A1
:10B458004F81744A5279002A01F08081744A127827
:10B46800013AD2B2072E84F8282102F0EE81002397
:10B478000793704BD4F83421D3F800A0684B059398
:10B48800049B9FED6D6AD4ED4C9A6C49C4F8343135
:10B498009A1A07EE902AF8EE677AB7EE007AC6EEA7
:10B4A800278A0025664BDFF8E891DFF8E881654FC9
:10B4B80003932E46D1ED006A94ED4BDA9FED629A24
:10B4C800DFED62AA9FED62CA9FED62AADFED62BA64
:10B4D8009FED62BA77EE69CA6CEEA6CAF4EEC7CAE7
:10B4E800F1EE10FA88BFF0EE47CA5D4B99ED008A7D
:10B4F8002B44D3ED007AF5EE407AF1EE10FA17D02E
:10B50800584B2B4493ED007A78EE476AB0EEE66A22
:10B51800F4EEC67AF1EE10FA08D5F5EEC06AF1EE4F
:10B5280010FACCBF37EE878A37EE678A83ED008A38
:10B538004D4B1A88930739D0022E37D09AF82E101F
:10B548004A4B07EE901A2B4493ED007A4B42F8EEE3
:10B55800E76A07EE903A26EE877AF8EEE77AB4EED5
:10B56800E77AF1EE10FA0AD407EE901AF8EE677A45
:10B57800F4EEC77AF1EE10FA88BFF0EE477A3C4B4A
:10B588003C4903EB460331F91600B3F90C30C31AF2
:10B5980007EE103AB8EEC77AD007E7EE497A41F1DC
:10B5A8007980354B93ED008A27EE888A059B94F8BD
:10B5B80068212B4493ED01EA78EE4EDA002A00F078
:10B5C800F7802E4BD4F86C2104991B688A1A9A428A
:10B5D80040F3EE809AF84830022B02F08581022E63
:10B5E80004F05184264B1B68990700F19780254B7E
:10B5F80087ED00CA1B689342C0F2CA80F7EE007A52
:10B60800F4EEE79AF1EE10FA40F1D28005991E4B5C
:10B61800D1ED017A93ED007AF0EEE77A3CE000BFD5
:10B628000055002074520020DC4A0020D02400205D
:10B63800B83E0020E464002000247449C846002075
:10B64800F0380020FC380020CDCCCC3DAE47813FFF
:10B65800000000000000C84200003443610BB63B04
:10B66800BC46002014260020E0640020202600208C
:10B67800C43E002090640020A4460020D04600204C
:10B688008C640020CC460020D8460020E04A0020E8
:10B698000826002008390020F4EEC77AF1EE10FAE7
:10B6A80040F18680D1ED027AF0EEE77AB4EEE77ADF
:10B6B800F1EE10FA7CDDD1ED037AF0EEE77AB4EE24
:10B6C800E77AF1EE10FA73DD0F4B1B689B075FD525
:10B6D8000E490F4B43E00F4B0F4C1E780293072E79
:10B6E8003FF4A7AE94F828310693002B3FF4B1AE8F
:10B6F800013B84F82831012E01F0AF8213B0BDEC74
:10B708000E8BBDE8F08F00BF8C6400209064002091
:10B71800C43E0020DC4A0020D0240020D34BD4496A
:10B72800DFF8C8E331F916C09EED008ADFF8C0E300
:10B7380087ED00CA03EB460028EE098AB0F90C0031
:10B74800A0EB0C0007EE900AF8EEE77ADEF80000AE
:10B7580027EE888A904278EE4EDABFF64FAFB3F9FB
:10B768000C20B1F900E0C348AEEB020E00688EEA87
:10B77800EE72A2EBEE7282421ADAB3F90E30B1F928
:10B788000220D21A82EAE273A3EBE27398420FDD39
:10B79800B94B1A88002384F86831002A43F074856D
:10B7A800B64AB74B1178186881F00101F5F713F81C
:10B7B800B44B2B4493ED000A039B2DEE000A022E96
:10B7C80020EE2D0AA3EC010A039304F0D583AE4BB7
:10B7D800D7ED006A93ED007AAC4BD3ED007AAC4B11
:10B7E80093ED006AAB4B67EE277A2B4427EEAC7AD1
:10B7F800D3ED007A67EE277AF0EE665AEDEEA75A97
:10B80800B1EE467AB4EEE57AF1EE10FA08DCB4EE61
:10B81800E56AF1EE10FA8CBFB0EE657AB0EE467AC2
:10B8280094ED4C6AF7EE007AB4EEE76AF1EE10FA9E
:10B83800ACBF0123002343B1F0EEE66AF0EEC77A0D
:10B84800F4EEE67AF1EE10FA01D587ED007A022ED1
:10B8580004F0C982904A914B52F826001B68B0EE5A
:10B868004E0A98478E4A8F4B52F826001B68984715
:10B878009AF8373023B18C4B1B88002B00F0718766
:10B88800B0EE4C8A894B38EE400A2B4493ED008A7F
:10B8980083ED000A9AF8483030EE480A20EE288AEC
:10B8A800002B33D0824B1B7813F0010300F0BE86C7
:10B8B800F7EE007AF4EEE79AF1EE10FA94F86831B0
:10B8C800C1F20A85002B00F0F187D4F86C31049A94
:10B8D800D31A784A12689A4218DD774BD3ED007A6A
:10B8E800F0EEEDDAF4EEE7DAF1EE10FA42F10D805F
:10B8F800614B1A88002384F86831002A00F0A28678
:10B908006E494A6912B10A6813604B746C4B94F81B
:10B9180078212B4493ED000A2DEE000A20EE088AC8
:10B9280088ED008A32B9039B87ED00CA03ED01CA8E
:10B9380088ED00CA0136032E09F1040908F104084C
:10B9480007F1040705F104057FF4CFAD029B1A78CF
:10B95800072A01F0C684012A01F0648700230393B3
:10B9680094F88021002A41F0AB81DFF888A1554B7B
:10B97800DAF800201968D60491F82C0000F10C8739
:10B98800DFF87491504AB9F81A3092ED006A4F4ABC
:10B998004F4ED2ED005AD6ED036A4E4A84ED646AE2
:10B9A80007EE103A4C4B92ED005AD3ED007AD3EDE6
:10B9B800013AD3ED024A84ED626AB8EEC77A35EEF1
:10B9C800C64A012236EEC77A84ED614AC4ED655A4B
:10B9D80084F89821C7EE055A0A8D534206EE103AAC
:10B9E8003E4BDFED3F6A93ED005A3E4B93ED004A24
:10B9F800B7EE007AF4EEC75A35EE045AF1EE10FAB3
:10BA080088BFF0EE475A35EE275AB8EEC66AF4EE0C
:10BA1800E65AF1EE10FA07EE902AB4EEC65AB8BF0D
:10BA2800F0EE665AF1EE10FAC4ED685AB8EE677A8D
:10BA380001F13283B4EEC75AF1EE10FA88BFB0EEC6
:10BA4800475A264BDFED286AD3ED017A254B93ED53
:10BA5800014A77EE847A25EE265A77EEA37AB4EE79
:10BA6800E76AF1EE10FA52DC48E000BFC43E00205D
:10BA780090640020D4460020888500208A85002014
:10BA88008C85002078460020B4450020180000204E
:10BA9800EC46002084460020BC450020B845002024
:10BAA800104600200C460020E064002040260020BC
:10BAB800484B0020D0460020DC460020908500201E
:10BAC80090460020E46400204C3D0020B03E002059
:10BAD800004C002084470020FC380020F03800206B
:10BAE80000000000083900206F12833AA4460020A5
:10BAF800CC460020105500205C860020B4EEE77A82
:10BB0800F1EE10FA8CBFB0EE676AB0EE476AED4B03
:10BB18004A8DD3ED027A9FEDEC7A534204EE103A47
:10BB280074EEA77AB8EEC44A26EE076AF4EEC47A31
:10BB3800F1EE10FA0AD407EE102AB8EE474AB4EE2E
:10BB4800E74AF1EE10FA88BFB0EE674ADF4ADFED48
:10BB5800DE7A527824EE274A0AB9B1EE444A002820
:10BB680041F00486B7EE003AD94E3278002A02F046
:10BB78003A86D849DFEDD87AD1ED024AD1ED016A8B
:10BB880091ED037A66EE244AE5EE264AE4EE074A8A
:10BB980063EE244AF4EEE74AF1EE10FAB4BFF0EE91
:10BBA800673AF0EE643A98BFF0EE647A012ACDED78
:10BBB8000A4A02F0658691ED067AD1ED052AD1EDA3
:10BBC800076A26EE077AA5EE227AA4EE267A23EEF5
:10BBD800077AB4EEE77AF1EE10FAB4EEE37A8CBFA6
:10BBE800F0EE676AF0EE476AF1EE10FA88BFF0EE01
:10BBF800676AB4BFF0EE637AF0EE477A022A8DEDF9
:10BC08000B7A00F0DE8091ED0A7AD1ED092AD1EDA8
:10BC18000B3A26EE077AA5EE227AA4EE237A23EED3
:10BC2800077AB4EEE67AF1EE10FAB4EEE77A8CBF52
:10BC3800F0EE663AF0EE473AF1EE10FA98BFF0EE01
:10BC4800636AA8BFF0EE477A032A8DED0C7A00F0FC
:10BC5800B88091ED0E7AD1ED0D2AD1ED0F3A26EE8E
:10BC6800077AA5EE227AA4EE237A23EE077AB4EEB9
:10BC7800E67AF1EE10FAB4EEE77A8CBFF0EE663AA7
:10BC8800F0EE473AF1EE10FA98BFF0EE636AA8BFFB
:10BC9800F0EE477A042A8DED0D7A00F09280D1ED0E
:10BCA800123AD1ED112A91ED137A66EE233AE5EEB8
:10BCB800223AE4EE073A63EE233AF4EEE63AF1EE7E
:10BCC80010FAF4EEE73A8CBFB0EE667AB0EE637A1B
:10BCD800F1EE10FA98BFF0EE476AA8BFF0EE637A6B
:10BCE800052ACDED0E3A6CD0D1ED163AD1ED152AD4
:10BCF80091ED177A66EE233AE5EE223AE4EE073A3A
:10BD080063EE233AF4EEE63AF1EE10FAF4EEE73A8F
:10BD18008CBFB0EE667AB0EE637AF1EE10FA98BF97
:10BD2800F0EE476AA8BFF0EE637A062ACDED0F3A27
:10BD380047D0D1ED1A3AD1ED192A91ED1B7A66EE6A
:10BD4800233AE5EE223AE4EE073A63EE233AF4EEBC
:10BD5800E63AF1EE10FAF4EEE73A8CBFB0EE667A06
:10BD6800B0EE637AF1EE10FA98BFF0EE476AA8BF1A
:10BD7800F0EE637A072ACDED103A22D091ED1E7AC3
:10BD8800D1ED1D2AD1ED1F3A26EE077AA5EE227ACB
:10BD9800A3EE847A27EE037AB4EEE67AF1EE10FA8F
:10BDA800B4EEE77A8CBFB0EE666AB0EE476AF1EEA1
:10BDB80010FA8DED117A98BFF0EE466AA8BFF0EE42
:10BDC800477A77EEE67AF7EE006AF4EEE67AF1EE75
:10BDD80010FAC4ED4C7A43F3868586EEA77A022AD8
:10BDE800DDED0B7A67EE244A67EE877ACDED0A4AD5
:10BDF800CDED0B7A2DD0DDED0C7A67EE877A032A2C
:10BE0800CDED0C7A25D0DDED0D7A67EE877A042A20
:10BE1800CDED0D7A1DD0DDED0E7A67EE877A052A15
:10BE2800CDED0E7A15D0DDED0F7A67EE877A062A0A
:10BE3800CDED0F7A0DD0DDED107A67EE877A072AFF
:10BE4800CDED107A05D0DDED117A27EE877A8DEDEC
:10BE5800117A2249096811F0805801F0F081F6EE54
:10BE6800005AC4ED685A002A02F0B7841C4B94EDBE
:10BE7800656A1C491C4F1D78DFF874E094F9983105
:10BE880094ED645AB7F90670C878DAF80010DEED58
:10BE9800004A0597BDEEC66A07EE103AB9F81A705F
:10BEA800124B079716EE10EABDEEC56A05F0010CB5
:10BEB80001F4805701F0100501F4800108911B7806
:10BEC80018E000BFF03800206F12833A5C39002078
:10BED800BD4A0020F446002000000000A43E0020D7
:10BEE800484B0020403F00204A840020345700205F
:10BEF800F0460020D4ED616AD4ED627AB8EEC77AD4
:10BF080016EE101A002840F02F87002D41F0FD8210
:10BF1800D24D9DED0A5A95ED006AD14825EE866A04
:10BF2800A5EE076AB0EE675AA6EE265ABDEEC56AB8
:10BF380016EE108A16EE107AF045A8BF77464145EE
:10BF4800C8BF0F4606EE107AB8EEC66A012A80ED21
:10BF5800006A00F0DC8095ED046A9DED0B5A25EE31
:10BF6800866AA5EE076AB0EE675AA6EE265ABDEEB7
:10BF7800C56A16EE108A16EE107AF045A8BF774605
:10BF88004145C8BF0F4606EE107AB8EEC66A022AC7
:10BF980080ED016A00F0BB8095ED086A9DED0C5AB2
:10BFA80025EE866AA5EE076AB0EE675AA6EE265A0F
:10BFB800BDEEC56A16EE108A16EE107AF045A8BFD7
:10BFC80077464145C8BF0F4606EE107AB8EEC66AF6
:10BFD800032A80ED026A00F09A8095ED0C6A9DEDC7
:10BFE8000D5A25EE866AA5EE076AB0EE675AA6EEE8
:10BFF800265ABDEEC56A16EE108A16EE107AF0457E
:10C00800A8BF77464145C8BF0F4606EE107AB8EE7E
:10C01800C66A042A80ED036A79D095ED106A9DED11
:10C028000E5A25EE866AA5EE076AB0EE675AA6EEA6
:10C03800265ABDEEC56A16EE108A16EE107AF0453D
:10C04800A8BF77464145C8BF0F4606EE107AB8EE3E
:10C05800C66A052A80ED046A59D095ED146A9DEDEB
:10C068000F5A25EE866AA5EE076AB0EE675AA6EE65
:10C07800265ABDEEC56A16EE108A16EE107AF045FD
:10C08800A8BF77464145C8BF0F4606EE107AB8EEFE
:10C09800C66A062A80ED056A39D095ED186A9DEDC5
:10C0A800105A25EE866AA5EE076AB0EE675AA6EE24
:10C0B800265ABDEEC56A16EE108A16EE107AF045BD
:10C0C800A8BF77464145C8BF0F4606EE107AB8EEBE
:10C0D800C66A072A80ED066A19D095ED1C6A9DED9F
:10C0E800115A65EE865AE7EE055AE6EEA57AFDEE98
:10C0F800E77A17EE905AAE45A8BFAE46A942D8BF18
:10C10800714607EE901AF8EEE77AC0ED077ABCF1AF
:10C11800000F00F03687534A1268002A40F03E8725
:10C12800514A127892B1307868B14D4FDFF8588192
:10C138000025E8B2D8F80030B7EC010A9847307803
:10C1480001358542F5DB494A12689047029B1A7807
:10C15800072A01F0DC800025DAF80020530501F1F8
:10C168001080434B1B78BBB1424AB9F81A30B2F978
:10C1780006209A4210DC404B1B78012B01F07A8391
:10C18800192B01F077830E2B06D0082B04D03B4ED9
:10C198000023B360C4F8403194F8AA6126B1384B43
:10C1A8001B889F0741F0288394F8B021002A40F0AB
:10C1B800878799F81E70002F00F03084022F01F055
:10C1C8000A83032F41F0038399F82030C3EB43110E
:10C1D80003EB8101C90089B299F81F300233DBB241
:10C1E800002A00F08385002900F08085254807682B
:10C1F800B1FBF7F10FB2A4F8E071002B03F0548003
:10C2080007EE907AF8EEE77AF7EE006A86EEA77AFC
:10C218001A4E012BD4ED7D6AD6ED007A77EEE67AD8
:10C2280067EE877AC4ED797A3AD0D6ED017AD4ED03
:10C238007E6A77EEE67A022B67EE877AC4ED7A7A21
:10C248002ED0D6ED027AD4ED7F6A77EEE67A032B0C
:10C2580067EE877AC4ED7B7A22D017E0F446002097
:10C2680024390020B04500205C5A002030570020B7
:10C27800E42000204A8400205C390020004C002083
:10C28800E06400204439002028570020D6ED037AC6
:10C29800D4ED806A77EEE67A67EE877AC4ED7C7A29
:10C2A80002990978092903F03B81002F40F3BC83E8
:10C2B8009BB394ED7D7AD4ED797A77EE877A012B6A
:10C2C800C4ED7D7AC6ED007A21D094ED7E7AD4ED66
:10C2D8007A7A77EE877A022BC4ED7E7AC6ED017AF8
:10C2E80015D094ED7F7AD4ED7B7A77EE877A032B9D
:10C2F800C4ED7F7AC6ED027A09D0D4ED807A94ED48
:10C308007C7A77EE877AC4ED807AC6ED037A013BB2
:10C31800022BB8BF0223DBB20693069B002A18BF84
:10C3280002239E46CC4BDFEDCD6A1A68029B9178BA
:10C338001878137807EE903AF8EEE77AB0EE007ABC
:10C3480067EEA67AF4EEC77AF1EE10FA40F38F861C
:10C35800DFEDC36A37EEC77AB0EE676AA7EE266AE2
:10C36800F0EE466A96ED007A9FEDBE6A27EE066A01
:10C37800F0EEC65A84ED546AC4ED575A99B107EEE7
:10C38800101AB8EEC75A9FEDB57A66EE064A25EE42
:10C39800075AB7EE007A37EE457A64EEA54AA4EE5E
:10C3A800857A26EE076A9FEDB07A537926EE877A6A
:10C3B80027EE067ACBB1DFEDA96A9FEDAC6A65EE90
:10C3C800A65A06EE903AF8EEE66A66EEA56AF4EE2C
:10C3D800C66AF1EE10FA01F3A081F7EE005A75EE85
:10C3E800E66A85EEA66A27EE067A0C289FEDA08AF3
:10C3F800DFEDA06A00F04A87B4EEC87AF1EE10FAD1
:10C4080098BFB0EE478AB4EEE68AF1EE10FAB8BFEC
:10C41800B0EE668A84ED4E8ABEF1000F00F0DD8032
:10C42800B0EE007AF4EEC77AF1EE10FA05DD37EED9
:10C43800C77ADFED8B6AE7EE267A96ED017ADFEDB3
:10C44800896A27EE267AF0EEC75A84ED557AC4ED4C
:10C45800585A99B106EE901A9FED806AF8EEE66A8E
:10C4680027EE075A66EE866AB7EE006A36EE666A07
:10C4780025EE255AA5EE266A27EE067ADFED7A6ABA
:10C48800937967EEA67A67EE877AABB107EE103A32
:10C49800B8EEC77A9FED716ADFED746A27EE257AE8
:10C4A80027EE067AB4EEE67AF1EE10FA41F3398116
:10C4B800DFED716A67EEA67A0C2800F0C786DFED1B
:10C4C8006C6A9FED6C7AF4EEE67AF1EE10FA88BFAA
:10C4D800F0EE667AF4EEC77AF1EE10FAB8BFF0EE35
:10C4E800477ABEF1010FC4ED4F7A76DD5378DFED60
:10C4F8005B6A07EE903AF8EEE77AB0EE007A67EEFC
:10C50800A67A537AF4EEC77AF1EE10FA05DD37EE23
:10C51800C77ADFED536AE7EE267A96ED027ADFED09
:10C52800516A27EE267AF0EEC75A84ED567AC4EDA2
:10C53800595A9BB106EE903A9FED486AF8EEE66AC2
:10C5480027EE075A66EE866AB7EE006A36EE666A26
:10C5580025EE255AA5EE266A27EE067ADFED426A11
:10C56800D37967EEA67A67EE877AFBB107EE103AC1
:10C57800B8EEC77A9FED396ADFED3C6A27EE257A77
:10C5880027EE067AB4EEE67AF1EE10FA01F3D780D8
:10C59800B5EEC07AF1EE10FA02F10683B7EE006A42
:10C5A80036EE477AC6EE076A67EEA67A0C2800F0E0
:10C5B8008B86DFED2F6A9FED2F7AF4EEE67AF1EEA7
:10C5C80010FA88BFF0EE667AF4EEC77AF1EE10FA48
:10C5D800B8BFF0EE477AC4ED507A092800F02286F9
:10C5E80099F82160002E40F0D785002384F8B031F7
:10C5F80015F032F8002840F03D83204B1B7823B912
:10C608001F4B9B78002B41F0F280049805F012FA3A
:10C61800029B1E78072E7FF46EA8F8F7D3FE194BFD
:10C62800029A401B1678D880FFF765B894F86821FD
:10C63800002A3FF46BA9144A84F868311288002A4A
:10C648007FF45EA9114A124B1178186881F0010134
:10C65800F4F7C1F8FFF75AB9E86400200AD7233C79
:10C66800D7A368416F12033B00004843A4707D3F85
:10C6780000C0F94400C0F9C40000C842A34100202A
:10C688006E600020E04A0020888500208A8500200E
:10C698008C85002094ED577AB1F90000D4ED586AE2
:10C6A800B1F902E0E24AF4EEC76A80EAE0738EEA82
:10C6B800EE71A3EBE073F1EE10FAA1EBEE71B8BFE7
:10C6C800F0EE476A8B42B8BF0B4607EE103A137874
:10C6D800B8EEC77A27EE097A002B40F0B880D54B20
:10C6E80093ED006AB4EEEA6AF1EE10FA41F17A804D
:10C6F800F7EE005A75EEC65A3BEEC77A65EE8B5ACE
:10C70800CD4BA7EE256A93ED007A26EE076AB5EEC3
:10C71800C06AF1EE10FA40F28E85CAEE065AB7EEFC
:10C72800007AB0EE476AA6EEE56AF0EE466AF4EEE5
:10C73800C76AF1EE10FA88BFF0EE476AF5EEC06AF4
:10C74800F1EE10FAB8BFF0EE4C6ABC4B93ED007AEC
:10C7580067EE877AA7EEA68AFEF728BF0122FEF7C2
:10C7680081BEB74BB74A2B4493ED007AD2ED007ADD
:10C77800B54B67EE277AF7EE006AF4EEE67AF1EE4B
:10C7880010FA93ED007A88BFF0EE667A67EE877A42
:10C7980027EE888AFFF776B8AC4BDFF8EC921A7868
:10C7A800AB4ED5075CBFB9F81820A4F88C21A94A6C
:10C7B800D6ED037A128807EE102AB8EEC77AF4EE9F
:10C7C800C77AF1EE10FA41F2C587A34D2B8807EE20
:10C7D800103AB8EEC77AF4EEC77AF1EE10FAC1F261
:10C7E80055809E4A9E4D92ED006AD5ED006A94F9F7
:10C7F8009821C4ED646A76EE665A012AC4ED626A2D
:10C80800C4ED615A84ED656A01F0D785049BC4F8CC
:10C818009C31002537EEC77AFCEEE77A914E84ED1D
:10C82800687A17EE902AA4F88C21012296ED005A16
:10C8380084F898218C4A954241F2BC878B4BD3ED02
:10C84800007AD3ED013AD3ED024AFFF7C3B87A4B29
:10C8580093ED005AB5EEC05AF1EE10FA40F3EB84AE
:10C86800834BD3ED004AF5EEC04AF1EE10FA40F3DF
:10C87800E28434EEC77A66EECA5A87EE246AC5EEB9
:10C88800856AB7EE007AB4EEC76AF1EE10FA88BF8F
:10C89800B0EE476AB5EEC06AF1EE10FA76EE876A36
:10C8A800B8BFB0EE4C6A66EE266A40E7714AD2ED30
:10C8B800007AB0EEC87AB4EEE77AF1EE10FA7FF7B4
:10C8C80025A86D4AD2ED007AB0EEED7AB4EEE77A9B
:10C8D800F1EE10FA7FF71AA8684AD9ED007A92EDBE
:10C8E800007AF0EEE77AF4EEC77AF1EE10FA7FF507
:10C8F8000DA801220499C4F86C1184F86821FEF788
:10C90800E8BF07EE102A1978DFF88081C4F80C71A7
:10C91800B8EEC77AF7EE006A132986EE879AB8F957
:10C928000400B4F810619BED070A01F0D284544A60
:10C93800544992ED001AD2ED053A92ED122A92ED81
:10C94800173AD2ED091AD2ED0E4A92ED016A92ED2C
:10C95800064A92ED0A7AD2ED0F5AD2ED132AD2ED99
:10C96800186A92ED045AD2ED030A67EE897A69EEE5
:10C97800288A29EE088AE1EE273A01EB8607002586
:10C98800A2EE283AC4F80051C4F80451E1EE884AEE
:10C99800A6EE274AE7EE085A92ED167A92ED0D6A4E
:10C9A80092ED021AD2ED0C1AC7ED003AE2EEA86A2F
:10C9B80025EE635A27EE437A92ED0B2AD2ED152A1B
:10C9C800C7ED204AA0EEE34A26EE646AD2ED143A97
:10C9D80082ED054AA1EE275AF0EE477AE1EEE45AD5
:10C9E800A2EE086AE2EEC36AE3EEA87A82ED065A7E
:10C9F800C2ED0E5A82ED0F6A87ED403AC2ED176A12
:10CA0800C2ED187AC4F80851721C02F01F02A4F88B
:10CA18001021A8F80400029BFEF723BCA4F8E071DB
:10CA2800002A3FF4E5AD0A4E4FF0020E7AE400BF4B
:10CA3800B0460020B8460020AC460020A84600209A
:10CA48002C260020A04600209C460020484B0020B1
:10CA5800004C0020884700208A470020B03E002074
:10CA680074470020904700208FD00300FC38002036
:10CA7800B4460020E0460020DC460020E4460020C2
:10CA8800FC3B0020903900205C860020E04A002012
:10CA98009C4A1178D4F818719B4B9FED9C7AFE0044
:10CAA8009A1982ED007A002979D09948B0EE476A40
:10CAB800F0EE476A0022F0EC017A013267EEA77ABD
:10CAC80005EE902AB4EEE77AF1EE10FAF8EEE55AA0
:10CAD800B8BFB0EE677A8A4276EEA76AA7EEA56A73
:10CAE800E9D1F5EEC06A9A19F1EE10FA82ED007AF2
:10CAF80055DDC6EE265A874A87490988F7EE007A37
:10CB080075EEE75AD2ED007A65EEA77AFDEEE77A80
:10CB180017EE902A812A42F357808A42A8BF0A4614
:10CB280007EE902AF8EEE77A7C4AF01902EB8002C9
:10CB380092ED057AD2ED003A92ED066A92ED014A3D
:10CB4800D2ED046AD2ED034A92ED025AA3EEA77A17
:10CB5800A4EE276A66EEC76AA7EE646ABDEEC77AD6
:10CB6800E5EE276A17EE100A812882ED056AC2ED04
:10CB7800066A42F326808142A8BF014607EE901A52
:10CB8800F8EEE77AFCEEE77ACDED057ABDF81420E9
:10CB980099198A801FB9BEF1130F02F0AC86BEF155
:10CBA800150F41F0DC801E44DFF89081B28828F828
:10CBB8001720D4F814515A4A013582FB053251190D
:10CBC800EA17C2EBA102C2EBC202AD1AC4F81451B3
:10CBD8005448D4F81C11049B534D02682D78C4F8AE
:10CBE8001C31591A0A440260002D40F0DB8107EE1F
:10CBF800901A4E4EDFF864914D4FB8EEE78A06F56D
:10CC0800F07506F51378F6EC017A9BED070ADBF868
:10CC18000832F8EEE77A284627EE800A9847A5F109
:10CC2800E000DBF828319847A5F17000DBF898316F
:10CC38009847D6F8EC00DBF8AC309847D7ED007A87
:10CC4800A9EC010AE0EE087A2435A845E7EC017A58
:10CC5800D9D1029B1E78FEF742BD364B364A196879
:10CC68001288364BC96919805A8013B0BDEC0E8BF7
:10CC7800BDE8F08F324C14F0E5FB6378022B00F02E
:10CC8800E985032B7FF4B9AC41F2B813E35C002BC0
:10CC980041F0158341F2A403E35C002B41F00A83C1
:10CCA80041F2E803E35C002B41F00E8341F22C13C0
:10CCB800E35C002B3FF4A1AC224824F08DFD9CE4FA
:10CCC800214B224E1A7812F0010F327840F04C8333
:10CCD800002A00F0458592001D491E48DFF880A013
:10CCE800DFF8809027F020FBFFF715BAB4F8E07161
:10CCF800013F3FB2002FA4F8E0717FF791AE164EC6
:10CD0800FFF7D6BA72390020683C00200000000006
:10CD1800D02400207439002070390020903B002076
:10CD2800932449927445002068390020B4520020A9
:10CD3800784500204C66002068310020E04A002039
:10CD4800CC660020F8770020484B0020BD4A002020
:10CD58003830002024390020004C002004550020E1
:10CD6800105500205C860020002D00F0BD86BCF127
:10CD7800000F42F0A382CA4D002B42F0378195ED97
:10CD8800006A9DED0A5AC74825EE866AFDEEE44A18
:10CD9800A5EE076AB0EE675AA6EE265A14EE901A68
:10CDA800BDEEC56A16EE10CA16EE107AF445A8BF95
:10CDB80077466145C8BF0F4606EE107AB8EEC66AD8
:10CDC800012A80ED006A00F0DF8095ED046A9DED90
:10CDD8000B5A25EE866AA5EE076AB0EE675AA6EEEC
:10CDE800265ABDEEC56A16EE10CA16EE107AF4453C
:10CDF800A8BF77468C45B8BF0F4606EE107AB8EE46
:10CE0800C66A022A80ED016A00F0BE8095ED086AC4
:10CE18009DED0C5A25EE866AA5EE076AB0EE675AB4
:10CE2800A6EE265ABDEEC56A16EE10CA16EE107AA0
:10CE3800F445A8BF77468C45B8BF0F4606EE107A72
:10CE4800B8EEC66A032A80ED026A00F09D8095ED6F
:10CE58000C6A9DED0D5A25EE866AA5EE076AB0EEBE
:10CE6800675AA6EE265ABDEEC56A16EE10CA16EE29
:10CE7800107AF445A8BF77468C45B8BF0F4606EE32
:10CE8800107AB8EEC66A042A80ED036A7CD095ED64
:10CE9800106A9DED0E5A25EE866AA5EE076AB0EE79
:10CEA800675AA6EE265ABDEEC56A16EE10CA16EEE9
:10CEB800107AF445A8BF77468C45B8BF0F4606EEF2
:10CEC800107AB8EEC66A052A80ED046A5CD095ED42
:10CED800146A9DED0F5A25EE866AA5EE076AB0EE34
:10CEE800675AA6EE265ABDEEC56A16EE10CA16EEA9
:10CEF800107AF445A8BF77468C45B8BF0F4606EEB2
:10CF0800107AB8EEC66A062A80ED056A3CD095ED1F
:10CF1800186A9DED105A25EE866AA5EE076AB0EEEE
:10CF2800675AA6EE265ABDEEC56A16EE10CA16EE68
:10CF3800107AF445A8BF77468C45B8BF0F4606EE71
:10CF4800107AB8EEC66A072A80ED066A1CD095EDFD
:10CF58001C6A9DED115A65EE865AE7EE055AE6EE13
:10CF6800A57AFDEEE77A17EE905AAE45A8BFAE4611
:10CF7800A942D8BF714607EE901AF8EEE77AC0EDDD
:10CF8800077A002A3FF4C7A892004749454827F086
:10CF9800CBF9464A1268002A3FF4C2A808F038FBC9
:10CFA800FFF7BEB807EE901A414D424BDFF80881F3
:10CFB800DFF808910394F8EEE78A05F5B8760027BC
:10CFC800CDF818801C46029BDBED077A1B78172BDF
:10CFD80051D095ED007AB8EEC78A082B28EE278A3B
:10CFE80007D1B0EE480A059327F072FB059BA8F815
:10CFF8000000DAF8002092000BD5002F02F0078716
:10D00800B0EE480ADBF8083206F170009847B0EE37
:10D01800408AB0EE480ADBF82831A6F1700098473C
:10D02800DBF8983130469847029B1B78032BB0EE0B
:10D03800408A2CD0D5F8F000DBF8AC30B0EE480AC6
:10D048009847D9ED007AA4EC010AE0EE287A013776
:10D05800032F06F1240608F1020805F10405E9EC9E
:10D06800017AB0D1029B039C1E78FEF738BBF0EE24
:10D07800676AFFF777B995ED007A0BEB4702B8EED0
:10D08800C78A128FA8F8002028EE278AB1E727F070
:10D098001FFBA8F80000CDE7B0EE465AFEF7D1BC5A
:10D0A800F44600202439002038300020B045002004
:10D0B800B452002004550020E04A002078450020A2
:10D0C8009B499C4BD1F8EC101B6844F620608142C8
:10D0D800A8BF0146B1F57A7FB8BF4FF47A7189B21B
:10D0E80013F0100FA4F8B211DAF8003000F0C98379
:10D0F800DB0441F16D85904BD3F800E0BEF8327047
:10D108007F088E4E8E48D4F8B431D6ED037AA0FB52
:10D1180001018809642191FBF0F11429BDEEE77A39
:10D1280004EB4306A8BF142101339942C4F8B43173
:10D1380017EE10CADCBF0023C4F8B43104EB430374
:10D14800A6F8B8C1B3F9B83107EE103AB8EEC77A05
:10D1580077EEC77AFDEEE77ACDED037ABDF90C10CC
:10D1680081EAE173A3EBE173BB4201F3A48675493D
:10D178004FF07E530B60FFF71CB8734B0293734C50
:10D1880026E5DBF80830002B3EF4EBAF7049A1F13F
:10D198004C009847FEF7E5BF1E216648F4F7A3FB4D
:10D1A80000283FF422AA6B4B1B885A063FF51DAA9C
:10D1B80094F80432B34242F0D581624BD4ED827ABE
:10D1C800D3ED016A94ED505ADFED635A9FED636A1F
:10D1D80027EEC57A68EE277AA8EE267AE5EE267A53
:10D1E800B4EEE57AF1EE10FA88BFB0EE657AB4EEE7
:10D1F800C67AF1EE10FAF4EEE57AB8BFB0EE467AE8
:10D20800F1EE10FA88BFF0EE657AF4EEC67AF1EE28
:10D2180010FAB8BFF0EE467A84ED4E7AC4ED507A33
:10D22800FFF7E3B9FDEEC87A4D4A17EE903A9780BA
:10D23800D380FFF7D5B9DFED4B6AFFF786BADAF886
:10D24800001049023EF50BAEFEF70DBE9FED427A87
:10D25800DFED426A4249F4EEC77AF1EE10FA98BF60
:10D26800B0EE677AFDEEE77AB4EEE67AF1EE10FA00
:10D2780017EE903AB8BFB0EE667ABEF1010F84EDB2
:10D288004F7A4B803FF732A9FFF7AAB9B4EEC87AB4
:10D29800F1EE10FA98BFB0EE478ABDEEC77AB4EE49
:10D2A800E68ADFF8BCC0F1EE10FA17EE103AB8BF04
:10D2B800B0EE668A84ED4E8AACF80030BEF1000FFD
:10D2C8007FF4AEA8FFF78CB9BDEEE77A244B17EED2
:10D2D800102A9A80FFF76DB9002B3EF417ABFEF7C2
:10D2E800F4BAF8F76FF8029BDFF874801A78079B96
:10D2F800012AA0EB0300A8F8020000F09582072A93
:10D308007EF42CABF8F75EF80390FEF729BBF8F72C
:10D3180059F8029B12491A78039B072AA0EB0300CD
:10D3280088807EF418AFF8F74DF80546FEF714BF6D
:10D3380058010020A43E0020E4640020004C002096
:10D34800D34D621018000020DC4A0020D0240020B1
:10D35800D4520020E064002000C0F94400C0F9C4A1
:10D36800E04A002000000000002A00F0F981D4ED16
:10D37800583A94ED574AD4ED627AF34994ED617ABC
:10D3880091ED005AD4ED555A94ED546AEF4DF0489A
:10D39800F4EEC43AF3EE046AF1EE10FA77EEA64A18
:10D3A80000F1C28295ED026A26EE656AB0EE674A20
:10D3B800A6EE074AB4EEE44A34EE666AF1EE10FAD5
:10D3C80048BFB0EE456A012A80ED006A00F0C881C6
:10D3D80095ED066A26EE656AB0EE674AA6EE074A3C
:10D3E800B4EEE44A34EE666AF1EE10FA48BFB0EEE5
:10D3F800456A022A80ED016A00F0B28195ED0A6A59
:10D4080026EE656AB0EE674AA6EE074AB4EEE44A2D
:10D4180034EE666AF1EE10FA48BFB0EE456A032AA8
:10D4280080ED026A00F09C8195ED0E6A26EE656A31
:10D43800B0EE674AA6EE074AB4EEE44A34EE666AEE
:10D44800F1EE10FA48BFB0EE456A042A80ED036A8F
:10D4580000F0868195ED126A26EE656AB0EE674A9D
:10D46800A6EE074AB4EEE44A34EE666AF1EE10FA24
:10D4780048BFB0EE456A052A80ED046A00F0708165
:10D4880095ED166A26EE656AB0EE674AA6EE074A7B
:10D49800B4EEE44A74EE666AF1EE10FA48BFF0EEB4
:10D4A800456A062AC0ED056A00F05A81D5ED1A6A68
:10D4B80066EEE56AB0EE674AA6EE874AB3EE046AFE
:10D4C800B4EEE44A74EE466AF1EE10FA48BFF0EEA4
:10D4D800456A072AC0ED066A00F04281D5ED1E6A4A
:10D4E800DFF874A2DFF8749266EEE55AE5EE877A03
:10D4F800F4EEE74A77EEC67AF1EE10FAC8BFF0EE1E
:10D50800457AC0ED077AFEF706BE904D9DED0A5AA2
:10D5180095ED006ABCF1000F41F0E68125EE866AC0
:10D528008B48A5EE076AB0EE675AA6EE265ABDEEFE
:10D53800C56A16EE10CA16EE107AF445A8BF7746EB
:10D548006145C8BF0F4606EE107AB8EEC66A012AD2
:10D5580080ED006A3FF418AD95ED046A9DED0B5A15
:10D5680025EE866AA5EE076AB0EE675AA6EE265A39
:10D57800BDEEC56A16EE10CA16EE107AF445A8BFBD
:10D5880077466145C8BF0F4606EE107AB8EEC66A00
:10D59800022A80ED016A3FF4F7AC95ED086A9DED2B
:10D5A8000C5A25EE866AA5EE076AB0EE675AA6EE13
:10D5B800265ABDEEC56A16EE10CA16EE107AF44564
:10D5C800A8BF77466145C8BF0F4606EE107AB8EE89
:10D5D800C66A032A80ED026A3FF4D6AC95ED0C6A60
:10D5E8009DED0D5A25EE866AA5EE076AB0EE675ADC
:10D5F800A6EE265ABDEEC56A16EE10CA16EE107AC9
:10D60800F445A8BF77466145C8BF0F4606EE107AB5
:10D61800B8EEC66A042A80ED036A3FF4B5AC95ED0E
:10D62800106A9DED0E5A25EE866AA5EE076AB0EEE1
:10D63800675AA6EE265ABDEEC56A16EE10CA16EE51
:10D64800107AF445A8BF77466145C8BF0F4606EE75
:10D65800107AB8EEC66A052A80ED046A3FF494ACE5
:10D6680095ED146A9DED0F5A25EE866AA5EE076AB8
:10D67800B0EE675AA6EE265ABDEEC56A16EE10CA77
:10D6880016EE107AF445A8BF77466145C8BF0F4625
:10D6980006EE107AB8EEC66A062A80ED056A3FF4EF
:10D6A80073AC95ED186A9DED105A25EE866AA5EEC5
:10D6B800076AB0EE675AA6EE265ABDEEC56A16EEA0
:10D6C80010CA16EE107AF445A8BF77466145C8BF60
:10D6D8000F4606EE107AB8EEC66A072A80ED066A8B
:10D6E8003FF452AC95ED1C6A9DED115A65EE865AD1
:10D6F800E7EE055AE6EEA57AFDEEE77A17EE905AC0
:10D70800AE45A8BFAE46A942C8BF8E4607EE90EA0E
:10D71800F8EEE77AC0ED077A33E49FED0E6AFEF77C
:10D7280062BEB5EEC07AF1EE10FA01F14182B7EEB1
:10D73800006A36EE477AC6EE076AFEF7BBBEDFED33
:10D74800056AFEF731BF00BFF0460020F44600200E
:10D75800243900200000C842105500205C860020B3
:10D76800DFF878A3DFF87893FEF7D5BCC8494A7983
:10D77800002A3EF4F7A9C74A1278002A3EF4F2A913
:10D788000B78C549DFEDC54A07EE903A0B88B8EE2D
:10D79800677A07EE902A06EE903AF8EEE77AF8EE06
:10D7A800666A67EE277AB7EE007A87EEA63AB4EE95
:10D7B800E43AF1EE10FA88BFB0EE643AB4EEC73A34
:10D7C800F1EE10FAB8BFB0EE473AFEF7CDB9B44B58
:10D7D8005988FEF701BDB4F8B21101F57A7189B222
:10D7E800FEF7FABCAF4B93ED006AFEF790BF0498C2
:10D7F8000DF0B0F9FEF709BFAB4B9FEDAC7AD3ED56
:10D80800087AF4EEC77AF1EE10FA00F2F7849FED89
:10D81800A87AA84ED6ED037A77EE877AC6ED037A12
:10D82800FEF7C2BCDFF8BC82F7F7CCFDA249D4F8FA
:10D838007C2109680390821A511AC4F87C01A8F85F
:10D848000420A8F80610FEF78BB8F7F7BBFD079081
:10D85800FDF70FBEA3784FF0010A072B3EF6CDAEB9
:10D86800DFE813F03D0755072D072207BE0682069D
:10D878008C063907914B9B7B002B3EF488ACFEF756
:10D888008BBCD8003FF534ACFEF793BCB4F88C5190
:10D89800954240F2FE8494F8A451002D40F0C687CA
:10D8A800874A884E92ED007AD6ED007A94F998214D
:10D8B800C4ED647A77EE676A012AC4ED627AC4ED32
:10D8C800616A84ED657A02F00880049BC4F89C3193
:10D8D8007D4A9FED777A92ED005A84ED687A0122AD
:10D8E80084F89821FEF7A6BF784B1B88002B40F0E0
:10D8F800F385774A774B11781868F2F76CFFD4F8FC
:10D908006C21049B9A1AFDF76ABE734BD9ED007A15
:10D9180093ED007AF0EEE77AF4EEC77AF1EE10FABA
:10D928007DF7F4AFFDF7E4BFD5ED015A65EEC65AB1
:10D93800B0EE674AA5EE874AB4EEE44A74EE665A3A
:10D94800F1EE10FA48BFF0EE455A012AC0ED005A30
:10D958003FF406AFD5ED055A65EEC65AB0EE674AF4
:10D96800A5EE874AB4EEE44A74EE665AF1EE10FA70
:10D9780048BFF0EE455A022AC0ED015A3FF4F0AE16
:10D98800D5ED095A65EEC65AB0EE674AA5EE874A44
:10D99800B4EEE44A74EE665AF1EE10FA48BFF0EEBF
:10D9A800455A032AC0ED025A3FF4DAAED5ED0D5AB6
:10D9B80065EEC65AB0EE674AA5EE874AB4EEE44A69
:10D9C80074EE665AF1EE10FA48BFF0EE455A042A92
:10D9D800C0ED035A3FF4C4AED5ED115A65EEC65AF0
:10D9E800B0EE674AA5EE874AB4EEE44A74EE665A8A
:10D9F800F1EE10FA48BFF0EE455A052AC0ED045A78
:10DA08003FF4AEAED5ED155A65EEC65AB0EE674A8C
:10DA1800A5EE874AB4EEE44A74EE666AF1EE10FAAF
:10DA280048BFF0EE456A062AC0ED056A3FF498AE95
:10DA3800D5ED196A66EEC66AB0EE674AA6EE874A61
:10DA4800F3EE045AB4EEE44A74EE656AF1EE10FAA5
:10DA580048BFF0EE456A072AC0ED066A3FF480AE7B
:10DA6800D5ED1D6ADFF874A0DFF8749026EEC66A5B
:10DA7800E6EE077AF4EEE47A77EEE57AF1EE10FA5C
:10DA8800B8BFF0EE457AC0ED077AFEF744BB00BF99
:10DA98007C640020FE4B0020E84B0020713DAA3F2B
:10DAA800E0510020AC4600204C4500208FC2753C58
:10DAB80000000000004C002044390020188A002093
:10DAC800B03E002074470020904700208885002041
:10DAD8008A8500208C850020E4460020105500200F
:10DAE8005C860020E04A0020D94D002B41F0A08040
:10DAF80095ED006A9DED0A5AD64825EE866AFDEE38
:10DB0800E44AA5EE076AB0EE675AA6EE265A14EE66
:10DB1800901ABDEEC56A16EE108A16EE107AF04518
:10DB2800A8BF77464145C8BF0F4606EE107AB8EE43
:10DB3800C66A012A80ED006A3EF4E9AA95ED046AF6
:10DB48009DED0B5A25EE866AA5EE076AB0EE675A78
:10DB5800A6EE265ABDEEC56A16EE108A16EE107AA3
:10DB6800F045A8BF77468845B8BF0F4606EE107A3D
:10DB7800B8EEC66A022A80ED016A3EF4C8AA95ED9D
:10DB8800086A9DED0C5A25EE866AA5EE076AB0EE86
:10DB9800675AA6EE265ABDEEC56A16EE108A16EE2C
:10DBA800107AF045A8BF77468845B8BF0F4606EEFD
:10DBB800107AB8EEC66A032A80ED026A3EF4A7AA74
:10DBC80095ED0C6A9DED0D5A25EE866AA5EE076A5D
:10DBD800B0EE675AA6EE265ABDEEC56A16EE108A52
:10DBE80016EE107AF045A8BF77468845B8BF0F46AD
:10DBF80006EE107AB8EEC66A042A80ED036A3EF48F
:10DC080086AA95ED106A9DED0E5A25EE866AA5EE58
:10DC1800076AB0EE675AA6EE265ABDEEC56A16EE3A
:10DC2800108A16EE107AF045A8BF77468845B8BF27
:10DC38000F4606EE107AB8EEC66A052A80ED046A29
:10DC48003EF465AA95ED146A9DED0F5A25EE866A95
:10DC5800A5EE076AB0EE675AA6EE265ABDEEC56A6B
:10DC680016EE108A16EE107AF045A8BF774688455A
:10DC7800B8BF0F4606EE107AB8EEC66A062A80EDDF
:10DC8800056A3EF444AA95ED186A9DED105A25EEF2
:10DC9800866AA5EE076AB0EE675AA6EE265ABDEE6A
:10DCA800C56A16EE108A16EE107AF045A8BF7746B8
:10DCB8008845B8BF0F46FEF708BA674ED4ED017A1B
:10DCC80094ED006A3188726977EEA77AF0EE006AFF
:10DCD800B0EE677AA6EE267A4E1E04EBC601D6EEA3
:10DCE800267A08391032F6EE003A27EE237A67EEE4
:10DCF800A37A84ED207AC4ED217A584C274604F1A2
:10DD0800800091ED027A91ED036AD7ED036AD7EDB1
:10DD1800027A52ED014A12ED025A37EE674A76EE60
:10DD2800C65A77EE277AE4EE845A013EA1F108013B
:10DD3800E5EE047A07F1080702F1080236EE267AC2
:10DD480000F10800E4EE877AE5EE475A67EEA37A19
:10DD580025EEA37AC0ED007A80ED017AD1D1BEF12B
:10DD6800140F7EF428AFF7F72DFB039BDFF8008133
:10DD7800C01AA8F80200D4F81451FEF71CBFD4F852
:10DD88001831B4F810C1364ACCF120095FFA89F984
:10DD98000CEB431702EB87075FEA990201F0BC8599
:10DDA800013216012F48304907EB060807F1100227
:10DDB80012ED024A12ED035A12ED016A12ED047ACD
:10DDC80050ED024A50ED035A50ED016A50ED047AC5
:10DDD80064EE244A65EE255A66EE266A67EE277ACF
:10DDE8001032904541ED024A41ED035A41ED016A76
:10DDF80041ED047A00F1100001F11001D8D11B485F
:10DE0800A6F110010F4400EB0108214419F00302A8
:10DE180009D0B7EC017AF8EC017A67EE277A013A73
:10DE2800E1EC017AF5D1BCF1000F41F05380BEF16D
:10DE3800140F7EF4C0AEF7F7C5FA039BDFF8308005
:10DE4800D4F81451C01AA8F80200FEF7B4BE00BFF7
:10DE5800F44600202439002078390020D0240020FE
:10DE680090390020203B0020E0240020103B0020B7
:10DE7800E04A0020D04E318873684FEA51094FEAD2
:10DE880089005FEAD10C04EB000204EB810500F085
:10DE9800A18000F110010CF1010CC84F02EB0C1C21
:10DEA8002944103203F1100E05F1100050ED032A39
:10DEB80050ED043A17ED043A17ED032A50ED026AC3
:10DEC80010ED016A17ED021A57ED010A11ED044A27
:10DED80011ED035A52ED044A52ED035A12ED027A3B
:10DEE80052ED017A51ED021A11ED010A73EE238AFF
:10DEF80032EE228A47ED048A07ED038A71EE268AFC
:10DF080030EE868A47ED028A07ED018A74EE848A2C
:10DF180035EE858A42ED048A02ED038A77EE218A7E
:10DF280037EE808A42ED028A02ED018A73EE633A87
:10DF380075EE655A1EED035A32EE623A74EE644A83
:10DF480025EE638A1EED044A23EE052A64EE652A4F
:10DF5800A3EE048A1032944524EE843AA3EE842A70
:10DF680007F110070EF1100EA5EE853A00F110002A
:10DF780001F11001E4EE852A00ED078A00ED082A78
:10DF880001ED073A41ED082A5EED055A1EED065AE5
:10DF980071EE666A30EEC66A31EEC77A70EE677A5D
:10DFA80026EE253A65EEE63A25EE674A67EE054A1B
:10DFB800E6EE053AA6EE853AA7EE254AE7EEA54A2B
:10DFC80000ED063A40ED053A01ED064A41ED054AF5
:10DFD8007FF46CAF1FFA89F91A464946784820F051
:10DFE80053FB72684946284620F04EFB029B1A787C
:10DFF800142A7FF4C0AEB6E66F4E7148B268B18994
:10E0080025F08CF9029B93F800E0BEF1140F01F0A3
:10E01800EB84D4F814510135C4F814514EE6DFF8F6
:10E02800B89199F800108F0801F00386654E07F142
:10E0380001084FEA481806EB080C06F12002A6F181
:10E04800700012ED076A52ED056A12ED037A52ED7F
:10E05800017A52ED025A12ED084A52ED064A12EDC3
:10E06800045A26EE066A66EEA66A27EE077A67EE77
:10E07800A77AA4EE046A20329445E4EEA46A00F17B
:10E088001000A5EE057AE5EEA57AF1EEC65AB1EED6
:10E09800E66AF1EEC76AB1EEE77A40ED085A00ED9C
:10E0A800076A40ED066A00ED057ACAD1A8F1200298
:10E0B800324404EB071711F0030018BF08320FD0E1
:10E0C80052ED017A12ED027A67EEA77A0138E7EE8F
:10E0D800077A02F10802B1EEE77AA7EC017AEFD1EC
:10E0E800BEF1140F01F06D840135C4F81451FEF728
:10E0F800D1BCD4F8185134493448354BEA0011449E
:10E1080015448A88196800EE102A643AC82AA8BFFC
:10E11800C822782AB8BF782207EE902AB8EEC07ACB
:10E12800F8EEE77A00EB850577EE670A77EE876AFF
:10E1380067EE877A20EEA67AB8EE400AC7EE870A1D
:10E148002846D5F81490D5F81880EF692E6A20F083
:10E158007BFD029BC5F8149093F800E0C5F8188081
:10E16800BEF1140FEF612E6201F01E84D4F818215D
:10E17800184BD4F81451013283FB0213A3EBE2735A
:10E1880003EB4303D31A0135C4F81831C4F814510A
:10E19800F7E5F7F717F9029B039093F800E0BEF153
:10E1A800140F05BFDFF83480D4F81451D4F8145193
:10E1B800A8F80050FDF75FB878390020E024002067
:10E1C800D024002050250020683C002094540020D2
:10E1D800005500205655555572390020E04A002058
:10E1E800306E99BC2716983DA40DC93F843459BE9A
:10E1F800DB0F4940D06D393A00000000F0EEE76AC5
:10E20800B7EE005A35EE665A1FED0B4A5FED0B5A12
:10E218001FED0A6A1FED0C7A94ED6B0AF1EEC54A00
:10E22800E6EE845AF5EEC07AA6EEA56AF1EE10FA8B
:10E23800A6EE867A48BF5FED127A27EE247A48BFA9
:10E2480037EEC77A27EE000A26F042FAB0F5617F6A
:10E2580000F3A28607EE900AF8EEE76A5FED1B7AF4
:10E2680066EEA76A07EE906ABDEEE67AF8EEE77A00
:10E2780017EE103A2033402B41F295841FED220A05
:10E2880026F026FA00B207EE900AB8EEE77AFFF712
:10E29800C0BAC14A02F1500503E00432954200F0C9
:10E2A800C5821378262BF8D19678D3789E42F4D27B
:10E2B800FFF7F1BAB94823F08FFAFEF7F1BCB84876
:10E2C80023F08AFAFEF7E6BCB64823F085FAFEF793
:10E2D800EDBCB54DB54F95ED004A95ED057AD5EDF8
:10E2E800014A95ED066AD5ED046A95ED035AD5ED18
:10E2F800025A67EE897A07EB8602A4EE277AA4EE23
:10E30800A76A66EEC76AA5EE476AE5EEA76A20EE39
:10E31800070A85ED056AC5ED066A82ED007A29EEE1
:10E32800088A26F0D5F969EE288AD5ED0E5AD5ED7A
:10E33800176A95ED091AD5ED121A95ED0F5A95ED54
:10E34800187A95ED0A2AD5ED132A95ED0D6AD5EDC3
:10E35800167A95ED0C3AD5ED0B3A95ED154AD5EDB3
:10E36800144AE1EE085A002207EB8601E8EEA16A9A
:10E3780000B2C4F80021A2EE085AC4F80421C4F877
:10E388000821A8EEA27A26EE656A67EEE67AA3EE81
:10E39800655AA3EE886AA6EEC47AE8EEA47A85EDFB
:10E3A8000E5AC1ED205A85ED0F6AC1ED406A85ED20
:10E3B800177AC5ED187AFEF727BBD4F89C51049B51
:10E3C8005D1BFEF727BABBF93820CBF8201007EE03
:10E3D800902A0121F8EEE77ACBF86020CBF87C1080
:10E3E8000022012FCBED1C7ACBED1B7ACBF87420E1
:10E3F80001F06B82AF427CF4A2AFBBF93A20CBF8B4
:10E40800642007EE902A00210122F8EEE77ACBF883
:10E418002410CBF890200022012FCBED217ACBEDF0
:10E42800207ACBF8882001F05482AF427CF4BBAF4D
:10E43800BBF93C20CBF8682007EE902A0021012286
:10E44800F8EEE77ACBF82810CBF8A4200022012FA9
:10E45800CBED267ACBED257ACBF89C207CF4D7AF90
:10E468009FED538A032E49D04CB107EE904AF8EE3F
:10E47800E77AF4EEC87AF1EE10FA01F1DF834D4A3B
:10E488004D4C1168DBF86820A8F8060094F82001C4
:10E4980002EB550292FBF5F50022CBF828508A6270
:10E4A8000A63CA6228B1454A126832F480637CF470
:10E4B800B1AF434A126812F4003241F0FE8141487C
:10E4C8001146835C012B02F10C0200F092830131AA
:10E4D8001829F6D1FCF79EBF3B494B69002B3DF448
:10E4E8007EA83A483A4B008893FBF0F00B684FF04F
:10E4F800010E186081F811E0FDF771B8B0EE480A16
:10E5080026F0E6F800B2AFE723690622652BA27071
:10E5180034D92278032A14BF6FF0FF026FF07F020C
:10E52800A3F1650303EA020303F1010314BF4FF4E7
:10E53800807280229A42236120D23A68E7680232C8
:10E5480003EB0708904581F04984224A6760D16F40
:10E55800C4F80880490203FB01F30521176042F85B
:10E568001C3C42F8183CA170A2681B49012024F009
:10E5780015FB012841F028840623A37000211748C1
:10E5880023F02CFF012841F01F84A3780133DBB26C
:10E59800A370FFF762B900BF9035002070770020A4
:10E5A80084780020B4770020FC3B002090390020BC
:10E5B800000000004C660020D0240020DC6400200D
:10E5C800D04300204475030890850020A8850020CA
:10E5D80020A1070060780020D06600203C78002049
:10E5E8002278237DAF4FDFF8FC92032A14BF4FF443
:10E5F80080784FF08008002B42D0012BFBD1AA4B2A
:10E6080062681968386800234FEA412E4FF0FF31DD
:10E61800B1FBFEF112EB010B43F1000C0021614547
:10E6280000F1020008BF584538BF83465A469F4943
:10E63800022012F023FE032801F26B8101A353F894
:10E6480020F000BF03C600085DE6000803C6000806
:10E658005DE600086268A3682669991AB14284BF1A
:10E66800E260216103283FF44FAF0133B3FBF8F2B6
:10E6780008FB12320AB143449B1A002263602275D8
:10E688003A6849460232002012F0F8FD032801F2E8
:10E69800408101A353F820F003C6000851E70008A1
:10E6A80003C6000811E5000841F27013E35C002B73
:10E6B8003DF4A3AF7E4823F08FF8FDF79EBF7D4B56
:10E6C80000930320A070302305227B49784824F06A
:10E6D80039FCFDF792BF03236370FDF78EBF00235B
:10E6E8000AAE31461846092212F088FC01287DF44A
:10E6F80084AF0A9B93F8FE21552A01F0128141F25A
:10E70800B41202210123A1546370FDF776BF0AAE4B
:10E7180041F2FC173146E0590023092212F06EFC41
:10E7280001287DF46AAF00230A9A2370B2F80B30EF
:10E73800B3F5007F01F0E38241F2B4120321012313
:10E74800A1546370FDF759BF636884F814A00133BE
:10E75800A36054E7594A5A4DD2ED006A594A95EDDB
:10E76800006A1278C4ED646A84ED656A002A00F0D4
:10E77800238276EE665A94F99821C4ED615A0132E3
:10E78800C4ED626A00F08A85049BC4F89C310025B8
:10E7980037EE677AFCEEE77A4B4E84ED687A17EE2F
:10E7A800902AA4F88C21FF2296ED005A84F898212B
:10E7B800FEF740B8DFED457A454B94ED687AC3ED36
:10E7C800007AC3ED017AC3ED027A424BF0EE674A54
:10E7D800F0EE673A1968FDF7FDB83F4B1D7805F074
:10E7E800010CFDF794BC3D49DFED3D7A0968C4EDA5
:10E7F8004C7A11F0805840F0C383DAF8001011F415
:10E80800800800F0EC814FF00008B6EE007A67EE61
:10E81800877AF4EEE57AF1EE10FAC8BFF0EE675A9F
:10E8280040F3AE83C4ED685AFDF71DBB234A244D5F
:10E83800D2ED007A234A95ED007A1278C4ED647A15
:10E8480084ED657A002A00F0318377EE676A94F9DF
:10E858009821C4ED616A0132C4ED627A00F05A86EB
:10E86800049BC4F89C3100259FED187A164E84ED60
:10E87800687AFF2296ED005A84F89821FDF7DABFEE
:10E8880073EEE77AB7EE007AF4EEC77AF1EE10FA93
:10E89800C4ED4C7A41F3278084EEA77A8DED0A7A8D
:10E8A800FDF7D7BAD4780020DC780020D4660020A1
:10E8B8003C7800203D210308008603084C3D0020D9
:10E8C80078470020345700208C47002000000000C3
:10E8D800FC380020E4640020484B0020A43E0020BF
:10E8E80000000080D0660020002F00F0CD8625EEC5
:10E8F800866ACC48A5EE076AB0EE675AA6EE265A95
:10E90800BDEEC56A16EE10CA16EE107AF445A8BF19
:10E9180077466145C8BF0F4606EE107AB8EEC66A5C
:10E92800012A80ED006A3DF4F6AB95ED046A9DED91
:10E938000B5A25EE866AA5EE076AB0EE675AA6EE70
:10E94800265ABDEEC56A16EE10CA16EE107AF445C0
:10E95800A8BF77466145C8BF0F4606EE107AB8EEE5
:10E96800C66A022A80ED016A3DF4D5AB95ED086AC6
:10E978009DED0C5A25EE866AA5EE076AB0EE675A39
:10E98800A6EE265ABDEEC56A16EE10CA16EE107A25
:10E99800F445A8BF77466145C8BF0F4606EE107A12
:10E9A800B8EEC66A032A80ED026A3DF4B4AB95ED71
:10E9B8000C6A9DED0D5A25EE866AA5EE076AB0EE43
:10E9C800675AA6EE265ABDEEC56A16EE10CA16EEAE
:10E9D800107AF445A8BF77466145C8BF0F4606EED2
:10E9E800107AB8EEC66A042A80ED036A3DF493AB48
:10E9F80095ED106A9DED0E5A25EE866AA5EE076A1A
:10EA0800B0EE675AA6EE265ABDEEC56A16EE10CAD3
:10EA180016EE107AF445A8BF77466145C8BF0F4681
:10EA280006EE107AB8EEC66A052A80ED046A3DF44F
:10EA380072AB95ED146A9DED0F5A25EE866AA5EE28
:10EA4800076AB0EE675AA6EE265ABDEEC56A16EEFC
:10EA580010CA16EE107AF445A8BF77466145C8BFBC
:10EA68000F4606EE107AB8EEC66A062A80ED056AE9
:10EA78003DF451AB95ED186A9DED105A25EE866A66
:10EA8800A5EE076AB0EE675AA6EE265ABDEEC56A2D
:10EA980016EE10CA16EE107AF445A8BF77466145FF
:10EAA800C8BF0F4606EE107AB8EEC66A072A80ED90
:10EAB800066A3DF430AB95ED1C6A9DED115A65EE82
:10EAC800865AE5EE075AE6EEA57AFDEEE77A17EEE6
:10EAD800902A9645A8BF96468A42A8BF714607EE77
:10EAE800901AF8EEE77AC0ED077AFDF714BBBEF18D
:10EAF800010F7FF7B5AC07EE103AB8EEC77AC7EE4C
:10EB0800876AB1EEE68AADE4BEF1010F40F3E18613
:10EB180007EE103AB8EEC77AC7EE876AB1EEE68A12
:10EB2800032E13D04CB107EE904AF8EEE77AF4EED4
:10EB3800C87AF1EE10FA01F18180DBF8642002EB6B
:10EB4800550292FBF5F2CBF824206EE4B0EE480AA9
:10EB580025F0BEFD00B2E5E7BEF1010F40F3B58632
:10EB680007EE103AB8EEC77AC7EE876AB1EEE68AC2
:10EB7800032E13D04CB107EE904AF8EEE77AF4EE84
:10EB8800C87AF1EE10FA01F15980DBF8602002EB47
:10EB9800550292FBF5F2CBF820202BE4B0EE480AA0
:10EBA80025F096FD00B2E5E7F7EE006AFDF7FCBC3C
:10EBB800F7EE006AFDF77EBC76EEC65AF0EE466ABE
:10EBC800D9E58222FDF7E4BFDFED177AFDF7ACBF88
:10EBD800164BD3F800E0BEF93270FEF792BAB6EEE3
:10EBE800007AF4EEC75AF1EE10FA3FF70EAEFDF7D1
:10EBF8003AB9D4F824614A003EB1551800EB8505AE
:10EC080076786D78B542BCF405AC0A4400EB820016
:10EC18000022C4F82401A4F80C22C4F81022FCF73E
:10EC2800F9BB00BF2439002000000243E46400203F
:10EC380095ED006A9DED0A4AE44825EE866AFDEEE8
:10EC4800E43AA4EE076AB0EE674AA6EE264A13EE47
:10EC5800901AB4EEC45AF1EE10FAB0EE446A88BFC6
:10EC6800B0EE646ABDEEC66A16EE108A16EE107A29
:10EC7800F045A8BF77464145C8BF0F4606EE107A53
:10EC8800B8EEC66A012A80ED006A3DF440AA95ED07
:10EC9800046A9DED0B4A25EE866AA4EE076AB0EE7B
:10ECA800674AA6EE264AB4EEC45AF1EE10FAB0EE60
:10ECB800446A88BFB0EE646ABDEEC66A16EE108A72
:10ECC80016EE107AF045A8BF77468845B8BF0F46BC
:10ECD80006EE107AB8EEC66A022A80ED016A3DF4A3
:10ECE80016AA95ED086A9DED0C4A25EE866AA4EEF3
:10ECF800076AB0EE674AA6EE264AB4EEC45AF1EEA9
:10ED080010FAB0EE446A88BFB0EE646ABDEEC66A17
:10ED180016EE108A16EE107AF045A8BF7746884599
:10ED2800B8BF0F4606EE107AB8EEC66A032A80ED21
:10ED3800026A3DF4ECA995ED0C6A9DED0D4A25EEAD
:10ED4800866AA4EE076AB0EE674AA6EE264AB4EED3
:10ED5800C45AF1EE10FAB0EE446A88BFB0EE646AA5
:10ED6800BDEEC66A16EE108A16EE107AF045A8BFF8
:10ED780077468845B8BF0F4606EE107AB8EEC66AE1
:10ED8800042A80ED036A3DF4C2A995ED106A9DED51
:10ED98000E4A25EE866AA4EE076AB0EE674AA6EE2A
:10EDA800264AB4EEC45AF1EE10FAB0EE446A88BFAF
:10EDB800B0EE646ABDEEC66A16EE108A16EE107AD8
:10EDC800F045A8BF77468845B8BF0F4606EE107ACB
:10EDD800B8EEC66A052A80ED046A3DF498A995ED57
:10EDE800146A9DED0F4A25EE866AA4EE076AB0EE16
:10EDF800674AA6EE264AB4EEC45AF1EE10FAB0EE0F
:10EE0800446A88BFB0EE646ABDEEC66A16EE108A20
:10EE180016EE107AF045A8BF77468845B8BF0F466A
:10EE280006EE107AB8EEC66A062A80ED056A3DF449
:10EE38006EA995ED186A9DED104A25EE866AA4EE36
:10EE4800076AB0EE674AA6EE264AB4EEC45AF1EE57
:10EE580010FAB0EE446A88BFB0EE646ABDEEC66AC6
:10EE680016EE108A16EE107AF045A8BF7746884548
:10EE7800B8BF0F4606EE107AB8EEC66A072A80EDCC
:10EE8800066A3DF444A995ED1C6A9DED114A65EEAC
:10EE9800865AE7EE045AE6EEA57AB4EEE75AF1EEA2
:10EEA80010FAC8BFF0EE647AFDF721B977EEC76AA9
:10EEB800F0EE477ACBE4BEF834309FED457A07EEA2
:10EEC800903AF8EEE77A434B67EE877AC3ED007A1B
:10EED800FDF76FB9404A4FEA89065FEA9C0900EBE3
:10EEE800060802EBC313264400F0FE8609F1010967
:10EEF8004FEA091903EB090703F1100208F11000A2
:10EF080006F1100112ED024A12ED035A12ED016AE0
:10EF180012ED047A50ED024A50ED035A50ED016AA1
:10EF280050ED047A64EE244A65EE255A66EE266AA8
:10EF380067EE277A1032974241ED024A41ED035AB3
:10EF480041ED016A41ED047A00F1100001F1100170
:10EF5800D8D1A9F110094B4408EB09004E441CF024
:10EF6800030C3EF464AFB3EC017AF0EC017A67EE7F
:10EF7800277ABCF1010CE6EC017AF4D1FEF757BF11
:10EF8800B7EE007A77EE677AF4EEE75AF1EE10FA08
:10EF980088BFF0EE675A45E407EE906ADFED0F6A26
:10EFA800F8EEE77A66EEA65A9FED0D5A9FED0D6AC8
:10EFB8009FED0D7AA5EE856A26EEA55AA5EE867A0E
:10EFC800E5EE076A26EEA70AFFF75AB924390020AA
:10EFD8006F12833A180000209039002084F9223FEC
:10EFE80092E741B99730083C15A82ABE95ED006A0A
:10EFF8009DED0A4AAE4825EE866AFDEEE43AA4EE97
:10F00800076AB0EE674AA6EE264A13EE907AB4EE87
:10F01800C45AF1EE10FAB0EE446A88BFB0EE646AE2
:10F02800BDEEC66A16EE10CA16EE101AF445A8BF51
:10F0380071466745C8BF394606EE101AB8EEC66A6B
:10F04800012A80ED006A3DF49FAF95ED046A9DEDBD
:10F058000B4A25EE866AA4EE076AB0EE674AA6EE6A
:10F06800264AB4EEC45AF1EE10FAB0EE446A88BFEC
:10F07800B0EE646ABDEEC66A16EE10CA16EE101A35
:10F08800F445A8BF7146BC45B8BF394606EE101A0C
:10F09800B8EEC66A022A80ED016A3DF475AF95EDB7
:10F0A800086A9DED0C4A25EE866AA4EE076AB0EE62
:10F0B800674AA6EE264AB4EEC45AF1EE10FAB0EE4C
:10F0C800446A88BFB0EE646ABDEEC66A16EE10CA1E
:10F0D80016EE101AF445A8BF7146BC45B8BF3946AC
:10F0E80006EE101AB8EEC66A032A80ED026A3DF4ED
:10F0F8004BAF95ED0C6A9DED0D4A25EE866AA4EEA0
:10F10800076AB0EE674AA6EE264AB4EEC45AF1EE94
:10F1180010FAB0EE446A88BFB0EE646ABDEEC66A03
:10F1280016EE10CA16EE101AF445A8BF7146BC4573
:10F13800B8BF394606EE101AB8EEC66A042A80ED42
:10F14800036A3DF421AF95ED106A9DED0E4A25EE58
:10F15800866AA4EE076AB0EE674AA6EE264AB4EEBF
:10F16800C45AF1EE10FAB0EE446A88BFB0EE646A91
:10F17800BDEEC66A16EE10CA16EE101AF445A8BF00
:10F188007146BC45B8BF394606EE101AB8EEC66AD5
:10F19800052A80ED046A3DF4F7AE95ED146A9DEDFD
:10F1A8000F4A25EE866AA4EE076AB0EE674AA6EE15
:10F1B800264AB4EEC45AF1EE10FAB0EE446A88BF9B
:10F1C800B0EE646ABDEEC66A16EE10CA16EE101AE4
:10F1D800F445A8BF7146BC45B8BF394606EE101ABB
:10F1E800B8EEC66A062A80ED056A3DF4CDAE95ED07
:10F1F800186A9DED104A25EE866AA4EE076AB0EEFD
:10F20800674AA6EE264AB4EEC45AF1EE10FAB0EEFA
:10F21800446A88BFB0EE646ABDEEC66A16EE10CACC
:10F2280016EE101AF445A8BF7146BC45B8BF39465A
:10F2380006EE101AB8EEC66A072A80ED066A3DF493
:10F24800A3AE95ED1C6A9DED114A65EE865AE7EE70
:10F25800045AE6EEA57AB4EEE75AF1EE10FAC8BF02
:10F26800F0EE647AFDEEE77A17EE901A8E45A8BFA5
:10F278008E468F42D8BF774607EE907AF8EEE77A47
:10F28800C0ED077AFDF77DBE0A494A69002A3CF4B9
:10F298008FAA0A6813604B74FCF78ABAD4F89C5199
:10F2A800049B5D1BFFF774BA034EFCF7F9BF00BF60
:10F2B8002439002090850020004C0020002F00F009
:10F2C800AC83E04D9DED0A4A95ED006A25EE866A0D
:10F2D800A4EE076AB0EE674AA6EE264AB0EE446A84
:10F2E80033B1B4EE445AF1EE10FAC8BFB0EE646A16
:10F2F800FDEEE44ABDEEC66A14EE907A16EE101AD8
:10F308008F4214EE90CA00F3F2847145A8BF71468B
:10F3180006EE101ACC48B8EEC66A012A80ED006ADB
:10F328003CF4F9AE95ED046ADDED0B4A25EE866AEC
:10F33800A4EE876AF0EE674AE6EE264AB0EE646A03
:10F34800002B00F0BB84B4EEE45AF1EE10FA40F35F
:10F35800B58439467145A8BF714606EE101AB8EE55
:10F36800C66A022A80ED016A3CF4D5AE95ED086ABA
:10F37800DDED0C4A25EE866AA4EE876AF0EE674A50
:10F38800E6EE264AB0EE646A002B00F08D84B4EEF7
:10F39800E45AF1EE10FA40F3878439467145A8BF64
:10F3A800714606EE101AB8EEC66A032A80ED026AA4
:10F3B8003CF4B1AE95ED0C6ADDED0D4A25EE866A9A
:10F3C800A4EE876AF0EE674AE6EE264AB0EE646A73
:10F3D800002B00F05F84B4EEE45AF1EE10FA40F32B
:10F3E800598439467145A8BF714606EE101AB8EE21
:10F3F800C66A042A80ED036A3CF48DAE95ED106A66
:10F40800DDED0E4A25EE866AA4EE876AF0EE674ABD
:10F41800E6EE264AB0EE646A002B00F03184B4EEC2
:10F42800E45AF1EE10FA40F32B8439467145A8BF2F
:10F43800714606EE101AB8EEC66A052A80ED046A0F
:10F448003CF469AE95ED146ADDED0F4A25EE866A47
:10F45800A4EE876AF0EE674AE6EE264AB0EE646AE2
:10F46800002B00F00384B4EEE45AF1EE10FA40F3F6
:10F47800FD8339467145A8BF714606EE101AB8EEED
:10F48800C66A062A80ED056A3CF445AE95ED186A11
:10F49800DDED104A25EE866AA4EE876AF0EE674A2B
:10F4A800E6EE264AB0EE646A002B00F0D683B4EE8E
:10F4B800E45AF1EE10FA40F3D08339467145A8BFFB
:10F4C800714606EE101AB8EEC66A072A80ED066A7B
:10F4D8003CF421AE95ED1C6ADDED114A65EE865AC5
:10F4E800E4EE875AE5EEA67A002B00F0AE83F4EE40
:10F4F800C57AF1EE10FA40F1A8833A467245A8BFE2
:10F508007246944607EE90CAF8EEE77AC0ED077A9D
:10F51800FCF701BED4F89C51049B5D1BFFF7A4B90E
:10F5280096ED000A0593039225F0D2F84749DFF8D3
:10F5380050E1D1F8EC10DFF84CC1039AACF80000A8
:10F548008EFB013EC917C1EBAE1107EE901AF8EE1B
:10F55800E77A059BFDEEE77A17EE901AACF80210F1
:10F56800FCF7A3BE07EE906ADFED396A9FED397AA2
:10F5780084F80462F8EEE77A67EEA67A77EE876A8F
:10F58800BDEEE66A16EE103A2033402B40F2B58203
:10F59800DFED316A314BBDEEE77AC3ED016A17EE54
:10F5A800103A2033402B00F2EF829FED2D7AF4EED3
:10F5B800C77AF1EE10FA40F32384DFED2A5A9FED63
:10F5C8002A6A01E0F0EE477AF4EEC67AF1EE10FA14
:10F5D80037EEE57AF6DCDFED257AB4EEE77AF1EE80
:10F5E80010FA40F10A84DFED1F5A9FED216A01E00D
:10F5F800B0EE677AB4EEC67AF1EE10FA77EE257AB5
:10F60800F6D49FED147AF4EEC77AF1EE10FA40F3CF
:10F61800BE829FED137A77EE677A67EEA75A9FED61
:10F62800155A9FED156A9FED157AA5EE856A27EEA6
:10F63800A55AA5EE867AE5EE077AC4ED827AFDF73B
:10F64800C1BD00BFF4460020243900205801002025
:10F6580035FA8E3CDB0FC93F00000000180000207F
:10F66800DB0F4940DB0FC940E4CB1641DB0F49C033
:10F67800E4CB16C192E741B99730083C15A82ABED9
:10F68800D34D6210E04A002025EE866AA5EE076A8F
:10F69800B0EE675AA6EE265ABDEEC56A16EE100AF7
:10F6A800814200F3B0817045A8BF704606EE100A8B
:10F6B800B8EEC66AB8F1000F00F0CF83DE48012A21
:10F6C80080ED006A3CF427AD95ED046A9DED0B5A78
:10F6D80025EE866AA5EE076AB0EE675AA6EE265AA8
:10F6E800BDEEC56A16EE107AB94200F38A817745F5
:10F6F800A8BF774606EE107AB8EEC66AB8F1000FD2
:10F7080000F0F283022A80ED016A3CF404AD95ED25
:10F71800086A9DED0C5A25EE866AA5EE076AB0EEDA
:10F72800675AA6EE265ABDEEC56A16EE107AB94299
:10F7380000F371817745A8BF774606EE107AB8EED8
:10F74800C66AB8F1000F00F0F083032A80ED026A60
:10F758003CF4E1AC95ED0C6A9DED0D5A25EE866AF8
:10F76800A5EE076AB0EE675AA6EE265ABDEEC56A40
:10F7780016EE107AB94200F34C817745A8BF774658
:10F7880006EE107AB8EEC66AB8F1000F00F0C28330
:10F79800042A80ED036A3CF4BEAC95ED106A9DED39
:10F7A8000E5A25EE866AA5EE076AB0EE675AA6EEEF
:10F7B800265ABDEEC56A16EE107AB94200F32781C3
:10F7C8007745A8BF774606EE107AB8EEC66AB8F154
:10F7D800000F00F09483052A80ED046A3CF49BAC8A
:10F7E80095ED146A9DED0F5A25EE866AA5EE076A17
:10F7F800B0EE675AA6EE265ABDEEC56A16EE107A26
:10F80800B94200F302817745A8BF774606EE107A21
:10F81800B8EEC66AB8F1000F00F01483062A80ED2E
:10F82800056A3CF478AC95ED186A9DED105A25EE02
:10F83800866AA5EE076AB0EE675AA6EE265ABDEEAE
:10F84800C56A16EE107AB94200F3CC807745A8BF96
:10F85800774606EE107AB8EEC66AB8F1000F00F0E7
:10F868000783072A80ED066A3CF455AC95ED1C6ABF
:10F878009DED115A65EE865AE7EE055AE5EEA67A31
:10F88800FDEEE77A17EE902A914203DC7245A8BF95
:10F898007246114607EE901AF8EEE77AB8F1000FB3
:10F8A8007FF434AE089B002B7FF430AE059B079A9B
:10F8B8009342B8BFF0EE647A28E6604A1278032AC9
:10F8C80000F019820022FEF7FABD9FED668AFFF765
:10F8D8004FB99FED648AFFF723B9D4F89C51049B74
:10F8E8005D1BFDF7F5BF5649096811F080587EF495
:10F8F8008CAFFEF782BF9FED530ADFF8588125EEE3
:10F90800800A24F0E5FED4F81451A8F80600FDF7A3
:10F9180052B9237DFEF76FBE4B484C498046FEF72F
:10F9280075BA93F8FF21AA2A7EF4E9AED3F8C61176
:10F9380049B193F8C221A2F10B0001282DD902F098
:10F94800F702062A29D0D3F8D61149B193F8D22163
:10F95800A2F10B00012820D902F0F702062A1CD0D8
:10F96800D3F8E61149B193F8E221A2F10B0001287E
:10F9780013D902F0F702062A0FD0D3F8F61100299E
:10F988003EF4BDAE93F8F231A3F10B02012A04D97B
:10F9980003F0F703062B7EF4B2AE41F2FC1201230A
:10F9A800A150A370FEF7B4BEF5F70CFD029BDFF87B
:10F9B800A48093F800E0039BC01AA8F80200FEF7A1
:10F9C800D5BBF5F7FFFC029BDFF8888093F800E0D1
:10F9D800039B99F80010D4F81451C01AA8F8040031
:10F9E800FEF782BB0F4634E7F5F7ECFC029BDFF825
:10F9F800648093F800E0039BC01AA8F80200FEF7A1
:10FA080008BB0F4676E6084650E60F46FEE60F4668
:10FA1800D9E60F46B4E60F468FE60AA9BDEEE46ABA
:10FA280001EB820294460A48034D09941A4616EEE1
:10FA3800107A43462CE000BF24390020785B002070
:10FA4800A43E00200000C842103B0020D024002023
:10FA5800F4460020E04A002092E741B99730083C7C
:10FA680015A82ABE00000000E4CB1641DB0FC940F0
:10FA7800E4CB16C1DB0FC93FDB0F4940DB0FC9BF21
:10FA8800DB0F49C06145A5EC016A00F1100031D0D7
:10FA980090ED006AB1EC014A25EE866AA7EE046A89
:10FAA800B0EE674AA6EE864AB0EE446A32B1B4EECA
:10FAB800445AF1EE10FAC8BFB0EE646ABDEEC66AE9
:10FAC80016EE108A474506EE107A04DCF045A8BF0A
:10FAD800F04606EE108AB8EEC66A002BD2D1089C12
:10FAE800002CCFD1059CA046079CA045B8BFB0EE1E
:10FAF800646AC7E7099CFCF70EBBF4EEC77AF1EE1F
:10FB080010FA40F381815FED275A1FED296A01E061
:10FB1800F0EE476AF4EEC66AF1EE10FA36EEE57AD0
:10FB2800F6DC5FED296AB4EEE67AF1EE10FA40F100
:10FB380061815FED325A1FED326A01E0B0EE667AFC
:10FB4800B4EEC67AF1EE10FA77EE256AF6D41FED18
:10FB5800377AF4EEC76AF1EE10FA40F3B9801FED78
:10FB68003A7A77EE666A66EEA65A1FED455A1FED99
:10FB7800456A1FED457AA5EE856A26EEA55AA5EEDB
:10FB8800867AE5EE076A05E55FED4A7A55E51FEDE9
:10FB9800457AF4EEC77AF1EE10FA44BF1FED487AC1
:10FBA80077EE677A39E51FED4C7AF4EEC76AF1EE25
:10FBB80010FA40F328825FED535A1FED556A01E0B1
:10FBC800F0EE476AF4EEC66AF1EE10FA36EEE57A20
:10FBD800F6DC5FED556AB4EEE67AF1EE10FA40F124
:10FBE8007A815FED5E5A1FED5E6A01E0B0EE667ADB
:10FBF800B4EEC67AF1EE10FA77EE256AF6D41FED68
:10FC0800637AF4EEC76AF1EE10FA05DD1FED667A45
:10FC180077EE666AFFF7C6B91FED687AF4EEC76A31
:10FC2800F1EE10FA44BF1FED6A7A77EE666AFFF7C5
:10FC3800B9B9C54F07F18002FEF73DBAA8F806002A
:10FC4800ABF8A850C04CFBF7ECBBFDEEE77A17EE1B
:10FC5800902ABA42FFF656AC50E4BDEEC66A16EEDC
:10FC6800101AB942BFF62AAC39462AE4BDEEC66A74
:10FC780016EE101AB942BFF6FDAB3946FFF7FDBBC9
:10FC8800BDEEC66A16EE101AB942BFF6CFAB3946BA
:10FC9800FFF7CFBBBDEEC66A16EE101AB942BFF623
:10FCA800A1AB3946FFF7A1BBBDEEC66A16EE101A26
:10FCB800B942BFF673AB3946FFF773BBBDEEC66AF0
:10FCC80016EE101AB942BFF645AB3946FFF745BBE9
:10FCD8009FED9E7AF4EEC76AF1EE10FA44BF9FEDED
:10FCE8009C7A77EE666A3EE74046FFF738B914EE2D
:10FCF800901AFFF70DBB21F051F9FBF78BBB137C72
:10FD0800022B7EF419AD92F8FE31552B7EF414AD1A
:10FD180092F8FF31AA2B7EF40FADD689E7598D4BA7
:10FD280037441F6092F80DE041F210210EF1FF33C5
:10FD38007F2B44F801E03EF6FFACCEF100033EEA2B
:10FD480003037EF4F9AC4FEA4E2341F21821013B3C
:10FD58006350D08A00B9506A7F4941F20423E050C9
:10FD6800B2F811305B0103F2FF135B120B60B2F8BB
:10FD7800131001B9116A40001E440644891B41F260
:10FD8800082C40F6F476B1FBFEF1B14244F80C10B1
:10FD980040F235814FF6F476B14240F2D18003212A
:10FDA8002170D26A6D493B44184441F20C2641F255
:10FDB8001C230978A051E25009B924F083FAA378EA
:10FDC8000133A370FCF719BC02287CF416AC41F28D
:10FDD800B4120123A3546370FCF70FBC22F0C8F9D6
:10FDE8002369FEF7B2BB94F87831002B7BF4AEADF3
:10FDF800FBF799BDF0EE476AA9E6F0EE477A00E412
:10FE0800B0EE677AFFF7E7BBB0EE667A89E6132BA8
:10FE180005D1B0EE480A24F05BFC069B1880B0EED2
:10FE2800480ADBF808324E489847029B1B78132B88
:10FE3800B0EE408A7DF4EDA824F04AFC069B588079
:10FE4800FDF7E7B8089B002B7FF4E8AC059B079FFC
:10FE5800BB42B8BFB0EE646AE0E4089B002B7FF4B5
:10FE68002DAC059B07988342B8BFB0EE646A25E4C1
:10FE7800089B002B7FF4F5AC059B079FBB42B8BFDE
:10FE8800B0EE646AEDE4DFED377AB4EEE7EAF1EE5E
:10FE980010FA26DCDFED347AB4EEE7EAF1EE10FA78
:10FEA8001FD4324BD3ED007AB1EE677AF4EEC7DA9D
:10FEB800F1EE10FA12D4F4EEE7DAF1EE10FA88BF98
:10FEC800F0EE67DA2A4B87ED00CA1B689342BBF64F
:10FED80095ABFBF7F9BBF0EE476A90E6F0EE47DA30
:10FEE800F0E7DFED24DAEDE7089B002B7FF40AAC9E
:10FEF800059B079FBB42B8BFB0EE646A02E4089B4B
:10FF0800002B7FF468AC059B079FBB42B8BFB0EEDF
:10FF1800646A60E4089B002B7FF43AAC059B079F5A
:10FF2800BB42B8BFB0EE646A32E4089B002B7FF492
:10FF38000CAC059B079FBB42B8BFB0EE646A04E4F3
:10FF48000222227000222DE7D0240020DB0FC9BF37
:10FF5800DB0F49C0CC780020EC780020AC7800207A
:10FF68009454002000C0F84400C0F8C4E8460020BB
:10FF7800CC46002000000000244A254B10681B686E
:10FF88009847244BD7ED006A93ED007A224BD3EDC6
:10FF9800007A224B83ED020A214B67EE277A2B4425
:10FFA80027EEAC7AD3ED007A1E4B67EE277AF0EE97
:10FFB800665AEDEEA75A93ED006AB1EE467AB4EEB2
:10FFC800E57AF1EE10FA08DCF4EEC65AF1EE10FA12
:10FFD8008CBFB0EE467AB0EE657A134B1B78012BD6
:10FFE80002D0192B7BF41CACDFED107AF4EEE7DAC3
:08FFF800F1EE10FACCBF012369
:020000040801F1
:100000000023FBF71CBC01232370FEF799BBB0EE65
:10001000667AE2E56046002074460020B445002080
:1000200018000020F038002084460020EC46002014
:100030008C320020000096420C4B1B78DB0700D569
:1000400070470B490B68002BFAD04FF47A7202FB11
:1000500003F39842F4D3074B1B781BB9064B9A68FD
:100060001B69136000230B60704700BF484B0020E2
:10007000244D0020184D0020044D002008B50FF03D
:1000800057FE024B024ADA60FEE700BF00ED00E0D7
:100090000400FA05024A034B1278197817F004BCE1
:1000A000A8240020A92400209F4B1B7803B170478F
:1000B0002DE9F0439D4D2B688BB013B90BB0BDE813
:1000C000F0839B4E9B4A3378044601A8D75C14F01A
:1000D000B7FC736803F5C333A0339C4205D9032FE3
:1000E00068D8DFE807F0485C3F10934B1B78DB07CC
:1000F000E4D42B68002BE1D01B681B68002BDDD0FB
:1001000020469847DAE704AF384614F099FC97E8A0
:10011000070007AB03C39DF810101A80002974D1A3
:1001200008A817F06BFB0DF11E0017F07FFB384697
:100130000A2207A925F064FA7F4B1A78071C18BF1A
:10014000012702F001027D49337808787460013399
:1001500093FBF0F100FB11333370002AC9D0002F5C
:10016000C7D1ABE7DFF8D08198F8002012F0010288
:1001700051D00027E7E79DF80430DFF8BC8143B396
:1001800098F80030D9075CD56C4A337811787460E0
:10019000013393FBF1F201FB123333708EE704A8B5
:1001A00017F044FB0746002840D1634B1A7802F051
:1001B0000102C8E7604A61493378097810787460B1
:1001C0000133C00793FBF1F201FB1233337090D57A
:1001D00074E798F80030DA07D6D404A817F00EFBBD
:1001E000002840F0848055493378087898F800203A
:1001F0007460013302F0010293FBF0F100FB113354
:100200003370002A3FF475AF58E70DF11D0107A8C0
:1002100017F018FB87E707A817F0FCFA00284AD167
:1002200098F80020002702F001028CE707A814F0DC
:1002300007FC9DF81E009DF8103083422ED1002748
:10024000B3E704A90DF1030017F0FCFA0028CAD0A7
:1002500007A814F0F5FB9DF81C009DF803309DF8ED
:100260001D10834203D19DF810308B42BBD02B6808
:100270004BB11A79824206D35A798A4203D31B685A
:10028000DB6803B198472D4A3378117874600133E5
:1002900093FBF1F201FB123333702AE72B68002B3A
:1002A00083D09A79824280D31B681B69002B3FF46C
:1002B0007CAF984779E7272010F0BCFA0746002862
:1002C000AED01F4BDB88002BAAD1272010F056FAA6
:1002D0009DF81C308146E8B1002BA1D1012017F018
:1002E000BDFA98F800204F4602F001022BE707A85C
:1002F00014F0A6FBBDF82000BDF8103083423FF497
:1003000072AF2B68002BBED01B689B69002BBAD044
:100310009847B8E7002B83D017F0A0FA98F8002090
:1003200002F001020FE700BFA34100204C4B002068
:10033000E8260020E82F0020484B0020EC2F00206A
:10034000504B00202DE9F04F2DED028BA0F10A0358
:1003500089B00C46ED2B00F27686DFE813F022011F
:1003600074067406740674067406740674067406BD
:1003700074067406740674067406740674067406AD
:1003800074067406740674067406740674062F02E6
:100390007406740674062C067406740674069901B5
:1003A0007406560174063E01740633017406280271
:1003B000740603027406EF01740674067406EA01FB
:1003C000E4017406D20174067406CC017406A5011A
:1003D0007406740674068A04740674067406740639
:1003E0006C047406020174063B0629057406740643
:1003F00074067406740674067406FD047406CF044D
:1004000074069C047406650574066006740674061A
:10041000740674060503F105EA05B905EE007406D5
:1004200074062803A60274066F02E90274067406B5
:1004300074067406DE0274067406BD027406740641
:100440007406AF02F303BB037A03740674067406E2
:100450006C03740674064C03740674067406740602
:1004600074067406740674067406740674067406BC
:10047000740674067406050374067406740674061E
:10048000740674067406740674067406740674069C
:10049000740674067406740674067406740674068C
:1004A000740674067406740674067406740674067C
:1004B000740674067406740674067406740674066C
:1004C0003E03740674067406740674067406740695
:1004D000740674067406740674067406740674064C
:1004E000740674067406740674067406740674063C
:1004F000740674067406740674067406740674062C
:10050000740674067406740674067406740674061B
:10051000740674067406740674067406740674060B
:10052000740674067406740674066204380474064D
:1005300074067406740674060904AF4E337853B11A
:10054000AE4F002537F8021F2046F0F74BFE3378F8
:100550000135AB42F6DC012009B0BDEC028BBDE8F1
:10056000F08FA54E3378002BF5D0A54F0025B84667
:10057000236817F81520591C21601A7098F801108B
:1005800001EB810101EB810101F2EE2189B22046EC
:10059000F0F728FE33780135AB4208F10208E7DCBA
:1005A000D9E7984D284622F027FF0028D3DD2B46B7
:1005B0000544226813F8011B501C9D4220601170F5
:1005C000F7D1C8E7904D05F1800655F8041F204685
:1005D000F0F7F1FDAE42F8D1BDE78C4D05F14006D4
:1005E000B5F880102046F0F7FDFD236895F88220CD
:1005F000591C21601A70236895F883200435591C12
:10060000AE4221601A70EBD1A5E7814D0B682A7AC2
:10061000591C21601A70A98B2046F0F7E3FD298B45
:100620002046F0F7DFFD698B2046F0F7DBFD2368FD
:10063000EA7C591C21601A70A98C2046F0F7D2FD83
:10064000E98C2046F0F7CEFD2368AA7F591C216073
:100650001A70236895F82020591C21601A70698C43
:100660002046F0F7BFFD2368EA7A591C21601A7012
:10067000E9682046F0F79FFD23682A7C591C216019
:100680001A70236895F82120591C21601A7062E7BE
:100690000B68604A581C11782060197023685278E2
:1006A000591C21601A7056E70B685A4A5A4D117846
:1006B0005A4A581C2060197011682046F0F77BFDDB
:1006C0002368534A591C127A21601A7029882046DF
:1006D000F0F788FDA9882046F0F784FD2989204697
:1006E000F0F780FD20460021F0F77CFD2046002138
:1006F000F0F778FD2FE7084608224549F0F744FD5A
:1007000029E70B68464A474990785D1C25601870B8
:1007100023685278581C20601A7023680A79591C83
:1007200021601A7017E70B680122991821601A706E
:1007300011E708460021F0F73EFD0CE73A4D3B4E2D
:1007400005F1200795F90210394B93F906208A42EA
:1007500003F1080300F07A849E42F6D10835BD42C9
:10076000F0D1F8E6334B03F15A0522685979501C51
:100770002060117022681978501C20601170226866
:100780005978501C2060117022689978501C2060A4
:1007900011702268D978501C206011702268197974
:1007A0000633501C9D4220601170DED1D3E60B68E9
:1007B000174A591C527D21601A70CCE61E4D05F176
:1007C0005006287820F0F2FD2368027A591C216037
:1007D0001A7023686A78591C21601A702368AA78F5
:1007E000591C21601A702368EA780435591CAE42FE
:1007F00021601A70E5D1AEE6E05100204884002067
:100800009C36002046600020945B0020985B00200E
:100810005C8600205C390020A82F0020508E00202C
:10082000E43E0020AC24002088860020805A00206E
:10083000605A0020DC43002090350020AF4D0B684B
:100840002A68591C127821601A702B6822689978DE
:10085000531C2360002311702A6821681A44013355
:100860005279481C032B20600A70F5D123682A684E
:10087000591C127A21601A7023682A68591CD27890
:1008800021601A7023682A68591C127921601A7035
:100890002B6820465989F0F7A5FC2A682368527A0C
:1008A000591C21601A702A68F8E620460021F0F7EA
:1008B00082FC20460021F0F795FC4CE6904D08465E
:1008C0002988F0F78FFC69882046F0F78BFCA9880F
:1008D0002046F0F787FC3EE68A4D05F16006A988C0
:1008E0002046F0F77FFCE9882046F0F77BFC298959
:1008F0002046F0F777FC2368AA7A591C21601A7009
:100900002368EA7A591C21601A7055F80C1B20469E
:10091000F0F751FCAE42E2D11DE67B49522322683A
:10092000501C2060137011F8013F002BF7D112E624
:10093000764800232268056803EB4301561C6D5C72
:1009400026601570026825680A446E1C527826607D
:100950002A70026825680A4401339278691C0A2BC0
:1009600021602A70E6D1F6E500258146DFF8C881CE
:10097000DFF8C8B1049503950595069501214FF65A
:10098000FF7A05E001350B2D00F07E8318F9011F79
:100990004F1C4AFA05F3F5D0DE07F3D5BBF800305B
:1009A0002B41D807EED505A8F0F792FFEAE7584D9E
:1009B00008462988F0F716FC69882046F0F712FCF3
:1009C000B5F90430534AD91782FB0323C1EBA301C5
:1009D000204689B2F0F706FCBDE50B684E4A591C6B
:1009E0001278216005A81A70F0F7F4FA23685A1CEF
:1009F00022601870AFE50B68484F591C3A782160A7
:100A00001A703B78002B3FF4A6AD0025EEB23046BD
:100A100014F0EAF823684278591C216030461A70B5
:100A200014F0E2F801892046F0F7DCFB3B78013551
:100A3000AB42EBDC8FE53A4D0846298AF0F7D2FB52
:100A4000698A2046F0F7CEFBA98A2046F0F7CAFB58
:100A500081E5DFF8ECE00027FEB271460023226852
:100A6000501C206016702268501C20601370226891
:100A700011F8010F0133551C062B25601070EED1C3
:100A80000137062F0EF1060EE6D126490023226813
:100A9000501C206017702268501C20601370226860
:100AA00011F8010F0133551C0B2B25601070EED18E
:100AB00023681D4A581C07212060197023680021F3
:100AC000581C20601970236892F8F020591C21608E
:100AD0001A7040E50B68154A15491078154A5D1CD7
:100AE0002560187023688978581C20601970236865
:100AF0009278591C21601A702DE500BFE86400202F
:100B00007C4700202442002038590308E464002078
:100B1000906400206766666682380020BD4A002027
:100B2000105700207B5C0020985B0020745200204E
:100B3000C43E0020D43E002068590308E064002031
:100B4000575C00200A68AC4BAC491878551C2560EE
:100B5000107022685878551C2560107022689B78A8
:100B6000501C206013702046C988F0F73BFBF2E46C
:100B700005A8F0F72FFA00283FF4EDACBDF81410EB
:100B80002046F0F72FFB23689DF81620591C2160A2
:100B90001A7023689DF81720591C21601A70236869
:100BA0009DF81820591C21601A7023689DF819209F
:100BB000591C21601A7023689DF81A20591C216065
:100BC0001A702046BDF81C10F0F70CFBC3E48C4BE8
:100BD00003F1700522681978501C2060117022689A
:100BE0005978501C2060117022689978501C206040
:100BF00011702268D978501C206011702268197910
:100C0000501C2060117022685979501C20601170AE
:100C1000226899790733501CAB4220601170D9D1FA
:100C200099E4784D0846E989F0F7DCFAA98920466D
:100C3000F0F7D8FA8FE40B68734D591C2A792160BC
:100C40001A7023686A79591C21601A702988204615
:100C5000F0F7C8FA2368AA79591C21601A706988CC
:100C60002046F0F7BFFA2368EA79591C21601A7010
:100C700071E40B6800255A1C0A60204629461D7045
:100C8000F0F799FA29462046F0F795FA29462046CA
:100C9000F0F791FA5FE45D4E0B6872795C4D591C78
:100CA00021601A702B682046198CF0F79BFA2B688C
:100CB0002046D98BF0F796FA71892046F0F792FA20
:100CC000B1892046F0F78EFA2B682046598CF0F750
:100CD00089FA2B682046998CF0F784FAF18920462E
:100CE000F0F780FA318A2046F0F77CFA2A68236808
:100CF00092F82620591C21601A702CE4434EF37898
:100D0000002B00F09A820B680822591C21601A708F
:100D100023680122991821601A7023683D4D591CDF
:100D20002A7921601A702368AA78591C21601A70E8
:100D300029882046F0F756FAE9892046F0F752FA5A
:100D40002368F279591C21601A702368EA78591CCB
:100D500021601A70FFF7FFBB16F08AFDFF280546D9
:100D600000F0828208A8002300F80C3D16F052FD26
:100D70002268294B511C2160157022681978501C7B
:100D80002060117022685978501C20601170226810
:100D90009978501C2060117022689DF81410501C26
:100DA0002060117020469988F0F71CFAFFF7D3BB3A
:100DB0000B681A4D591C012221601A702368AA7809
:100DC000591C21601A7009F0B3FE2368144A1549B2
:100DD0005E1C26601870B1F90010B2F90000F0F73F
:100DE00025FC23685A1C2260187029882046F0F7D9
:100DF000F9F9FFF7B0BB00BFBC3E00207C470020E4
:100E0000E4420020C43E0020944700207452002099
:100E1000E464002010570020504B00206E6000203A
:100E2000223D0020283D002020460021F0F7DAF97D
:100E300020460021F0F7D6F920460021F0F7D2F93C
:100E40002368B14D00265A1C22601E7023682A6850
:100E5000591C92F82C2021601A7023682A68591CAA
:100E600092F8362021601A7023682A68591C92F87B
:100E7000372021601A7023685A1C22601E70236874
:100E80005A1C22601E7023685A1C22601E702B6838
:100E90002046598FF0F7A6F92B682046198FF0F7F6
:100EA000A1F923682A68591C92F82E2021601A7033
:100EB00023685A1C22601E702B682046598EF0F75A
:100EC00091F92B682046998EF0F78CF9FFF743BB18
:100ED0008E4D8F4E9FED8F8ADFF88082DFED8E8AF8
:100EE00005F120070EE0FCEEE77ACDED017ABDF8C2
:100EF000041020460435F0F775F9BD4206F11806D6
:100F00003FF429AB717C0029F3D0844BD5ED007AF6
:100F10001B78012BE7D1824B1B68DB0440F18381F6
:100F2000F5EE407AF1EE10FA40F0B18140F2DC517A
:100F3000DFE7084610227B49F0F726F9FFF70BBBE5
:100F4000794B9B8AB3F5006F00F27581B3F5806F22
:100F500000F29B81B3F5007F34BF01270227734D58
:100F600005F10C0655F8041B91FBF7F1204689B2F8
:100F7000F0F738F9AE42F5D16D4D6E4F05F10C0624
:100F8000B5EC010AD7ED077A80EE270A23F0A4FB1F
:100F900081B22046F0F726F9AE42F1D1664D05F157
:100FA0000C0655F8041B204689B2F0F71BF9AE4237
:100FB000F7D1FFF7D0BA614D08462988F0F712F94A
:100FC000A9882046F0F70EF929892046F0F70AF99A
:100FD000FFF7C1BA0B685A4D01269A190A601E70B4
:100FE00010F07EFD002840F03481564B2268511CE1
:100FF00021601070226841F2B410511C185C21600D
:1010000041F27811107059582046890AF0F7D3F848
:10101000A96A20464908F0F7CEF8FFF79CBA0B689A
:10102000494A4A49D0784A4A5D1C256018702368AD
:101030004979581C206019702368D278591C2160A6
:101040001A70FFF788BA0020FFF786BA23685A1C87
:101050002260197029882046F0F7C4F82368EA78DE
:10106000591C21601A7023682A79591C21601A7052
:101070002368AA79591C21601A7023686A79591C5F
:1010800021601A70FFF76ABBDFF8D4A000254FF08B
:10109000A8080135C5F1200208FA02F2A5F12003E3
:1010A0002AFA05F6164328FA03F31E43282D06F004
:1010B00001024FF000030BD01343EAD0E8B20FF067
:1010C000B9FB0028E5D0294605A8F0F701FCE0E7C8
:1010D000204B1B78DA0700F1C28000251E4E2F46F8
:1010E00002E00135282D3DD029463046F0F7FFFBC0
:1010F0000028F6D0294605A8F0F7F9FB002840F0B3
:101100008D800137EDE700BFE46400202439002022
:10111000505600200000404200E082443457002036
:10112000105500201439002098640020C864002065
:101130000455002088520020C4470020A82F00201A
:10114000B0860020CC660020C43E00202C66002023
:10115000D43E0020484B0020D08F0020DB9B9141E3
:1011600090E33FF46E4B6F4DB3F850102046F0F70C
:1011700039F86D4B1988204689B2F0F733F86B4B7C
:1011800019684B0103F02002C1F340031343C1F37C
:10119000800243EA4203C1F3C00243EA8203C1F37F
:1011A000401243EAC20301F0100119432046F0F750
:1011B00019F803A904222046EFF7E6FF23682978EF
:1011C0005B4A581C2060197011886429A8BF6421EB
:1011D0002046F0F707F8B9F1960F4BD000212046D2
:1011E000F0F700F82168B7F1190348BFA7F112031F
:1011F000A3F3C4034A1C226020461A460B7004A9BC
:10120000EFF7C2FF23684B4A581C11212060197068
:1012100020461168EFF7CFFFFFF79DB9394603A8C5
:10122000F0F756FB6DE7F4EEC87AF1EE10FA52DAF9
:101230004FF47A715DE6082791E60B68B1783E4A73
:10124000581C2060197023681278591C21601A708C
:1012500063E595F82420394BAABB3046C6E6059BCA
:1012600043F00103059338E723685A1C2260187085
:10127000FFF771B923680322591C21601A70236893
:101280006A78591C21601A70ACE7042767E6F4EE0F
:10129000C87AF1EE10FA3FF549AEF4EEE87AFDEEC9
:1012A000E77AF1EE10FA17EE901A2BD86FF4F97373
:1012B000303903FB01F140F2E73391FBF3F101F226
:1012C000DB5189B215E65978022916D003290CBFE3
:1012D000042030468AE6FDEEE77A40F2E73217EE68
:1012E000903A303B02FB03F388FB0312D917C1EBA2
:1012F000622101F2E93189B2FBE5042A34BF022000
:10130000032073E640F2F313A1F5836103FB01F1BF
:1013100040F2E73391FBF3F101F2DD5189B2E8E5E8
:1013200058010020948C0020643100208C6400203F
:1013300068310020DC640020B83E0020CC6600202C
:1013400038B5094D2B8823EA0000834228800AD053
:10135000064B1421FF220E2002241C7059709A7033
:101360001FF03CFE288838BDE064002008450020BE
:1013700038B5094D2B881843834228800AD0074B83
:101380001421FF220E2002241C7059709A701FF045
:1013900025FE288838BD00BFE064002008450020F5
:1013A000024A136818431060704700BFDC640020D5
:1013B0006A4B6B4870B55822012500211D7024F03E
:1013C00048F9684A6849694C694800230B60136012
:1013D00000F01AFD2946052000F066FD6579291CFC
:1013E0004FF0070018BF012100F05EFDA679311C07
:1013F0004FF0080018BF012100F056FDA37A002B22
:1014000000F081805B4C002D40F08A80311C18BFB9
:101410000121092000F048FD2168574EC1F34051D9
:101420000E2000F041FD3168CA0700F18980504D5F
:1014300011F0020176D1003118BF0121032000F024
:1014400033FD4E4A4E4B128C93FBF2F3642BB8BF24
:10145000642301210420C5F8143100F025FD494B17
:101460000620197800F020FD01210A2000F01CFD63
:1014700021680B20C1F3404100F016FD21680C20CB
:10148000C1F3802100F010FD21684B0508D53E4BCB
:101490001B7A083B012B9CBF4FF4FA63C5F88032DE
:1014A000C1F300410D2000F0FFFC21680E20C1F3C4
:1014B000405100F0F9FC21680F20C1F3804100F099
:1014C000F3FC21681020C1F3C06100F0EDFC0121A4
:1014D000112000F0E9FC0121122000F0E5FC0121BF
:1014E000132000F0E1FC294B1968B3F8464029B1FC
:1014F0000BF024FC014608B9C4F3C0011420BDE878
:10150000704000F0D1BCE37A1A4C002B7FF47BAF23
:10151000216811F480213FF47CAF002D3FF476AFB9
:10152000012176E70121022000F0BEFC184B316852
:10153000DB6A642BB8BF642301F00201AB677AE772
:10154000144B0B4D1B68642B4FF00101B8BF642393
:1015500008466B6400F0A8FC316869E71828002091
:10156000C02700201C280020BC2700207C6400200D
:1015700058010020105500208C640020888600202F
:1015800040420F00E03500205C860020B041002082
:10159000986400200055002030B4034600F1240573
:1015A000064C07CC0C3343F80C0C43F8081C43F8EA
:1015B000042CAB42F4D130BC704700BF745903080F
:1015C000034B33F80C2F02809B788370704700BF69
:1015D00074590308084B196861B130B45D68074C51
:1015E000642202FB05F2B2FBF1F2228030BC002043
:1015F00018605860704700BFF02600206831002056
:101600000B4A136803605368436030B59368094C14
:1016100083601421002301FB03429579AD0602D5B6
:101620001379C37230BD0133092BF4D130BD00BF33
:1016300083590308047E0308704700BF6F4B1B7873
:10164000002B3AD02DE9F0416D4B6E4D9B79AC6883
:10165000A860013B82B0041B032B00F29C80DFE8F2
:1016600003F04A0231290FF0EBF8002800F09B80CC
:10167000654B66491B78B5F84220D1ED037AEA64E0
:10168000DB0700F1AA8002FB04F007EE900ADFED11
:10169000606A604BB8EEE77AD5ED127A5A60E7EEF1
:1016A000267A1A60BDEEE77AC5ED127A85ED117AD9
:1016B00083ED027A02B0BDE8F081564A13605360B0
:1016C00093607047544B1B681801F3D5FF2013F04B
:1016D0008BFA03780A2B88BF00214E4B9CBFB0F9D0
:1016E0000420B0F90610296588BF0A466A655A6069
:1016F0001A609960DEE7494A494BD279DFF83081B8
:1017000033F81220B8F902304648B8F9001092B206
:1017100007EE902A40F6E44707FB02F6C3EB1633C8
:10172000B8EE670A4FF47A7606FB03F393FBF1F306
:10173000AB61EEF7DFFED5F818E0D5ED047ADFED0A
:10174000346AB8F90220334BB8F900C0C3F804E09A
:101750000EFB04F007EE100AB8EEC77ABCEEC06AC2
:10176000E7EE267A8DED016ABDF80410C5ED047A26
:10177000BDEEE77A07FB01F7C2EB173706FB07F66A
:1017800083ED027A96FBFCF685ED037A6E611E60AE
:1017900002B0BDE8F0811F4B00221A605A609A60C7
:1017A00002B0BDE8F0811C4B1B68DE067FF560AF20
:1017B000154BB5F842201B78EA64D9077FF563AF73
:1017C000B5F94010184B00FB01F083FB0013C01764
:1017D000C0EBA3100244EA6455E7FDEEE77A134E2E
:1017E00017EE900AA0F57A7101FB01F386FB030660
:1017F000D817C0EB26100844E2E700BFFE4B0020DC
:101800007C640020F0260020484B0020004C002083
:101810002FE33E31BC6200201055002028850020B7
:10182000488500200C270020D34D62101F85EB5106
:10183000B43E0020F0B53E4B5B79012B83B03DD028
:10184000022B0FD03B4B00221A805A803A4B1B7858
:10185000022B05D1374A394B5188128819805A809A
:1018600003B0F0BD364B1B681B01EFD5FF2013F012
:10187000BBF903780A2B56D8B0F902203149D317A7
:1018800081FB0212C3EBA2039BB207EE903AB8EEC3
:10189000670A2D4C04F15C00A4F85A30EEF72AFEDA
:1018A000FCEEC07A234AB4F85A30CDED017A538069
:1018B000BDF80430A4F858301380C7E7234A244BFE
:1018C0009278214D33F81240A4B207EE904A05F108
:1018D0008400B8EE670AEEF70DFE1E4A154910782F
:1018E00096785378FCEEC07A00EB4010CDED017A8B
:1018F000BDF8042044F6FB77C3EB033300FB027210
:1019000000FB0474B2FBF3F2B4FBF3F3B2FBF6F2A8
:10191000B3FBF6F392B29BB2A5F88020A5F8823013
:101920000A804B8092E79FED0C0A0023B1E700BFCD
:101930007C640020E84B0020DC4A0020E04A0020C4
:101940001055002067666666F02600202885002076
:10195000488500200B8D002000000000F8B52D4DBB
:101960002D4968792D4C2E4B2E4E042264270A7087
:1019700001284FF0000184F8A82084F8B170A4F881
:10198000AA10A4F8AC1084F8B010C4F8B4103170E8
:101990001980598021D0022810D0A979224A002329
:1019A0000129136084F8B8305360936023D0022972
:1019B00012D11E4A636453609360F8BD282204F17B
:1019C000580023F046FE4CF250319FED190A04F105
:1019D0005C00EFF739FEE0E7F8BD282204F1800053
:1019E00023F037FE4CF250319FED110A04F18400D0
:1019F000EFF72AFED1E70F4AE36053609360D360AC
:101A00009FED0D0A02F110004CF25031BDE8F84094
:101A1000EFF71ABE7C640020785B0020F0260020DF
:101A2000E84B0020FE4B0020BC6200203427002041
:101A3000CDCCCC3DFC260020CDCCCC3EF8B5264C00
:101A400094F8B930002B46D094F8BA30002B42D02D
:101A500094F8BB3003F0FF07002B3CD1D4F8BC3026
:101A6000C31A002B37DB1D4B1D491B780625013B94
:101A700005FB03120A26128CB2FBF6F2D4F8C06002
:101A800006F1010E0E4405FB031196F82E60CB8B78
:101A9000C4F8C0E0724318441044BEF10E0F88BF72
:101AA000C4F8C070C4F8BC00F2F7B1FB012384F89D
:101AB000BB300C4BD4F8C4201B8AD4F8C810536038
:101AC00000234B620B889BB243F001030B80136829
:101AD00043F001031360F8BDF026002000870020CA
:101AE000745903080C870020044B587920B1044B2B
:101AF0001878003018BF0120704700BF7C640020B8
:101B0000FE4B00201F4B1878002839D01E4A13893D
:101B1000FBB11E4A9FED1E6AD2ED026A07EE903AB3
:101B2000F8EEE66AF8EE677A07EE103A77EEE66AC4
:101B3000B8EEC77A66EE866AC6EE877AFDEEE77A79
:101B400017EE900A6428A8BF642020EAE070C0B2B3
:101B5000704710B40F4B54781B88117804FB103277
:101B6000091B642300FB01F003FB02F3B3FBF0F05D
:101B70006428A8BF64205DF8044B20EAE070C0B27E
:101B8000704700BFFE4B00207C640020BC62002038
:101B90000000C842E84B00202DE9F04F794D81B09C
:101BA000F3F714FCD5F8D0400022C5F8CC20002C67
:101BB00000F0A580237D052B074617D9216A2369EC
:101BC0000B44C31A9342B8BF05F1D0010ADBD5E03C
:101BD000137D052B0AD9136A12691344FB1A002BD3
:101BE00080F2CC8051F8042F002AF1D14FF0010B84
:101BF0000023B9461E46C5F8CC3098469A4627467B
